:1000000000560020C565000015650000256500004C
:100010003D650000556500006D65000000000000B2
:1000200000000000000000000000000085650000E6
:100030009565000000000000A5650000B5650000A2
:10004000FD6400000000000000000000590D0100E8
:10005000890C0100050D01000000000000000000F7
:10006000D543000051F1000031F10000A10D010065
:10007000000000000000000000000000C10D0100B1
:100080002DE9F843054688464FF0A0441C4EDFF8A2
:1000900078901C4F237E002BFCD1A37E2BB94FF010
:1000A00001022274A37E002BFBD072B6735DF3B9FC
:1000B00000F02EF8C0B90122D9F8103043F0040343
:1000C000C9F8103087F83220BFF34F8F00BF30BF20
:1000D00087F83200D9F8103023F00403C9F8103043
:1000E000BFF34F8F62B6D5E700BF30BFFAE70023FA
:1000F0007355B8F1000F00D0C04762B6BDE8F88371
:10010000D82800200000105000ED00E000000000A2
:100110005FF800F01D430000FFFFFFFFFFFFFFFF40
:10012000FFFFFFFFFFFFFFFFFFFFFFFFFFFFFFFFDF
:10013000FFFFFFFFFFFFFFFFFFFFFFFFFFFFFFFFCF
:10014000FFFFFFFFFFFFFFFFFFFFFFFFFFFFFFFFBF
:10015000FFFFFFFFFFFFFFFFFFFFFFFFFFFFFFFFAF
:10016000FFFFFFFFFFFFFFFFFFFFFFFFFFFFFFFF9F
:10017000FFFFFFFFFFFFFFFFFFFFFFFFFFFFFFFF8F
:10018000FFFFFFFFFFFFFFFFFFFFFFFFFFFFFFFF7F
:10019000FFFFFFFFFFFFFFFFFFFFFFFFFFFFFFFF6F
:1001A000FFFFFFFFFFFFFFFFFFFFFFFFFFFFFFFF5F
:1001B000FFFFFFFFFFFFFFFFFFFFFFFFFFFFFFFF4F
:1001C000FFFFFFFFFFFFFFFFFFFFFFFFFFFFFFFF3F
:1001D000FFFFFFFFFFFFFFFFFFFFFFFFFFFFFFFF2F
:1001E000FFFFFFFFFFFFFFFFFFFFFFFFFFFFFFFF1F
:1001F000FFFFFFFFFFFFFFFFFFFFFFFFFFFFFFFF0F
:10020000FFFFFFFFFFFFFFFFFFFFFFFFFFFFFFFFFE
:10021000FFFFFFFFFFFFFFFFFFFFFFFFFFFFFFFFEE
:10022000FFFFFFFFFFFFFFFFFFFFFFFFFFFFFFFFDE
:10023000FFFFFFFFFFFFFFFFFFFFFFFFFFFFFFFFCE
:10024000FFFFFFFFFFFFFFFFFFFFFFFFFFFFFFFFBE
:10025000FFFFFFFFFFFFFFFFFFFFFFFFFFFFFFFFAE
:10026000FFFFFFFFFFFFFFFFFFFFFFFFFFFFFFFF9E
:10027000FFFFFFFFFFFFFFFFFFFFFFFFFFFFFFFF8E
:10028000704700BF034613F8012B002AFBD1181A50
:1002900001387047004870477CE201003520704704
:1002A0000820704708B506F095F808BD08B506F0B7
:1002B00021F943690148984708BD00BF7CE201006D
:1002C00010B50C4611461A46012807D010B1022875
:1002D0000BD010BDE0B200F047F8FAE7BDF80830E7
:1002E000C9B2E0B200F082F8F3E7E0B200F040F902
:1002F000EFE700BF054B00229A80DA805A819A818D
:10030000B42119811A765A769A767047E42900202A
:10031000014B1878704700BFE429002010B4044650
:10032000034B0FCB84E80F00204610BC704700BF82
:10033000E82900200346054901F1140248691860C4
:10034000098B927999809A7118467047E4290020A8
:10035000044B187E012803D0987E003018BF01207E
:10036000704700BFE429002010B504461D4B1B78E0
:1003700013F0030F02D010F00C0F15D114F0030F7F
:100380001CD113F0080F02D014F0040F22D113F087
:10039000040F15D014F0080F12D0124B00229A80CF
:1003A000DA80B4221A810BE006F014F802690D4BD2
:1003B0001A61FFF79FFF00F013F901E0FFF79AFFC2
:1003C000084B1C70084C204600F08AFE204600F0C6
:1003D00037FB10BD034B00229A80DA80B4221A81C9
:1003E000EEE700BFE429002084E2010010B50446D6
:1003F00000F09EFF042C00D010BDFFF789FF10F025
:100400000C0F05D000F0A5FF4368984700F0F2F804
:10041000534C204600F0B2FE204600F0B7FB514B93
:100420001A78042A30D0082A43D04E4B5B89B3F5A2
:10043000616F05D34B4B0021598199890131998115
:10044000484B99894EF6602399424AD0454BD9884A
:100450004EF66023994248D0424B99884EF660236D
:10046000994246D012F0080F47D13E4B1B8BB3F593
:10047000807F70D03B4B9B7E13B1013B394A937612
:10048000384B1A7E5A76B7E73649CB8801339BB290
:10049000CB803549A1FB0301490901EB8101A3EBA5
:1004A000C1039BB2002BC0D12E494B8901334B8134
:1004B000BBE72C490B89013B0B818B8801339BB235
:1004C0008B802A49A1FB03014909C1EB0111A3EB70
:1004D00081039BB2002BA8D122494B8901334B8168
:1004E000A3E7204B00219981B0E71E4B0021D98062
:1004F000B2E71C4B00219980B4E700F02AFF436863
:1005000098470368984760B9164B1B7813F0080F9B
:10051000ABD0134800F06CFE78B1124BB4221A81B4
:10052000A3E700F016FF4368984700F0B2FD0128EA
:10053000EAD10C4BB4221A81E6E70A4B1B7813F080
:10054000080F92D0074B1B89002B8ED105F0D2FFEC
:100550000368984789E7034B06229A7690E700BF25
:1005600084E20100E4290020CDCCCCCC89888888A5
:1005700010B5072819D8DFE800F019041D2018234A
:10058000262C05F027FF044605F0B4FFC3684FF49E
:100590008062002120469847FFF7ACFE0E4800F02D
:1005A0009FFD04F1F00000F038FA10BD0A4800F099
:1005B000BBFDFAE7094B1975F7E7084B5975F4E7E6
:1005C000064B9975F1E7054BD975034800F088FD96
:1005D000EBE7024B1976E8E784E20100E42900200A
:1005E00008B580220021024819F087FC08BD00BF31
:1005F000002A00202DE9F04F85B082460022924962
:1006000011F832306FF3C71301F8323001EBC20337
:1006100058786FF3C710587098786FF3C7109870B8
:10062000D8786FF3C710D87018796FF3C7101871A6
:1006300058796FF3C710587198796FF3C710987194
:10064000D8796FF3C710D8710132102AD8D1DAF8EF
:100650000030984703900023029345E04FF00108D3
:100660004FF0140CB5423AD801974FF04C0933467D
:10067000464698462BE04FF001084FF0140CF1E786
:10068000425C42F08002425402F07F0202EB0C0B0B
:10069000BBF14C0F0FDD425C69F30602425401339B
:1006A0009BB29C420FD319461EF80320D209E7D013
:1006B000002EF4D0E4E7624410F801B062F3060BB8
:1006C00000F801B0EBE70135ADB2A84507D3A7426A
:1006D000F9D8019B5C4A02EBC50E7046E3E7029B2A
:1006E000013302930A2B66D09DF80880DAF828308F
:1006F00040469847012805D0DAF828304046984708
:100700000228ECD1DAF80C30404698478146DAF8F6
:10071000103040469847834603014C4A82FB03262B
:10072000F218DE17C6EBE2264FEAC903484A82FBFD
:1007300003271F44DB17C3EBA727DAF8183040461E
:100740009847DAF8083040469847002814BF10242C
:100750000424B6B2351B25EAE575ADB226440F2E4A
:10076000A8BF0F26B6B2BBB21F1B27EAE777BFB2FE
:100770001C44072CA8BF0724A4B2DAF8083040466E
:100780009847A9F143091FFA89F940F2B233994514
:100790003FF664AFBBF16E0F7FF66DAF002814BF5C
:1007A0004FF0140C4FF0010C002814BF4FF001085B
:1007B0004FF0000856E70026234F1FE0043AE55C9F
:1007C00062F30605E55404E0013AE55C62F30605D0
:1007D000E5540133082B0ED0C25CD209F9D1C25CBA
:1007E00002F07F02122AEFD8032AE7D8E25C6FF307
:1007F0000602E254EDE70136102E04D0002307EB89
:10080000C6000446E8E7039B1BB1002421460E4DB9
:1008100005E0FFF7E5FEF8E70134102C0DD00023CA
:1008200005EBC400C25C02F07F02092A84BF0131DB
:1008300089B20133082BF5D1EEE7034BA3F8801002
:1008400005B0BDE8F08F00BF002A0020E1000EE0F7
:1008500049D6B9F22DE9F04F83B00646019114460E
:100860000368984770B13E4A92F88230013382F8AB
:100870008230A146002C5ED00027B8469346DFF8B0
:10088000E8A037E0FFF7ACFE4FF00008019B83F8CB
:10089000008055E0F3682046984740B3336920460E
:1008A000984720B3F36820469847054633692046A9
:1008B000984700018AFB00230344C017C0EBE320E4
:1008C00080B2ED00274B83FB05232B44ED17C5EBCE
:1008D000A325ADB20BEBC000435D03F07F03122BE9
:1008E00005D808F101085FFA88F8019B1C700137F0
:1008F0004F4510D0FCB2B36A204698470128C9D0B2
:10090000B36A204698470228C4D0B36A2046984765
:100910000328ECD1BEE7B8F1000F0CD0104BB3F8B0
:100920008030402B10D8B8F1010F09D012D9002324
:10093000019A137004E04FF00008019B83F80080D7
:10094000404603B0BDE8F08F4FF00008019B83F8EC
:100950000080F5E74FF00008019B83F80080EFE787
:10096000002A002049D6B9F2E1000EE0431E9BB2F6
:100970004FF6FD7293421CD84B1E9BB293421AD87D
:1009800009010E4B83FB01231944C1F3CF21C000A1
:100990000B4B83FB00231844C0F38F20094B03EB60
:1009A000C101085C00F07F0013288CBF00200120EB
:1009B0007047012070470120704700BFE1000EE042
:1009C00049D6B9F2002A0020F8B506460F4C256832
:1009D000238903EB83035B00F4336B8005F08AFD0E
:1009E0000435238903EB830307690A22314605EBAB
:1009F0004300B847238901339BB223812268527890
:100A00009A4201D800222281F8BD00BF842A00202A
:100A1000704708B5FFF7D8FF08BD10B5044605F0CC
:100A200069FDC3684FF44472002120469847034B88
:100A30001C60462363700A23237010BD842A0020A3
:100A400030B5A5B00446436898474F4B1B7913F067
:100A5000030F09D0A368984710F0080F21D1A368AD
:100A6000984710F0040F1CD1474B1B7913F00C0F63
:100A700009D0A368984710F0020F41D1A3689847A6
:100A800010F0010F3CD1A36898473F4D2871E368EF
:100A900004A89847BDF81830EB8000236B8125B07F
:100AA00030BD002501950295ADF80C5005F022FDF2
:100AB000C3680A22294601A898479DF804300222FB
:100AC00062F302038DF80430E36810A89847BDF87C
:100AD0000430BDF8462062F30F13ADF80430E3682C
:100AE0000CA89847BDF83E30ADF80630E36808A87A
:100AF00098470B9BADF8083001A8FFF765FFB3E7F7
:100B0000002501950295ADF80C5005F0F3FCC36883
:100B10000A22294601A898479DF80430032262F36F
:100B200002038DF8043063689847BDF804300288EA
:100B300062F30B13ADF80430134A52891209C3F360
:100B4000072362F307138DF80530E36820A8984760
:100B5000BDF88230ADF80630E3681CA89847BDF8B0
:100B60007030ADF80830E36818A89847BDF86E30CB
:100B7000ADF80A30E36814A89847179BADF80C301D
:100B800001A8FFF721FF7EE7842A00202DE9F04F1E
:100B9000A9B0044643689847A368984710F0080F27
:100BA00004D1A368984710F0040F39D02368984700
:100BB00043689847054600F06CFA80B1236898476F
:100BC000436898478146002704970597ADF8187049
:100BD00002460A2104A800F048FAB846EEE028468A
:100BE00000F05BFA0028E9D163689847B0F86030FC
:100BF000002B40F07381B84BDD880135E36818A8FD
:100C00009847BDF868309D4200F0D781E3680EA890
:100C10009847B14BBDF84020DA805A8901325A8199
:100C200029B0BDE8F08FF368284698473369284615
:100C300098472368984743689847834600F035FAF9
:100C4000B0F1000AC0F2448163689847C388ADF8E8
:100C50000830636898470389ADF80A30636898479D
:100C60004388BDF808201344ADF80C3063689847FA
:100C70008388BDF80A201344ADF80E305FFA8AFA73
:100C8000DBF80C30504698470190DBF810305046A6
:100C9000984702AA0146019800F0C0F9002840F0E8
:100CA00019814FF4C973ADF8083040F66A03ADF806
:100CB0000A3040F2A623ADF80C3040F62413ADF80C
:100CC0000E30DBF80C30504698470190DBF81030BE
:100CD0005046984702AA0146019800F09FF900305B
:100CE00018BF01209DF8223060F345138DF82230A3
:100CF0006368984790F86330C3F302039DF824209B
:100D000063F302028DF824206368984790F866A088
:100D10000AF0FD0A6369984701280ED14AF0020AD9
:100D20006368984790F86830FF2B06D0636898474F
:100D300090F86830013380F868306368984780F82D
:100D400066A063689847BDF8243090F8662062F387
:100D5000C803ADF82430B368284698479DF825307D
:100D600060F382038DF82530B369284698471F2821
:100D700028BF1F20BDF8223060F38A13ADF822305F
:100D8000F369284698471F2828BF1F209DF8233065
:100D900060F3C7038DF82330336A28469847C0F3C1
:100DA0008F001F2828BF1F209DF8253060F3C70340
:100DB0008DF8253007A8FFF707FE0137D9F8003076
:100DC0009847FBB28342BFF40FAFFBB228AA13448B
:100DD00013F8905CCDF81C80CDF82080ADF824800D
:100DE000D9F8283028469847012805D0D9F8283066
:100DF000284698470328E0D12368984743689847D6
:100E00000646E3680AA89847BDF82CA005F072FBD7
:100E1000C3680A22414607A898479DF81C306FF323
:100E200002038DF81C30B36A28469847012814BF86
:100E3000002001209DF81C3060F3C3038DF81C30A6
:100E4000BDF81C30BDF82E2062F30F13ADF81C3036
:100E50004FEA1A129DF81E3062F303038DF81E301C
:100E60009DF820306AF303038DF82030F36828469C
:100E70009847BDF81E3060F30F13ADF81E3033698C
:100E800028469847BDF8203060F30F13ADF82030A6
:100E9000236912A898479DF822309DF8482062F3F4
:100EA00001038DF82230736A284698479DF8223056
:100EB00060F383038DF8223003F00C030C2B7FF4D6
:100EC000B2AE9DF8223043F00C038DF82230AAE632
:100ED000404607E7012005E7842A002000230A9303
:100EE0000B93ADF83030236898474368984706461F
:100EF00000F0DBF8051E4FDB05F0FCFAC3680A22A0
:100F000000210AA898479DF82830012262F30203C5
:100F10008DF82830E36814A89847BDF82830BDF84C
:100F2000562062F30F13ADF828306368984790F8A5
:100F3000603013F0020F3AD16368984790F8603040
:100F400013F0040F35D16368984790F8603013F0C0
:100F5000080F30D16368984790F8603013F0100F95
:100F600014BF062200229DF82A3062F303038DF895
:100F70002A30EDB2F36828469847BDF82A3060F36E
:100F80000F13ADF82A30336928469847BDF82C3046
:100F900060F30F13ADF82C300AA8FFF715FD636856
:100FA00098470023A0F860301B4A538123E60122B2
:100FB000D9E70422D7E70522D5E700250A950B9546
:100FC000ADF8305005F096FAC3680A2229460AA8FF
:100FD00098479DF82830042262F302038DF82830E8
:100FE000E36824A89847BDF82830BDF8962062F33E
:100FF0000F13ADF82830E36820A89847BDF88E306D
:10100000ADF82A30E3681CA898471F9BADF82C3038
:101010000AA8FFF7D9FCF9E5842A0020134672B12B
:10102000128882420DD89A8882420CD3DA888A428A
:101030000BD3588888428CBF0020012070470020C5
:10104000704700207047002070470020704710B59F
:101050000446084611460023224600F0BBF9002151
:10106000204600F0E4F9C0B210BD08B5002300F03E
:10107000B1F908BD08B500F0ADF908BD08B500210B
:1010800000F0D5F9C0B208BD08B500F0D0F9C0B283
:1010900008BD08B500F076F908BD08B500F086F97E
:1010A00008BD08B500F05AF908BD08B500F0E6F92A
:1010B00008BD000010B5436898470488003418BF85
:1010C000012405F017FA836822460321022098477D
:1010D00005F010FA8368224603210420984710BDCA
:1010E000F8B507460F4B1B68BBB1002425460D4ED3
:1010F00056F8253053B156F82530984703682BB180
:1011000056F8253098470368384698470134E4B2CA
:10111000254656F82430002BEAD13846FFF7CAFF9F
:10112000F8BD00BF1C120020F8B50746124B1B6823
:10113000F3B100242546104E56F825308BB156F8F1
:101140002530984743683846984750B156F82530BF
:101150009847C3682BB156F825309847C36838467E
:1011600098470134E4B2254656F82430002BE3D1E9
:101170003846FFF79FFFF8BD1C1200202DE9F04113
:1011800007461A4B1B68002B2DD000242646174D0E
:1011900005E00134E4B2264655F824301BB355F877
:1011A0002630002BF5D055F826309847436838464E
:1011B00098470028EDD055F82630984790F81480CD
:1011C000BB68984718EA000FE3D055F826309847D7
:1011D0008368002BDDD055F8263098478368384661
:1011E00098470028D5D0BDE8F08100BF1C12002030
:1011F0002DE9F04107461C4B1B68002B32D0002420
:101200002646194D05E00134E4B2264655F824304F
:101210002BB355F82630002BF5D055F826309847DB
:101220004368384698470028EDD055F8263098474F
:1012300090F81480BB68984718EA000FE3D055F87F
:10124000263098470369002BDDD055F826309847A3
:101250000369384698470028D5D0012000E00020D7
:10126000BDE8F0810020FBE71C12002008B54368B0
:1012700098470078C0F3400008BD704730B587B08C
:101280000446036898474368984702461F4903A8E5
:1012900000F0E9FC9DF8153013F0020F2ED0BDF8D8
:1012A0000C30CD3B9BB240F29D22934229D8BDF831
:1012B0000E2040F67B039A4225D99DF81430043B5A
:1012C000DBB2382B01D9002019E0002301930293EF
:1012D0004FF00203012565F387138DF8043005F004
:1012E00009F9436801A898476368984790F8603007
:1012F00043F0020380F86030284600E0002007B089
:1013000030BD0020FBE70020F9E700BF902A002055
:1013100008B54FF49F7354224021024800F08EFC20
:1013200008BD00BF902A0020004870479CE20100E1
:1013300010B51446012802D0022805D010BD1A4667
:10134000204600F081FDF9E71946104600F04AFDFD
:10135000F4E70148704700BFB4E2010038B5054624
:101360000368984748B10024AB68E0B29847034649
:1013700030B901340A2CF7D100E00023184638BDFB
:101380000123FBE738B505460368984750B10024B0
:10139000AB6AE0B29847012806D001340A2CF7D195
:1013A000002000E0002038BD0120FCE738B50546EC
:1013B0000368984750B10024AB6AE0B2984703280D
:1013C00006D001340A2CF7D1002000E0002038BDFF
:1013D0000120FCE72DE9F84F8246894616469846DB
:1013E00000252F4609E07B1CDBB20AF807404B457D
:1013F0001BD01F4601350A2D17D0ECB2B36A204628
:1014000098470028F6D0F36820469847834633690A
:1014100020469847B8F1000FE5D0424601465846AD
:10142000FFF7FCFD0028DED1E4E7BDE8F88F2DE9E9
:10143000F843074688460024264604E00136F6B203
:1014400001340A2C17D0E5B2BB6A28469847002819
:10145000F6D0FB682846984781463B69284698475E
:10146000B8F1000FEAD0424601464846FFF7D6FDE4
:101470000028E3D1E4E770B2BDE8F88338B505464B
:101480000368984760B10024AB6AE0B2984728B976
:1014900001340A2CF8D14FF0FF3038BD60B2FCE7C0
:1014A0004FF0FF30F9E7000008B54368984700782F
:1014B000C0F3C00008BD064B43221A80BE225A80EA
:1014C00040F2F5329A8040F6B502DA80704700BFEC
:1014D000AC2A0020F0B585B0044643699847244DF6
:1014E000A8762368984743689847024605F10801A3
:1014F00002A800F078FA9DF80830022B03D00025EE
:10150000284605B0F0BDBDF80A70BDF80C602A464B
:1015100031463846FFF782FD05460028F0D000230B
:10152000009301934FF00203042262F38503012527
:1015300065F387138DF8003047FA02F38DF8023017
:1015400046FA02F38DF8033006F00F0646EA071656
:101550008DF8046004F0CEFF4368684698476368DE
:10156000984790F8603043F0080380F86030C7E790
:10157000AC2A002010B584B00D4C4623039364239D
:1015800002931E230193032200921223012104F1EE
:10159000080000F001FA43232380BE23638040F259
:1015A000F533A38040F6B503E38004B010BD00BF5F
:1015B000AC2A002000487047BCE2010008B543682F
:1015C0009847037813F0240F14BF0120002008BDB2
:1015D00038B543689847C58804894188294482887A
:1015E0002244034B5D809C80D9801A8138BD00BFA6
:1015F000E42A00202DE9F04784B0804643689847EC
:101600000378C3F38009C3F34017D8F81430984720
:101610003F4D85F82600D8F8003098474368984732
:10162000024605F1140102A800F0DDF99DF808A0BA
:10163000BDF80A60BDF80C40AA1C21463046FFF7F1
:10164000EDFC30BB05F10A0221463046FFF7E6FC0F
:10165000034600285AD1184604B0BDE8F0872C4B49
:101660001A700023F7E71FB3294B1B78012B1FD0FB
:101670000023F0E7D8F80430984790F8603043F042
:10168000040380F860300123E5E70023E3E700234B
:10169000E1E70022BAF1010FE1D0BAF1020FF4D173
:1016A000B9F1000FDFD01FB9194B1B78002BEED119
:1016B000002301934FF00203012262F3850362F3DA
:1016C00087138DF80030124D2B788DF801303311CF
:1016D0008DF8023023118DF8033004F00F0444EA32
:1016E00006168DF8046004F005FF436868469847C5
:1016F0002B78002BBED0D8F80430984790F8603093
:1017000043F0200380F860300123A4E70122C1E701
:10171000E42A002030B587B00546036904A898473D
:101720009DF81330FBB9264C4623039364230293A0
:10173000242301930523009312230222114604F16E
:10174000140000F029F96B689847C5880189428820
:101750002A4483880B446580A180E28023816F2125
:1017600040F6F4021FE0164C0A230393642302930D
:10177000242301930723009312230322022104F15F
:10178000140000F009F96B689847C5880189428800
:101790002A4483880B446580A180E280238140F243
:1017A0002C4140F66602064B43205881998140F255
:1017B000F531D9811A8200221A7007B030BD00BFFE
:1017C000E42A002000487047D4E2010010B5044626
:1017D000028B038A9A4202D90123C375037594F8D8
:1017E0002730012B12D0A37C012B14D0A27D0D4BEE
:1017F00053F8223020469847012811D0022814BF00
:1018000000200220A38D0133A38510BD0423E375BE
:1018100001232375E7E70523E37501232375E5E736
:101820000120EFE72C120020C289B0F91A30B0F97C
:1018300022105B1A002BB8BF5B42934218DCB0F950
:101840001C30B0F924105B1A002BB8BF5B429A42DF
:1018500010DBB0F9282043889A4207DCB0F92C301D
:1018600040898342CCBF0020012070470020704790
:10187000002070470020704770B5044690F826504D
:10188000012D05D9AB1EDBB2012B08D9002070BD9C
:10189000012303750020A0750323E375F7E7068D88
:1018A000013636B20685FFF7BFFF08B9012323755D
:1018B000032D01D00020EAE723889E42BCBF01230C
:1018C000237563889E42C4BF012323750023A3753B
:1018D000627D237B9A4201D00020D8E7B4F92A30F8
:1018E000A2889342BCBF01222275E2889342C4BF02
:1018F00001232375B4F92C3022899342BCBF012205
:10190000227562899342C4BF012323750023638536
:10191000237D4BB100202075A685E38B6383238C48
:10192000A38301236375B2E7002363750220AEE74A
:1019300010B5044690F8263023B9438D0133438512
:10194000002010BD012B25D1FFF76EFF18B902232F
:10195000E3750123237501222285637D1344DBB2E5
:101960006375A275B4F92210E183B4F924202284AE
:101970003BB1237D2BB9607D012814BF00200120DD
:10198000DFE7002020750123A38560856183A283A2
:101990006375F0E70020D4E730B4BDF80850BDF817
:1019A0000C400280438001FB02F292B2AB1A8380AA
:1019B000A21AC280058144810173BDF81030C38131
:1019C000BDF8143003820023037543754385838576
:1019D0000385C3754FF6FF7242838283C2830284FC
:1019E000837530BC7047F0B585B005460C46164689
:1019F000002301930293ADF80C30898B608BFEF7C6
:101A0000B5FFD0B10A2201A93046FEF723FF012815
:101A100022D90023237563756385A3852385E37528
:101A20004FF6FF726283A283E2832284A3752B7038
:101A30006B80AB80284605B0F0BD0023237563752D
:101A40006385A3852385E3754FF6FF726283A283C6
:101A5000E2832284A375D5E79DF8047000B3F36890
:101A6000384698476084336938469847A084B36AFB
:101A70003846984784F82600B3693846984720834B
:101A80003046FFF70EFBA0B9002384F8273020462C
:101A9000FFF79CFE628BA38B28706A80AB80C9E73E
:101AA0004FF6FF736384A384002384F826302383D6
:101AB000E6E7012384F82730E9E700BF70B5044664
:101AC0000E4615788B6A28469847012801D00120D8
:101AD00070BD002323806380A380E3802381638122
:101AE000A381E38123746374227E02F0F80263F31E
:101AF000C3022276F36828469847A08133692846B6
:101B00009847E081237C01332374E0E72DE9F0411D
:101B100004460F461678CB683046984780463B69A6
:101B2000304698470546BB6A30469847032841D05F
:101B3000A389A8EB03031BB22380B4F902209A42C5
:101B4000B8BF1A4616466280B4F904709F42A8BF17
:101B50001F46A780E089281A00B2E080B4F9082067
:101B60008242B8BF02462281B4F90A108142A8BF5E
:101B700001466181B4F9125001EB050C604553DA5E
:101B8000491B884250DD521B904203DC227E42F00A
:101B900002022276EA1993424BDA7F1BBB4248DDF0
:101BA000721B9342DEBF237E43F00803237601209D
:101BB000BDE8F08100232374B4F90020E38A9A423F
:101BC00022DB217E01F00801002914BF0020102033
:101BD00059428A4206DC227E12F0040F04BF40F014
:101BE0000800C0B2B4F9062093420FDC237E13F044
:101BF000020F0BD140F00400C0B29142D8DB237E2B
:101C000013F0010F08D0D3E70020E1E7914207DB92
:101C1000237E13F0010F03D140F00200C0B2C7E7EA
:101C2000002808BF0120C3E7217E41F00101217691
:101C3000A9E7227E42F004022276B1E74182828245
:101C4000C3820023038043808380C3800381438158
:101C50008381C38103744374027E02F0F80263F34C
:101C6000C302027670472DE9F04186B004460D4666
:101C7000164600238DF81730314903AA03C982E8BC
:101C8000030000930193ADF808300A2269463046FC
:101C9000FFF7DDF980469DF800708DF81770B36A84
:101CA00038469847002831D0B8F1010F2ED1B369DA
:101CB00038469847AB8A834228D3B368384698475A
:101CC00020BBF3689DF817009847804633699DF85C
:101CD0001700984707462B7C06AA02EB830353F8AC
:101CE0000C3C0DF11702314628469847A989EA892C
:101CF0006B7C5E1C6E7421806280A4F80480E78097
:101D000023726072204606B0BDE8F08100232B806C
:101D10006B80AB80EB802B816B81AB81EB812B7473
:101D20006B742A7E02F0F80263F3C3022A762380E2
:101D30006380A380E380237201236372E2E700BF24
:101D4000ECE20100014B1888704700BF282B0020EF
:101D50000A207047024B5B6803EB0010807B7047E2
:101D6000282B0020024B5B680001185C704700BF05
:101D7000282B0020024B5B6803EB00104088704763
:101D8000282B0020024B5B6803EB00108088704713
:101D9000282B0020024B5B6803EB0010C0887047C3
:101DA000282B0020024B5B6803EB00100089704772
:101DB000282B0020024B5B6803EB00104089704722
:101DC000282B0020024B5B6803EB001080897047D2
:101DD000282B0020024B5B6803EB00104078704713
:101DE000282B0020014B198058607047282B0020B9
:101DF00000487047F4E2010001EB4011024B1B6800
:101E000033F91100704700BF302B002001EB401167
:101E1000024B5B6833F91100704700BF302B002084
:101E200001EB4011024B9B6833F91100704700BF72
:101E3000302B002001EB4011024BDB6833F911001D
:101E4000704700BF302B0020014B43F82100704742
:101E5000302B0020014B03EB8000704720E3010092
:101E6000004870471800002000487047E404002034
:101E700010B5064C04F110000DF0D8F8207504F1EF
:101E800018000DF0D9F82077204610BD4C05002031
:101E9000024A4FF4F071024809F058BE2CAB010021
:101EA0002C0500200149024809F0DCBE2CAB0100E2
:101EB0002C050020024A4021024809F047BE00BF1D
:101EC00040AB0100700500200149024809F0CABE7C
:101ED00040AB0100700500200048704788050020D5
:101EE000704700BF704700BF10B5054C04F10C00EF
:101EF0000DF09CF8E36820752361204610BD00BFFB
:101F0000D8050020004870473000002070B54678A2
:101F10000C4CB500294604F114000B4A09F016FEDA
:101F200031462046094A09F011FE2946201D084A7B
:101F300009F00CFE294604F10800064ABDE870408D
:101F400009F004BE1406002030AC010044AC0100CE
:101F500060AC01007CAC010010B50A4C0A4904F1E8
:101F6000140009F07FFE2046084909F07BFE201D81
:101F7000074909F077FE04F108000649BDE8104062
:101F800009F070BE1406002030AC0100DCAB01008B
:101F9000F4AB01000CAC010010B5054C04F10C00D1
:101FA0000DF044F8E36820752361204610BD00BFA2
:101FB00034060020004870474800002010B5074C48
:101FC000074A04F108000C2109F0C0FD2046BDE8D5
:101FD0001040044A062109F0B9BD00BF7006002078
:101FE000A8AC0100C0AC010010B5064C064904F1D4
:101FF000080009F037FE2046BDE81040034909F00B
:1020000031BE00BF70060020A8AC0100C0AC0100CA
:1020100000487047A0050020704700BF704700BF10
:1020200010B5064C04F10C000DF006F8207504F113
:1020300010000DF007F8204610BD00BFA8060020D4
:10204000004870476000002070B506780C4CB50061
:10205000294604F114000B4A09F078FD3146204668
:10206000094A09F073FD2946201D084A09F06EFD52
:10207000294604F10800064ABDE8704009F066BD33
:10208000E40600203CAD010050AD010068AD010048
:1020900080AD010010B50A4C0A4904F1140009F0A2
:1020A000E1FD2046084909F0DDFD201D074909F042
:1020B000D9FD04F108000649BDE8104009F0D2BD81
:1020C000E40600203CAD010050AD010068AD010008
:1020D00080AD010010B5064C04F10C000CF0ACFF13
:1020E000207504F110000CF0ADFF204610BD00BFBC
:1020F000040700202DE9F0410CF094FF0446FFF79F
:10210000B7FE0546FFF748FF0746FFF7E3FF224605
:1021100006462946012001F04BFE224629460220B0
:1021200001F046FEFFF7E0FE8046FFF779FF054627
:1021300022464146092001F03BFE224629460A205C
:1021400001F036FE22463946052001F031FE2246D6
:102150003146062001F02CFEFFF79AFEBDE8F04163
:10216000FFF7A8BE10B5FFF7C5FF094B1B689847DE
:10217000084B1B689847084B1B689847BDE8104000
:10218000064A074B127853F822305B68184700BFA5
:1021900090110020F4100020BC1000205D160020DB
:1021A00030AE010070B5FFF763FE0446FFF7F4FEA2
:1021B0000646FFF78FFF0546FFF774FEFFF784FE24
:1021C0002146012001F042FE2146022001F03EFEA0
:1021D0003146052001F03AFE2946062001F036FE80
:1021E000FFF782FE0546FFF71BFF0446294609203C
:1021F00001F02CFE2146BDE870400A2001F026BE09
:1022000070B500249CB011AE214630462C220BAD97
:10221000CDE90B44CDE90D440F94ADF8404017F0E3
:102220006CFE08ABCDE90233CDE90544CDE900569B
:102230000648049309940894CDF827402B46046877
:102240002A4629460B20A0471CB070BDD82B002081
:102250000B4A0C4B127810B553F82230DB689847C4
:10226000FFF7CEFFFFF79EFF074B1B699847074B11
:102270001B699847BDE81040054B1B69184700BF14
:102280005D16002030AE010090110020F4100020F7
:10229000BC10002070B5064607F038FE194D012825
:1022A00004462B781CD09EB99C421BD0012B1AD01F
:1022B000154E56F82330DB68984720462C7007F0FF
:1022C0002BFE2B7856F82330BDE870405B6818472A
:1022D000012E12D0032EE7D1022B03D00224E5E712
:1022E000012B00D170BDFFF7B3FF20462C7007F023
:1022F00013FEBDE87040FFF735BF002BF2D000247D
:10230000D4E700BF5D16002030AE0100614A2DE920
:10231000F04F1278604B8BB053F822305F4C9B68C3
:102320009847C0F3074307930990C0F3072A07F0C3
:10233000F9FD064607F0FAFDB379227883469A4202
:1023400004D0B07905F016FDB3792370544B012405
:10235000986805F093F80025ED23DFF8688151486F
:10236000DFF85491504F0593224621464346CDE96C
:102370000309CDE901550094642000F09BF93B6806
:1023800098F800209978914213D0F321CDE90155B6
:102390002546464A023305910392CDF810900094E9
:1023A00022462146642000F085F93B689B7888F836
:1023B00000300DF033F93B688DF82300DB78834261
:1023C0002CD1BBF1000F3ED1002D3CD1079B002B3F
:1023D00043D0737E002B49D1337E002B55D1079B10
:1023E000012B01D10EF096FE7222314B00921A6839
:1023F0003049314B632000F0A5F9FFF729FFFFF7C3
:10240000B1FE77222D4B00921A682A492A4B63208D
:1024100000F098F901200BB0BDE8F08F01224FF4D5
:10242000817100232648CDE90491CDE90133039061
:102430000DF1230364200092114600F03BF93B6844
:10244000D8780DF0D7F8002007F076FD337E002B0A
:10245000CAD0002007F060FDC6E7337E7BB9504646
:10246000FFF718FF01200BB0BDE8F08F337E002B83
:10247000F5D0284607F050FD4FF0010AEFE7079826
:1024800007F04AFD4FF0010AE9E7284607F044FD4E
:10249000A5E700BF5D16002030AE01005C160020ED
:1024A000080A0020FCAD0100340A002008AE01003B
:1024B0004C070020A4AD0100ECAD01005007002046
:1024C00024AE0100840700202DE9F04792B00446B5
:1024D000884607F027FD00233F4FC27DC7E9003340
:1024E0003B81002A56D094F82B0094F82AA094F847
:1024F0002990504594F8281038D8A0F1160EC21F24
:10250000A0F10F065FFA8EFED2B2F6B2894521D84D
:102510004B4612E0A3F10A04022C4ED800EB431400
:1025200038F91450012437F914C0AC45B8BF27F866
:1025300014500133DBB299420CD3022AEAD9022E9D
:102540002BD89C1F022C28D800EB4315022438F905
:102550001550E8E70130C0B20EF1010E013201362C
:1025600082455FFA8EFED2B2F6B2CFD23E22002171
:102570000DF10A0017F0C1FC002340F2015582243E
:1025800000971A4602A91E20ADF808508DF80D409C
:1025900007F084FE12B0BDE8F087BEF1020FC8D884
:1025A000A3F10A04022C11D99C1E022CC1D800EB05
:1025B000431438F914500324B5E79C1E022CB8D8F4
:1025C00000EB431438F914500024ACE700EB43143B
:1025D00038F914500424A6E760160020F0B5204E08
:1025E00083B0054601F1200014461F467160FDF7D7
:1025F00049FE1C4B1C4A9968213037604860946042
:1026000060782278E37802FB00F203F07F0303FB9B
:1026100002F3164C22790B60D3B2012B01D003B028
:10262000F0BD7721FF221E46114F397022712379A8
:10263000FF2B10D120222946684617F02FFC009B63
:10264000032B04EB830206DC019BD2F8052006FA7B
:1026500003F31342EBD105233B7003B0F0BD00BF81
:102660006C210020580A00203C0C00202C22002065
:10267000080B002070B504460E461546049A19460C
:1026800020F8022B20341E2217F0F6FC204631469B
:10269000DF2217F0F1FC45B13046FDF7F3FD294686
:1026A000C0F1DF02204417F0E7FC2046BDE870408F
:1026B000FDF7E8BDF0B5C5B004460E461546014627
:1026C000202204A81F4617F0E9FB049B032B0EDC15
:1026D00001221B48059900EB8303D3F805C002FAD9
:1026E00001F313EA0C0F02D00379934201D045B0F5
:1026F000F0BD4F9B4D99009300224E9B04A8FFF71D
:10270000B9FF4FF0000E9DF80BC04A9B4B9A63F344
:10271000060C8DF80F0020464C9C62F3C71C3B460C
:1027200004A902AA8DF808608DF809508DF80E40B2
:102730008DF80BC08DF80CE0FFF750FFD7E700BF16
:102740002C220020F0B5C5B004460D4616460146C1
:10275000202204A81F4617F0A1FB049B032B0EDCCC
:1027600001221548059900EB8303D3F805C002FA4E
:1027700001F313EA0C0F02D00379934201D045B064
:10278000F0BD4A9B3246009329463B4604A8FFF71A
:1027900071FF00258DF80F0004A902AA20462B46E0
:1027A000ADF808508DF80B508DF80C508DF80E5088
:1027B000FFF714FFE3E700BF2C220020F0B56446CA
:1027C00087B001F069FD002601F0B8FD0125042065
:1027D00040F22F372369A268DB68E168CDE9015632
:1027E0000090064D06480597CDE903057220FFF7D6
:1027F00061FF2369D86807B0F0BD00BFC0AF01001A
:1028000028AF01002DE9F04F91F81CE090F802C0CC
:102810000F460EFB0CF5097D85B00191DDF838807F
:102820004DB34446002605EB450C08EB0C1C226218
:1028300094F8245084F8246094F8255084F8256096
:1028400094F8265084F8266094F8275084F827607E
:1028500094F8285084F8286094F8295084F8296066
:1028600094F82A5084F82A6094F82B5084F82B604E
:102870003034A445DBD1BEF1000F32D03D460026F6
:10288000074603F1FF3921B3CB4600242B6906220A
:1028900013F804A002A84FEA6A01013117F0FEFA0A
:1028A000BA780AF0010306FB0233029A03EB4303F2
:1028B000920002EB0313039943441BF8012F186A9B
:1028C00001EB81018A4002431A622B7D0134A3424D
:1028D000DCDC2B7F0136019AB342914401DD297D76
:1028E000D1E705B0BDE8F08F2DE9F041002482B0BA
:1028F000089D2A622A6595F8242085F8244095F8D9
:10290000252085F8254095F8262085F8264095F85D
:10291000272085F8274095F8542085F8544095F8ED
:10292000552085F8554095F8562085F8564095F87D
:10293000572085F8574095F8282085F8284095F8C5
:10294000292085F8294095F82A2085F82A4095F80D
:102950002B2085F82B4095F8582085F8584095F89D
:10296000592085F8594095F85A2085F85A4095F82D
:102970005B2085F85B400A7D12B30F465E1E3B6903
:10298000062213F8048068464FEA6801013117F007
:1029900085FA08F00108009A4FEA4803984493002A
:1029A00003EB081301992B4416F8012F186A01EB69
:1029B00081018A4002431A623B7D0134A342DEDC7E
:1029C00002B0BDE8F08100BF2DE9F04F97B0684636
:1029D000D1F8013006AF1E7D1D7F796006FB05F33F
:1029E000D1F809205C00FA62DA1DD208A0EBC2001F
:1029F000854604F10803DB08DB0006A8ADEB030DF8
:102A0000F86006A8ADEB030D06AAADEB030DFB6A5B
:102A1000BC60DB68BA623B620A2322467400A046AF
:102A2000FF217B61386117F068FA06AB7B62B30067
:102A30007B637A697B681F2AD3F8053040F31981DC
:102A400010464446954901FB02F102EB421200EBAD
:102A5000421202EBC23201F1404102F14042203108
:102A6000013241F01F0103F5B46019625A629A62A3
:102A700030338342F9D18A480122049089488D215C
:102A8000039004230020A046029001920591009338
:102A90007C6907F13C0311466420FC63FFF70AFEE2
:102AA000BC6800212246B86A17F027FA2246FF21A7
:102AB000786A17F022FA142344463B6301F0ECFBDA
:102AC00001F03CFC0421FB6A4FF0000CDB68009134
:102AD0009621059172492022049173497220039135
:102AE0000121CDE9011C0F21FFF7E4FD45B34FF0B3
:102AF00000093B6AD7F824A0A3F1040BBB6AA3F139
:102B00000208002E00F0AB80D446DE464346A044C7
:102B10005EF8042F33F8020FBCF800108242C8BFE1
:102B200090B28A42B8BF91B2434518802CF8021B7C
:102B3000EED109F101097B6B4D459B44A244E0D1E4
:102B40003B6B013B3B63B9D1A046002D35D09B4682
:102B5000BB6AD7F80C90023BFB617B6AD7F8148004
:102B6000023B3B633B69BD61A3F1020AB6B150462B
:102B70000021D7F830C0FD6935F8023F3CF802EF7C
:102B800030F8022FA3EB0E039A42C8BF09F8018068
:102B900001F10101C8BF03808E42EDD1FB690BF149
:102BA000010B2344FB613B6BA24423443B63BB69A1
:102BB000B1445B45DAD1A046BD69A9217869FB6AB9
:102BC00001307861DB68059135490422049136496A
:102BD00004460391002001210092CDE9011020223A
:102BE0000F216420FFF766FD3E2C7FF422AFAC225C
:102BF0002B4B00922D4900226420FFF7A3FD0020FB
:102C0000CDE901000120AD21254B294A0090049314
:102C1000FB6864200591039229463246FFF74AFD7E
:102C2000AF221F4B0092234900226420FFF78AFD48
:102C30001B4B4FF0B00C049300230224CDE9013369
:102C40001D483B69324603902946CDF814C00094D4
:102C50006420FFF72FFD4437BD46BDE8F08F09F132
:102C600001097B6B4D45A0449B44A2447FF449AFCE
:102C700066E77A6944461146084800FB02F002EB19
:102C8000421201EB421202EBC23203F5B461186248
:102C90005A629A6230338B42F9D1ECE620841002FA
:102CA000C0AF010078AF010028AF010084AF010080
:102CB00098AF0100A4AF0100B4AF01002DE9F04FBF
:102CC000D2F80180D2F805C098F81C9098F814A0AA
:102CD000B9F1000F22D04FF0000E0139BAF1000F08
:102CE00017D00C468678D8F810200EFB06F60AEBB3
:102CF000020712F801BB14F8015F0BF00103334423
:102D000003EB43030CEB031303EB5B039742DD730D
:102D1000EFD10EF1010ECE455144DFD1BDE8F08F69
:102D2000F0B5DCE9002087B064460F46FFF7C6FF28
:102D3000D4E90221002040F239360125CDE9010015
:102D4000054C06483B46CDE90304059600956420F2
:102D5000FFF7B0FC07B0F0BDC0AF0100F0AE01005E
:102D60002DE9F04F8DB082788A4602EB42021201C3
:102D700000AFADEB020D6E46F8610021684617F01A
:102D8000BCF84FF4B4620021C84817F0B6F89AF8BE
:102D90001450BE6135B3DAF810000124054406E092
:102DA0005368854243EA0E0EC2F804E01AD010F8C8
:102DB000013B03F0010C4FEA4C0262441F2B04FA62
:102DC00003FE06EB0212EBDD117A203B8C4604FA7F
:102DD00003F3C1F301010B4363F3010C854282F855
:102DE00008C0E4D19AF81C30BB62002B00F083814C
:102DF000DAF81820002411460120FA62194412F86A
:102E0000013B00FA03F3914244EA0304F7D1FB6962
:102E10003C6293F802C0BCF1000F00F07D810021FC
:102E2000BA69C7F82CA010460D464FF0010B4FF0C1
:102E3000190992463B6AC3F313065FFA86F8C6F394
:102E4000072E360C01EB41030AEB03135C781A7A68
:102E50006FF3C3045C709C7A02F0030224F03F0419
:102E60009C7293F82E401A7224F01F045D7283F84E
:102E70002C5083F82D5083F82E4003F1080280F87F
:102E80000BB080F82F909379013123F00F03334377
:102E90008C4582F8048082F805E000F130009371DF
:102EA000D0D14FF040533A6AD7F82CA09A64BB6A4D
:102EB000002B00F02A81DAF81830FB6200234FF073
:102EC000010B7B629946794BBB624FF0000CFB6AA9
:102ED00029F0030213F80930BC6A0BFA03F8C8F3AF
:102EE0001308C8F30D039B00BB604FEA98337B6067
:102EF000131D3A61FB60C7F81480A6464FEA4C05E3
:102F0000BB69654403EB051505F130087646286872
:102F10006968AA68EB68103545450EF1100E0FC6BA
:102F2000F4D12388796A9AF80B2061F3090323808E
:102F3000002A40F0BD8023687A6962F31F33236062
:102F4000FB699AF80C00DB783A6A0BFA03F3013854
:102F500042EA03019AF81C20032800F2C880DFE847
:102F600000F0825B3602206894F82E5043EA10305D
:102F700025F01F05C0F31403013A45EA13454A45FD
:102F8000A08584F82E500FDDFA6A4A445078EAB2E0
:102F90000BFA00F00343C3F3140322F01F0242EACA
:102FA0001342A38584F82E20B9F1000F08D0FA6AE5
:102FB0004A4412F8012C0BFA02F21343C3F3140330
:102FC00083F4FF1383F4FF5383F01F032AE0E36AC3
:102FD000013A4A45C3F3140311DDFA6A4A445078B2
:102FE00094F82E200BFA00F00343C3F3044022F0C0
:102FF0001F020243A38584F82E20C3F31403B9F102
:10300000000F0FD0FA6A4A4412F8012C0BFA02F2B0
:103010001343C3F3140305E0226843EA1233DB438E
:10302000C3F31403E2681940A07B94F82E30C2F376
:10303000130222EA0102A18520F00F0023F01F03F2
:10304000C1F3044140EA12401943A281A07384F8FD
:103050002E103034BCF1000F15D1DAF818304FF0D3
:10306000010CFB6249E794F82E20C3F314031940C6
:1030700022F01F0242EA1142A18584F82E2030344A
:10308000BCF1000FE9D07A6A9AF81C302032C2F302
:1030900009027A62BA6A09F1010960324B45BA62E3
:1030A00033DDDAF81830FB620FE700BF98000460E8
:1030B000FB6A3A699918FA689D1811F8013B206873
:1030C0000BFA03F3226843EA103363F31F328D4295
:1030D0002260F2D12389BA6803F0030313432381EA
:1030E000A37A7A6823F03F031343A37228E7E36AC5
:1030F000C3F3140396E7FB6993F802C0BCF1000F19
:1031000007D14FF04053C3F848C03437BD46BDE83F
:10311000F08FBB6A3B6282E64FF040533A6A9A6492
:10312000CCE600BF2DE9F041827800AF02EB42020D
:103130001201ADEB020D884605460021684616F0E7
:10314000DCFE30220021614816F0D7FE6FF01F012F
:103150009DF8013098F80C2003F0F40343F00903C4
:10316000013A8DF800108DF801306C46032A03D81F
:10317000DFE802F0948002024FF0FF324FF040513E
:10318000002094F82E3084F82C2043F01F0384F89C
:103190002E3084F82D20C1F830014FF0013219266D
:1031A00004F1300528462346C4F80F20C4F8132044
:1031B000C4F81720C4F81B20E277E27284F82F606D
:1031C000D3F800C05E689968DA681033AB42C0F883
:1031D00000C046608160C26000F11000F0D198F834
:1031E00014303BB3D8F81000012603EB000C06E0C6
:1031F0005368844543EA0808C2F804801AD010F8DE
:10320000013B03F0010E4FEA4E0272441F2B06FAF7
:1032100003F804EB0212EBDD117A203B8E4606FA2E
:1032200003F3C1F301010B4363F3010E844582F8FC
:1032300008E0E4D12646DFF894E0F446306871688F
:10324000B268F3681036AE420EF1100EACE80F0013
:10325000F3D1DFF880C06034654630687168B268C9
:10326000F3681036A6420CF1100C0FC5F4D1BD4620
:10327000BDE8F0814FF0FF324FF04051002094F84C
:103280002E3084F82C2023F01F0343F00F0384F822
:103290002E3084F82D20C1F830017EE701224FF056
:1032A0004051E87894F82E308240C2F3044523F070
:1032B0001F0307482B43C2F3072584F82C2084F80A
:1032C0002D5084F82E30C1F8300166E738060460CE
:1032D000FFFF0F0068060460F0B50D46A9B04C2250
:1032E0000021044602A816F008FE00204FF04052CC
:1032F0002978ADF8040082F8A8106978BDF8042098
:10330000A87861F38A12C2F3072160F3C601ADF811
:1033100004208DF80510BDF8041002AB0DF12A024F
:10332000598502339342FBD14FF04056002286F874
:10333000A7202F7DC7B14FF0010C2969013911F881
:10334000013F28A818441C2B00F8982C02F1010218
:1033500008DD96F8A7001D3B0CFA03F30343DBB22C
:1033600086F8A7309742EAD102A915A84C2216F098
:10337000B9FD15A94C22094816F0B4FD4C2215A937
:10338000074816F0AFFD29462046FFF7E9FC204626
:103390002946FFF7C7FE024829B0F0BD4C00046083
:1033A000000004602DE9F04FD0F80D40D0F8016026
:1033B000D4F800C0D6F820E09CF800309CF801203A
:1033C00096F80090D5185FFA85F808F1010B03F123
:1033D000010A0F46591ED0F8090089B08EF829B0AD
:1033E0008EF822808EF824A08EF82510B9F1000FF7
:1033F0004CD001328EF8272000238EF828301A4650
:10340000636893F8008008F03F0802F114030EEBA4
:1034100043039978013268F30501112A9970F4D1B8
:1034200019211C4B1C4A83F82F1030339342FAD1D8
:1034300033796BB143685BB1164D9CF80D20314672
:1034400000953846FFF7DEF923685A781B78D518BF
:1034500049F6404301356D0093FBF5F540F2E91064
:1034600001220021042608AB43F8045D0B4C0590B3
:103470000B48CDE90121CDE90304114600966420F3
:10348000FFF718F9034809B0BDE8F08F0A3B8EF842
:103490002730B1E79800046038060460C0AF01002F
:1034A00038AF01002DE9F047D0F80D80D0F8015079
:1034B000D8F800302C6A93F801C01B7895F800E02A
:1034C0000CEB0302D2B202F1010A03F101090F462B
:1034D000591ED0F8096082B084F875A084F86E2077
:1034E00084F8709084F87110BEF1000F3BD00CF19D
:1034F000010C84F873C000231A4684F87430D8F89D
:1035000004C09CF8020000F03F0002F1140304EB39
:10351000430393F84E10013260F30501112A83F83A
:103520004E10F2D19CF80010114AC901301D08F06C
:103530000DFBD8F804300F4A197806F10800C901CC
:1035400008F004FB2B7953B1736943B1D8F800201C
:10355000094C527B294638460094FFF7C5F90648C6
:1035600002B0BDE8F0870A3B84F87330C3E700BFC0
:103570000CAF010024AF010038060460F0B500264E
:103580004FF0405301250424D0F80D20D0F801104D
:1035900050681268467090784FF00F0E83F82C0137
:1035A000D0784FF4B47C83F82D01107A83F82A0187
:1035B000907A83F82B01107983F82E01507983F8E3
:1035C0002F010F78C87883F825714F7983F88E70B2
:1035D00083F8840083F8815083F8806083F8AE40DC
:1035E00083F8AF400E7993F8890086EA050767F300
:1035F0000510022783F8890093F8A10066F30410F0
:1036000083F8A10083F88D4083F8B05083F8C5E0BB
:10361000A3F8C8C083F8CC70947B087A83F8004183
:103620008C7983F80541CC7983F80A4183F80D0140
:10363000497A83F81011117B83F8DA10D27A83F873
:10364000A020BDE8F04000F095BB00BF4FF0405314
:1036500010B5D0F80D10D0F809204C68526893F8D6
:1036600041116078054B02EBC01003EB0141802251
:1036700016F038FC63780133637010BD8007016079
:1036800070B5194B84B01B78044613B106F04AFCA0
:10369000C37ED4F80130DB7A23B3D4F80930DE6876
:1036A00006F1800506F50866A5F18000002319469D
:1036B000DA0182584DF823200133042B1144F7D14D
:1036C00000225DF82230D401A1EB430301325B10EC
:1036D000042A0351F5D10430A842E7D105F500755D
:1036E000B542E1D104B070BD971700204FF04053B0
:1036F0002DE9F041012604240025D0F80D20D0F852
:10370000011012684FF00F0890784FF0030E83F805
:10371000E000D07883F8E100107983F8E200507976
:1037200083F8E300107A83F8E600907A83F8E700E4
:103730004F79C87883F88E7083F8840083F88160AD
:1037400083F8805083F8AE4083F8AF400F7993F848
:10375000890087EA060C6CF305104FF01E0C83F805
:10376000890093F8A10067F3041083F8A10083F89F
:103770008D4083F8B06083F8C58083F887E0A3F8B4
:10378000C85083F8CCC0907B83F80001887983F817
:103790000501C87983F80A01497A83F81011117B71
:1037A00083F8DA10D27A83F8A020BDE8F04100F067
:1037B000E1BA00BF4FF040532DE9F041012600254A
:1037C000D0F80D10D0F80100D1E9002194784978A3
:1037D00083F8E040D4784FF0040883F8E14014798E
:1037E0004FF00F0E83F8E2405479B14083F8E34084
:1037F000147A314483F8E640947AC9B283F8E740FA
:103800004779C47883F88E7083F8844083F88160A8
:1038100083F88050077993F8894087EA060C6CF3A7
:1038200005144FF0030C83F8894093F8A14067F327
:10383000041483F8A14083F88D8083F8B06083F886
:10384000C5E083F887C0A3F8C85083F8CC10917BFB
:1038500083F80011817983F80511C17983F80A1181
:10386000417A83F81011117B83F8DA10D27A83F849
:10387000A020BDE8F08100BF2DE9F04F99B0734C56
:1038800006AF07F1240A7861714D0E4694E80F00E7
:103890008AE80F0007F1700307F134087B6407F131
:1038A000100350464146CAF80830CAF80C50FCF7DD
:1038B000E7FC94E80F00674C88E80F0007F110035D
:1038C000404607F14401C8E90234FCF7D9FC012065
:1038D00000F06CFC3861002800F0B3800023E9465A
:1038E0001A46D0F801505C48297D2C7FB961FC61F3
:1038F00001FB04FB6978B96029792B71F96002F149
:10390000140300EB43035988013241F4F861112A92
:103910005980F4D169460BF10703DB08A1EBC3031F
:103920009D46D6F80D20D6F809C0136806AC5B7822
:10393000DCF8081020465A467B60C7F820C016F015
:10394000D1FA7B68BBF1000F09D0224604EB0B00D3
:1039500012F8011B0431824202F8011CF8D148F030
:1039600001024AF00101CDE90021012019465A4621
:10397000234602F05BFF3B6A5A461868214616F060
:10398000B1FA40F241304FF0000B4FF0010C3B6AAE
:10399000BA691B68F969DFF8CC8005902F48CDE93A
:1039A00001BBCDE90308CDF800C06420FEF782FE1C
:1039B000D7F81CA0DA4518DD5846D7F818C0D7F854
:1039C00020E0BCF1000F0DDD00222B7DDEF81C1085
:1039D00000FB0323895C14F803B0013259446245AB
:1039E000E154F2D101305045EBD13246214678699D
:1039F000FFF764F9D7E9062140F24B300025012694
:103A0000CDE90480164823460390CDE90155642092
:103A10000096FEF74FFE2A46BB680F4C03F01F00CE
:103A200002F1140304EB43035988013260F38A1155
:103A3000112A5980F4D13B693A7BD3F801301A71CD
:103A4000CD464C37BD46BDE8F08F00BFD0A0010089
:103A5000BD270000212D000000000460FCAE010025
:103A6000F0AE0100C0AF01002DE9F04FADF50D7DC6
:103A700006AF78608A4600F065FA061E40F3C580FE
:103A8000002403E00134A64200F0BF80214601205B
:103A900000F066FA0028F5D007F1140E0546F4464A
:103AA000D0F8014004F12008664620686168A268E9
:103AB000E368103444450CF1100C0FC6F4D1002615
:103AC00020684FF4F072CCF800008EF80460C5F85E
:103AD00001E0DAF80D3001211B6807F138005B784E
:103AE0001C46FB6016F009FAADF5F16D06AB184601
:103AF00031464FF4F06216F000FA012C40F3898051
:103B00000124A146031FDFF82081BB60DAF80550CD
:103B100005F10F0B05F2AF555846112221460BF166
:103B2000300B16F0EAF9AB45F6D1012240F27A33B8
:103B3000042539496420CDE902610593114607F156
:103B40001003CDF81080CDF8049000953C61FEF78D
:103B5000B1FD00F0A1FB00F0F1FB40F27E332F4AF3
:103B60000593CDE902624FF0C04320220F2100955A
:103B7000CDF81080CDF804907220FEF79BFD4FF039
:103B8000C043B968DFF8A4C007F13802186851F8DB
:103B9000045F04338542BCBF14700860634502F1C2
:103BA0000102F3D14FF463731D4A0593CDE902621C
:103BB00007F13803CDF81080CDE9009620220F21BF
:103BC0006420FEF777FDFB680134A3429ED1524684
:103BD000786807F13801FFF771F84FF46474002238
:103BE0000120104907F13803CDE90122009003912B
:103BF000CDF81080059420220F216420FEF75AFD95
:103C000007F50777BD46BDE8F08F0023D3F80130F4
:103C1000FFDEDFF81480DAE748AF010058AF01009B
:103C2000F0AE010060AF0100C0AF0100800700608E
:103C300008B500F083FB022000F0B8FAD0F8093094
:103C4000986808BD08B500F079FB012000F0AEFAD5
:103C5000D0F80930D86808BD30B4D0F80D20D0F8BD
:103C60000930526815789DB19C685B68803C03F10F
:103C70007C00E41A00EBC515A0F18003221853F86C
:103C8000041F834242F8041FF9D18030A842F3D1C7
:103C900030BC7047704700BF002070474FF0405362
:103CA00093F84121002082F0010283F8412193F82A
:103CB000432182F0010283F8432170472DE9F04748
:103CC000482286B0FF212A4816F017F901A80BF008
:103CD000ADF9804602A80BF0AFF9074603A80BF038
:103CE000B1F918F0FF081DD04FF0000A4FF001099C
:103CF0001F4E04AD019B082213F80A4028466100BC
:103D000004F0030416F0CAF804EBC404049A344423
:103D1000059BA15C09FA03F30AF1010A0B43C245B2
:103D2000A354E7D117F0FF071FD04FF000094FF061
:103D300001080F4E04AD039B082213F809402846E2
:103D4000610004F00304043404EBC404344416F0AA
:103D5000A5F8DDE90423A15C013308FA03F309F1B6
:103D600001090B43B945A354E5D106B0BDE8F0877E
:103D7000C42C002008B50BF037FC054B1B7898428B
:103D800004D01846BDE808400BF010BC08BD00BFC9
:103D90008407002010B50BF027FC04460BF018FC3C
:103DA000844203D0BDE810400BF000BC10BD00BF42
:103DB00030B5013885B00C460A2810D8DFE800F08D
:103DC0003B3E0F3B26110F0F2611060003A80BF0F8
:103DD0002DF92246C1B2039801F07AFDA06305B027
:103DE00030BD03A80BF028F90223C5B203992A4677
:103DF0000093204604F1150300F092FC2246294668
:103E0000039801F079FBA06305B030BD03A80BF067
:103E10000DF90223C5B203992A460093204604F106
:103E2000150300F07DFC22462946039801F022F894
:103E3000A06305B030BDCB7A002BD0D01046214610
:103E4000FFF74AFA206205B030BD00BF01380928EB
:103E500008D8DFE800F0080808070505050505058E
:103E600000238B63704700230B627047037810B503
:103E7000022B04460BD0042B03D10022D0F80130D2
:103E80001A6200236374A374E374237510BDD0F821
:103E900009000849043007F0E5FED4F80900064996
:103EA000083007F0DFFE00236374A374E374237506
:103EB00010BD00BFD8AF0100F8AF0100002230B53F
:103EC00004460D4683B002AB43F8042D18460E4A53
:103ED000152107F03BFE22780C4B294653F822307F
:103EE00020469847C4F80500A06822686568E16824
:103EF000019B98601A605D60D960226901981A611F
:103F0000227D1A7503B030BDD0AF010034B001007E
:103F10000B4B1A680AB90CE01A46D2F81130002B84
:103F2000FAD10023C2F8110043748374C37403757B
:103F300070471860002343748374C374037570471B
:103F40006C160020054B1B6833B10020D3F81130EC
:103F50000130002BFAD17047184670476C160020CC
:103F600070B5164B88B01B687BB1002402E0D3F813
:103F7000113053B11A788242F9D101340029F6D0B8
:103F8000A142F4D1184608B070BD4FF4E17001228F
:103F90000024042608AB43F8041D094D0590094888
:103FA000CDE90124CDE90305114600966420FEF712
:103FB00081FB2346184608B070BD00BF6C16002078
:103FC0001CB0010024B0010070B5094E82B0346805
:103FD0004CB1084D0194D4F81140294601A807F0CE
:103FE00041FE002CF6D10023C6E9003302B070BDBB
:103FF0006C16002014B00100F8B5446805460BF0BB
:1040000011F8ACB123780B2B12D80B4E01460746A2
:1040100056F8333020469847D4F8110040B1037861
:10402000394606EBC3066860736898470120F8BDFF
:1040300000206860F8BD00BF8807002010B5044666
:104040000AF0F0FF636843B11C78054A014652F854
:10405000342018469047012010BD184610BD00BFFF
:104060008807002038B5446805460AF0DBFF4CB1EC
:104070002278054B014653F83230204698470023FA
:104080006B6038BD6C6038BD8807002070B582B0A9
:1040900005460C460AF0C6FF4FF0405393F8412105
:1040A000014682F0010283F8412193F8432182F016
:1040B000010283F84321286818B90CE0D0F81100F8
:1040C00058B10278A242F9D10A4A686002EBC402F0
:1040D00053689847012002B070BD4FF40B76064D2F
:1040E000064C00962B46002221466420FEF72AFB50
:1040F000F7E700BF880700201CB0010064B0010092
:1041000038B5046805460AF08DFF6CB16B685BB981
:104110002178064B2A6803EBC1035B6801466A609D
:1041200020469847012038BD002038BD8807002070
:1041300008B54FF0405393F8243093B172B60A4853
:10414000FFF7DEFF58B10123084A1375BFF34F8F05
:104150004FF040520020064908721370937062B607
:1041600008BD0BF011FBE9E76C16002000001050B1
:10417000D828002008B572B60948FFF7C1FF60B122
:104180000422084B1A75BFF34F8F4FF040530122A2
:104190000020054908721A709A7062B608BD00BF07
:1041A0006C16002000001050D8280020054B1B681A
:1041B00033B11A78824203D0D3F81130002BF8D1F2
:1041C000184670476C160020044B11B143F82010BC
:1041D0007047034A43F82020704700BF540700206F
:1041E000953C00000B4B70B51C680AF01BFF7CB1BE
:1041F0000546094E23782046294656F8233098472D
:10420000D4F81140002CF5D1BDE87040FFF7C2BDD5
:1042100070BD00BF6C1600205407002008B50E4B7F
:104220005A6802B108BD01461846FFF72FFF002863
:10423000F8D00A4B1B680BB10BF0A6FA0123084A11
:104240001375BFF34F8F4FF040520020054908729D
:104250001370937008BD00BF6C160020FC2800206E
:1042600000001050D828002038B50023064D074C18
:10427000074A08492B72236011600BF0F7FCBDE878
:104280003840FFF755BF00BFD82800209C170020FA
:104290009817002031410000002330B40124064962
:1042A000064D0748074A0B7207492B60047030BC63
:1042B0001160FFF73DBF00BFD82800209C170020E9
:1042C000971700209817002031410000002330B4D8
:1042D00001240649064D0748074A0B7207492B601F
:1042E000047030BC1160FFF745BF00BFD828002024
:1042F0009C17002097170020981700207541000098
:1043000008B50BF0C7FC00230249034A0B60136099
:1043100008BD00BF981700209C170020024B58686A
:10432000003018BF012070476C160020024B18683F
:10433000B0FA80F0400970476C16002008B50749B4
:1043400008200BF081F8FFF74DFF0BF0A3FC0023D2
:104350000349044A0B60136008BD00BF9D3C000088
:10436000981700209C17002008B572B60BF092FC3D
:1043700000230849084A0B60136062B6074A516877
:1043800031B1536006490820BDE808400BF05CB825
:1043900008BD00BF981700209C1700206C16002055
:1043A0009D3C000008B5044908200BF04DF8BDE81D
:1043B0000840FFF717BF00BF9D3C000008B5044947
:1043C000082015F081FEBDE80840FFF70BBF00BFD5
:1043D0009D3C000008222F4838B52F4C43682260CE
:1043E0002E4ACBB1002519781570022937D0D3F8A1
:1043F000113093B12748FFF7FFFD002846D0012375
:10440000274A1375BFF34F8F4FF0405200202549C4
:104410000872137093700DE0137001250021224B78
:1044200020481F4A1B680572117503B19847194847
:10443000FFF718FE10221D4B2260D3F8002112074F
:1044400008D5002208241A481A49C3F8804102708E
:10445000C1F840214FF0405300225A7038BDD3F8C4
:104460000D2051680A784978013A9142BFDAFFF786
:10447000E5FD58B101230A4A1375BFF34F8F4FF082
:10448000405208490D7213709370D3E70122054B17
:104490001A72CFE76C160020A40C0020961700209B
:1044A00000001050D8280020F828002000E100E08B
:1044B000A00C002000000250B8B4850005F10A03EA
:1044C00023F00703002800AFADEB030D11DD6B46B1
:1044D000043A15440239181F31F8024F52F8043FCC
:1044E00003FB04F3AA424FEA132440F8043F14608C
:1044F000F2D1BD46B8BC70472DE9F043089D1DB30D
:104500004FF04C0C01264FF00009079CD2B20CFB77
:10451000054CC9B29719C0B20F44A1F10A08A1F124
:10452000030EFFB280448644002B14BF45467546F7
:10453000A0702671E7706171A27184F81990A67657
:10454000E5714C346445EFD1BDE8F083F0B5012A44
:1045500083B0164605460C461F462DDC01466846CC
:1045600015F09CFC36B3009B3F2B1D46A8BF3F2592
:10457000019A002B134405F03F05B8BF00253F2BDF
:104580001A46A8BF3F22002B4FF0000102F03F0364
:10459000B8BF002304F1100207EB420C09B30A195B
:1045A000103207EB4202907965F3050090710131FA
:1045B000B142F3DB03B0F0BD104607F091FA0441BD
:1045C00006FB04F40F2C294606DD0122684615F08F
:1045D00065FC0126009BC7E73246684615F05EFC85
:1045E000C1E79CF8062063F305028CF80620DEE79D
:1045F000F0B5012A83B0154604460E461F462DDC51
:104600000146684615F04AFC009B2DB33F2B1C4623
:10461000A8BF3F24019A002B134404F03F04B8BF05
:1046200000243F2B1A46A8BF3F22002B4FF0000169
:1046300002F03F03B8BF002306F1100207EB420C63
:10464000F1B18A19103207EB4202907964F3050048
:10465000907101318D42F3D103B0F0BD104607F0E7
:104660003FFAF30744BF06416E4321462A46684697
:1046700054BF06F1FF36013615F010FC009BC5E76C
:104680009CF8062063F305028CF80620E1E700BFE2
:1046900070B5DCF80C3086B0644600259847FFF70B
:1046A0004DFED4E901230121042040F253261B6969
:1046B0000295CDE90001064D06480596CDE90305B2
:1046C0007220FDF7F7FFA368186906B070BD00BF40
:1046D000B0B00100BCB0010070B5644686B0DCF833
:1046E00008309847FFF72AFE002201214FF4757623
:1046F0000425636808481B690292084A0596CDE9BB
:104700000320CDE9005114227220FDF7D3FF636826
:10471000186906B070BD00BFB0B00100BCB00100A8
:104720002DE9F04F87B006AF4578D7F82890D01D17
:1047300020F0070009FB05F5ADEB000D0DF1180A9F
:104740000E465046002190461C4615F0D6FBA94562
:1047500041DB4FF0000B08F1FF3922224FF0FF310F
:10476000204615F0CAFB33784FFA8BF0B8F1010FF1
:10477000E0542DDD4FF0000E6FEA060C711C11F8AD
:10478000012BA356B3F1FF3F05D1431CAB42ACBF95
:1047900000235BB2A35498421AD092FBF5F005FBBC
:1047A0001020012814BF01204FF0FF302044825612
:1047B0009A420DD00CEB01029145A1EB060200F0EC
:1047C0009580904501DD1846D9E7BEF1000F4CD128
:1047D000BBF1000F46D09323DFF828B100930022ED
:1047E0005B4645496420FDF7ADFFB8F1000F6CDD75
:1047F000013EB14606EB080119F8013F93FBF5F2C3
:1048000005FB12324945E254F6D1012199200022DC
:104810003A4BCDE904B0CDE9011203930091234650
:1048200042466420FDF746FF0AF1FF3316F8012FD8
:10483000A256B14503F8012FF8D1012100249D258E
:104840002F48CDF810B0039053466420424605959A
:10485000CDE901140091FDF72DFF20460437BD4638
:10486000BDE8F08F4FF0010B77E70121892000228E
:10487000224BDFF890B0CDE9011205900091CDE90F
:10488000033B424623466420013EFDF713FF06EB3F
:1048900008010AF1FF3316F8012FA256B14203F8BE
:1048A000012FF8D1012400218D251548CDE90141C2
:1048B0000390CDF810B0642053464246059500940D
:1048C0002146FDF7F7FE2046C8E701219925002083
:1048D0000A4ACDE901100392CDF810B023460595A0
:1048E000009142466420FDF7E5FEA6E79045BCDD59
:1048F0004FF0010E184642E7DCB0010000B10100A4
:10490000CCB00100B0B001002DE9F843D2F801604D
:10491000074672780D46012A984618D9002814DDFA
:1049200000244FF04C094D1E00E07278510094FBBA
:10493000F1F301FB134315F8010F611009FB038329
:104940000134FFF703FEA742EFD1BDE8F88300284A
:10495000FBDD00244FF04C09331993F91530611039
:10496000002B05DB09FB03837278285DFFF7EEFD62
:104970000134A742F0D1BDE8F88300BF70B56446AA
:1049800086B0DCF800200B4BFFF7BEFFD4E9012313
:1049900001214FF417760020074D084C1B68CDE924
:1049A000010005960091CDE903457220FDF782FED6
:1049B00006B070BD14080460B0B001009CB00100E6
:1049C0002DE9F843D2F801501E466A78012A1ED913
:1049D00000281ADD01F1FF3821244FF04C0908EBC3
:1049E000000700E06A78510094FBF1F301FB1343E8
:1049F00018F8010F04EBD47109FB03634910FFF7AA
:104A0000F7FD474504F1FF34ECD1BDE8F8830028F9
:104A1000FBDD0C464FF04C0905F1140808EB0007CC
:104A200018F9013FC8F13601294401EBD171002B7F
:104A30004FEA610105DB09FB03636A782078FFF721
:104A4000D7FDB84504F10104EAD1BDE8F88300BF01
:104A500030B5644687B0DCF800200B4BFFF7B0FFA1
:104A600040F2DD350121002263680848084C1B68CC
:104A7000CDE90122CDE903040595009114227220AD
:104A8000FDF718FE07B030BD980604609CB0010029
:104A9000B0B00100F0B4147980F8E8405579049C76
:104AA00080F8E950957980F8EA50D57980F8EB5094
:104AB000957A80F8EE50157B80F8EF508D790E785E
:104AC00080F88E5090F8895045F0300580F8895074
:104AD00090F8A1506FF3041580F8A150CD7880F8BC
:104AE000A950002E51D180F8986090F88B5045F075
:104AF000010580F88B500125072700264FF0060C92
:104B000080F88D7080F8B05080F8C56080F88150D2
:104B100080F8805080F8AEC080F8AF700D79002C1E
:104B200080F88450557CB8BF033480F89F50957C42
:104B3000C4F38F04DBB280F89E5080F89C60A0F82C
:104B4000CA4080F8CD30D37C80F80031CB7980F832
:104B500005310B7A80F80A314B7A80F81031137DD9
:104B600080F8DA3090F8A330917D61F3061380F875
:104B7000A33090F8A330D17D61F3020380F8A33015
:104B8000537DF0BC80F8A0307047012580F8985024
:104B900090F88B506FF3000580F88B50ABE700BFA7
:104BA0002DE9F047D0F80160D0F80930747882B070
:104BB0006400D0F80D5033B10F460246196878787A
:104BC000274BFFF7A1FEB76B95F80DC08CB34FF0E4
:104BD0004C0938464FF0000809FB04790CF01F0C13
:104BE0000CF0030E4FEA8E1E4FEA9C0C002101F1DF
:104BF000100300EB430393F806A0DA790AF03F0AAA
:104C000022F0070201314AEA0E0A42EA0C02112997
:104C100083F806A0DA71EAD190F84A3080F848802B
:104C200023F01F0380F8498080F84A304C308145DA
:104C3000DCD133782A78A9786878CDE90074FFF759
:104C40005BFC40F61400234600902A4631464FF0A4
:104C50004050FFF71FFF02B0BDE8F047FFF79AB8DA
:104C60001408046049F640430144114403314900EB
:104C700093FBF1F140F2A51070B501220026042546
:104C800088B008AB43F8041D064C05900648CDE9F2
:104C90000126CDE90304114600956420FDF70AFDC5
:104CA00008B070BDB0B001008CB001002DE9F04F2C
:104CB000D0F80130D0F80D605C785A798BB065007F
:104CC00096F80380002A46D0D0F809209269002A7D
:104CD00041D0197D96F810B0DB68F1B14FF04C0E61
:104CE0009446614A0CEB010A0EFB052E03F1FF39D5
:104CF00019F8013F5B0865B110335B4A5800111881
:104D0000CB799CF800704C3267F3C7037245CB71C6
:104D1000F5D10CF1010CD445EAD1002D00F09E80B4
:104D20004C2251490B4602FB051283F825B04C3347
:104D30009342FAD101AF38462422002115F0DDF864
:104D4000B8F1020F21D0B8F1040F45D0B8F1010F2E
:104D500052D000212AE001AF38462422002115F06C
:104D6000CCF8B8F1020F10D0B8F1040F34D0B8F17C
:104D7000010F41D0002DECD170783278B178FFF777
:104D800071FF39480BB0BDE8F08F002DF4D03B46E1
:104D9000552105EBC500384403F1090203F8011B56
:104DA0009A42FBD19842F7D19DF804104FF0000CC5
:104DB0002D4C3846002301E010F8011FE2180133A2
:104DC000092B1172F8D10CF1010C654504F14C046A
:104DD000D2DD17F8091FECE7002DCDD03B46AA2104
:104DE00005EBC500384403F1090203F8011B9A42A0
:104DF000FBD18342F7D1D7E7002DBDD0B9464FF0A4
:104E0000000EDFF868804946DFF864C0002311E037
:104E1000012C05D1032B03F0010201DC724506D001
:104E200003EBC30208781CF8022002430A70013326
:104E3000082B06D0022CEBD19E45F1D10133082B73
:104E4000F8D10CF1010CE04501F10101DED10EF1C8
:104E5000010E754509F10909D5D1A5E72946242296
:104E600001A815F04AF887E714080460CD2C00204B
:104E7000C42C00202DE9F04F83B04C230C4692F84F
:104E8000018000AF4FEA480603FB06F3ADEB030DCC
:104E90000021914605461A4668467B609A4615F001
:104EA0002CF869465FFA84FC002E53D06B461A2416
:104EB0000DEB0A005A781C7002F0EC0242F002027C
:104EC0005A704C339842F5D1BCF1000F28D0002025
:104ED0004FF04C0B4FF0010E013D05E053690130DE
:104EE0002343604553611ADA15F8013F09EB0302C9
:104EF00092F915201F2B0EFA03F40BFB0212EDDDC5
:104F0000147E203BA2460EFA03F3C4F301041C43B3
:104F1000013064F3010A604582F818A0E4DB86B131
:104F200000234C255524B8F1020F07D105FB0312CD
:104F3000D07C547420F001009474D07401339E42EC
:104F4000F1DC7A68054814F0CDFF04480C37BD4603
:104F5000BDE8F08FBCF1000FF3D0B8E7140804608F
:104F6000F0B5D0F80130D0F809701E7D87B0FD692A
:104F7000BB6806B300224FF4807C14E0786835F8F3
:104F8000124050F822002402012838BF0120B4FB4F
:104F9000F0F0B0F5DC7F28BF4FF4DC7023F812008E
:104FA0000132B24207D028880028E7D123F812C086
:104FB0000132B242F7D140F20726002002254A789A
:104FC000064C0749CDE90100CDE90314059600958B
:104FD00001216420FDF76EFB07B0F0BDB0B0010009
:104FE00070B001002DE9F04F97B0814606AFDFF8B1
:104FF000D8C16E4E07F11C0807F12C0407F10C050F
:10500000F960BA6196E80F0088E80F00C8E9025C11
:105010004046214607F16803FB63FBF731F996E848
:105020000F00634E84E80F00C4E90256204607F1E2
:105030003C01FBF725F9FB6899F80120D3F80160E2
:10504000D3F80D507078D3F809A08001C7E9042A7D
:1050500044F0010406F044FDE98948F00105DAF85E
:1050600000303A69CDE9004501F09CFCDAE9000125
:105070003D69EB46EA1DAB0022F007020A33ADEBB7
:10508000020D23F007037A690DF11808002DADEB2E
:10509000030D7960F368146906AED7F80CA014DD2F
:1050A000002205F1FF3C9C44013B13F8011F18B19D
:1050B00010F801E008F802E01CB154F8211046F89D
:1050C0002210634502F10102EFD1F0B140F221223A
:1050D00005920022CDE901220122364B11460092B1
:1050E000354A6420CDE9033243462A46FDF7E2FA09
:1050F000DAF80130DAF80D10DA789AF80030013277
:10510000092B497B1ED0052B3ED094B100240420EE
:1051100001214FF4107C0294CDE90001264C274870
:105120003346CDE903042A46CDF814C06420FDF7C8
:10513000C1FA4946F868DD46FFF712FF4437BD461D
:10514000BDE8F08F7B6840F64A30CDE903630091FB
:10515000CDE901584FF4F0734FF4487101F0EAFCC7
:105160004FF40C7C0420164A1349002304910121BA
:10517000CDE901137B6800900392CDF814C02A4654
:105180006420FDF797FAC0E77B6840F64A30CDE926
:1051900003630091CDE9015882234FF4487101F077
:1051A000C9FC4FF40F7C0420064ADDE7E0A00100B3
:1051B0007D49000014B10100B0B0010028B1010028
:1051C0001CB1010048BB010091460000F8B59B00EE
:1051D00003F10A0424F0070400AF002AADEB040D2C
:1051E000EC460CDDBC69ACF10405013C224414F82A
:1051F000016F51F82660944245F8046FF7D11A46C2
:10520000614614F06FFEBD46F8BD00BF10B5D0F882
:105210000140D0F809204B781169227DE46882B002
:1052200008460094FFF7D2FF02B010BD70B5D0F869
:105230000150D0F80940EE6882B04B782A7DD4E95D
:1052400003100096FFF7C2FF287D2269A16802B013
:10525000BDE87040FFF730B9D0F809304A781869D6
:105260009200D96814F03EBE2DE9F047D0F80160F5
:10527000D0F80930747882B06400D0F80D5033B1A2
:105280000F46024619683878274BFFF799FBB76B32
:1052900095F80DC08CB34FF04C0938464FF000081C
:1052A00009FB04790CF01F0C0CF0030E4FEA8E1E64
:1052B0004FEA9C0C002101F1100300EB430393F82B
:1052C00006A0DA790AF03F0A22F0070201314AEA21
:1052D0000E0A42EA0C02112983F806A0DA71EAD11B
:1052E00090F84A3080F8488023F01F0380F8498006
:1052F00080F84A304C308145DCD133782A78A9785F
:105300006878CDE90074FFF7F7F84FF4D3602346CF
:1053100000902A4631464FF04050FFF7BBFB02B0E9
:10532000BDE8F047FEF736BD980604602DE9F04F62
:10533000D0F80130D0F80D605C785A798BB06500F8
:1053400096F80380002A44D0D0F8092090690028FC
:105350003FD01A7DD96896F810E0E2B14FF04C0AC0
:10536000DFF8889101EB020C013811F8013B10F8CD
:10537000017FC3F1210393FBF5F205FB12320AFB17
:10538000029223F0010320331344DA79614567F375
:10539000C702DA71E9D1002D00F0A1804C225349F7
:1053A0000B4602FB051283F825E04C339342FAD1F9
:1053B00001AF38462422002114F09FFDB8F1020FFE
:1053C00021D0B8F1040F45D0B8F1010F52D000211F
:1053D0002AE001AF38462422002114F08EFDB8F1F6
:1053E000020F10D0B8F1040F34D0B8F1010F41D042
:1053F000002DECD170783278B178FFF733FC3B4860
:105400000BB0BDE8F08F002DF4D03B46552105EBE5
:10541000C500384403F1090203F8011B9A42FBD18D
:105420009842F7D19DF804104FF0000C2F4C3846ED
:10543000002301E010F8011FE2180133092B11725B
:10544000F8D10CF1010C654504F14C04D2DD17F8DC
:10545000091FECE7002DCDD03B46AA2105EBC50086
:10546000384403F1090203F8011B9342FBD1834244
:10547000F7D1D7E7002DBDD0B9464FF0040CDFF8C7
:10548000748005F1040A49461948ACF1040E002362
:1054900012E0012C05D1032B03F0010201DD96453A
:1054A00007D003EBC30291F800B0825C42EA0B0222
:1054B0000A700133082B06D0022CEAD19C45F0D1AA
:1054C0000133082BF8D10130804501F10101DED113
:1054D0000CF1010CE24509F10909D4D1A2E72946F2
:1054E000242201A814F009FD84E700BF9806046097
:1054F000C42C0020CD2C00202DE9F04F83B04C238C
:10550000567800AF750003FB05F3ADEB030D904635
:10551000834689461A46684600217B609A466C4657
:1055200014F0EBFC002D5BD06B4600200DEB0A0164
:105530005A78187002F0EC0242F012025A704C33A2
:105540009942F5D1B9F1000F2EDD00214FF04C0A40
:105550004FF0010E0BF1FF3C07E05369013143EAC4
:105560000B0B8945C2F814B01DDD1CF8013F08EB98
:105570000302C3F1210092F915201F280EFA00FB47
:105580000AFB0242E9DD107EC3F1010383460EFAF5
:1055900003F3C0F301001843013160F3010B8945A7
:1055A00082F818B0E1DC8DB100234FF04C0C6FF0A5
:1055B0005500022E07D10CFB0342D17C507421F020
:1055C00001019074D17401339D42F2DC7A68214666
:1055D000054814F087FC04480C37BD46BDE8F08F41
:1055E000B9F1000FF2DDB0E79806046070B5D0F8AD
:1055F000092086B0D4699368218851B356689D1EEE
:10560000301F383601E034F8021F50F8042F090229
:10561000012A38BF0122B1FBF2F2B2F5DC7F28BFCC
:105620004FF4DC72864225F8022FECD140F2C235ED
:10563000002202240C480D49CDE90122CDE90310D6
:1056400005950094142201216420FDF733F806B07B
:1056500070BD4FF480709A1E03F11C0122F8020FF6
:105660008A42FBD1E2E700BFB0B0010070B0010098
:105670002DE9F04F95B06F4E06AF07F11405DFF836
:10568000D0C1B9603A6196E80F0085E80F0007F1D4
:10569000600307F124047B6307F10803C5F80CC01D
:1056A00028462146AB60FAF7EBFD96E80F00624E04
:1056B00084E80F0007F10803C4E90236204607F129
:1056C0003401FAF7DDFDBB6844F00104D3F8016052
:1056D000D3F809907078C7F80C90D3F80D8045F096
:1056E0000105800106F0FCF9B8F80E10D9F8003079
:1056F0001422CDE9004501F055F9357DEA46EA1D51
:10570000AB0002F4FC720A33ADEB020D03F4FF634D
:10571000F9680DF11808ADEB030DF268D9E9000343
:1057200006AE7B600C69D7F8089085B10023013A7A
:1057300012F8011F18B110F801C008F803C01CB11D
:1057400054F8211046F8231001339D42F0D100B3E4
:1057500040F28E32059200224FF0010B374BCDE91B
:105760000122374A5946CDE90332CDF800B043460D
:105770002A466420FCF79EFFD9F80130D9F80D10B5
:10578000DA7899F800305A440A2B497B1DD0062B51
:105790003DD094B140F2AE34002001214FF0040C12
:1057A00005940290264C27483346CDE903042A4647
:1057B000CDE900C16420FCF77DFFD546B868FFF74E
:1057C00015FF3C37BD46BDE8F08F7B6840F64A3098
:1057D000CDE903630091CDE901584FF4F0734FF424
:1057E000487101F0A7F940F29E3C0420164A144982
:1057F00004910021CDE901B159467B6800900392E4
:10580000CDF814C02A466420FCF754FFC1E77B683A
:1058100040F64A30CDE903630091CDE90158822377
:105820004FF4487101F086F940F2AA3C0420074A7F
:10583000DDE700BFE0A00100514A000034B10100E3
:10584000B0B0010048B101003CB1010078BB0100DB
:10585000D946000010B5D0F80140D0F809200B78E7
:105860001169227DE46882B008460094FFF7AEFC1F
:1058700002B010BD70B5D0F80150D0F80940EE6804
:1058800082B00B782A7DD4E903100096FFF79EFCC6
:10589000287D2269A16802B0BDE87040FEF70CBE09
:1058A0004FF0405393F84111D0F80930090401F149
:1058B000C041D86801F58431502214F013BB00BFF9
:1058C000D0F809300A7818699200D96814F00ABB38
:1058D0002DE9F0474C2692F8018000AF4FEA4804CA
:1058E00006FB04F6ADEB060D824689466846324655
:1058F00000216D4614F001FB002C5ED06B461A208F
:105900000DEB06015A78187002F0EC0242F0020228
:105910005A704C339942F5D119F0FF012AD00AF19F
:10592000FF304FF04C094FF0010E014405E0536980
:10593000814243EA0C0353611BD010F8013F93FBF3
:10594000F4F204FB12321F2B0EFA03FC09FB025285
:10595000EDDD92F818C0203BE2460EFA03F3CCF3DB
:10596000010C43EA0C0363F3010A814282F818A098
:10597000E3D1F4B12B4655212E44B8F1020F05D1E5
:10598000DA7C597422F001029974DA744C339E4225
:10599000F3D100264FF04C080A4B08FB065118467D
:1059A0004C2214F09FFA03460136B44203F154032B
:1059B000F3D10448BD46BDE8F08719F0FF01AED130
:1059C000F7E700BF4409046008B50520FEF7EEFBC9
:1059D00010B1D0F80930186908BD00BF08B5FEF74E
:1059E000ADFC0520FEF7E2FB10B1D0F809301869D4
:1059F00008BD00BF08B5FEF7A1FC0920FEF7D6FBE5
:105A000010B1D0F80930186908BD00BF4FF04053FD
:105A100093F841314A78D0F8090003491B049200F9
:105A2000C068194414F05EBA6808016008B5062021
:105A3000FEF7BCFB10B1D0F80930186908BD00BFF3
:105A400008B5FEF77BFC0620FEF7B0FB10B1D0F8DE
:105A50000930186908BD00BF8200014814F042BA3D
:105A6000A0170020F0B4D0F809300B4E1C6906F1E5
:105A7000300735460FCDBD4220606160A260E36013
:105A800006F1100604F11004F3D107CE2060616026
:105A9000A260F0BC704700BFA017002008B5FEF759
:105AA0004DFC0A20FEF782FB10B1D0F809301869CE
:105AB00008BD00BF2DE9F043002ADDE907EC21DD38
:105AC0004C2707FB0EC7013901EB020811F8016FE3
:105AD000BEF1000F4FEA8606C6F10A064FEA6606D7
:105AE0000CDD644610367600A519EA7993F800902B
:105AF0004C3469F3C702A742EA71F5D1414503F17D
:105B00000103E3D1BEF1000F09DD4C2303FB0ECEF0
:105B1000C0B28CF825000CF14C0CF445F9D1BDE86D
:105B2000F08300BFF0B40024D0F80D70D0F801C0AD
:105B30007D7BDCF8380005F01F0505F00306B60193
:105B4000AD0804F1100300EB43039979DA7901F011
:105B50003F0122F00702013431432A43112C99718D
:105B6000DA71EED1002290F84A3080F8482023F014
:105B70001F0380F84A3080F84920BC783D786300E4
:105B80007A789CF80010DBB2EE18C670827004714F
:105B90004471857100297FD00A3A1344C3710024EF
:105BA00001254FF04053447685763A7983F8E82012
:105BB0007A7983F8E920BA7983F8EA20FA7983F8C8
:105BC000EB20BA7A83F8EE203A7B83F8EF209CF83A
:105BD000062083F88E2093F8892042F0300283F863
:105BE000892093F8A12064F3041283F8A1209CF883
:105BF000032083F8A920002952D183F8981093F844
:105C00008B2042F0010283F88B204FF04053012299
:105C1000002104244FF4F97083F88D4083F8B020FC
:105C200083F8C51083F8812083F880209CF8044015
:105C300083F884407C7C83F89F40BC7C83F89E4042
:105C400083F89C10A3F8CA0083F8CD20FA7C83F86F
:105C500000219CF8072083F805219CF8082083F890
:105C60000A219CF8092083F810213A7D83F8DA2074
:105C700093F8A320B97D61F3061283F8A32093F86B
:105C8000A320F97D61F3020283F8A3207A7D83F8D3
:105C9000A020F0BCFEF77EB8033A1344C3717EE740
:105CA00083F8985093F88B2064F3000283F88B20DC
:105CB000ABE700BF2DE9F04FB0F1000885B0D2F896
:105CC00001A046DD99464FF0000B4F1E4C239AF879
:105CD0000160CBF1210404EBD4740BF00305012E19
:105CE0004FEA640403FB059517F8011F34DC3246C4
:105CF00002A814F0D3F846B3029B3F2B1946A8BF65
:105D00003F21039A002B134401F03F01B8BF00214B
:105D10003F2B1846A8BF3F20002B00F03F004FF05C
:105D20000002B8BF002004F1100C05EB4C0C4AB384
:105D3000A318103305EB430393F806E061F3050E57
:105D400083F806E00132B242F1DB0BF1010BD845DA
:105D5000BCD105B0BDE8F08F3046019105F0C0FE22
:105D6000044106FB04F40F2C019906DD012202A870
:105D700014F094F80126029BBFE7324602A814F003
:105D80008DF8B9E79CF8063060F305038CF806300F
:105D9000D8E700BFF0B5D0F809308BB01968D0F85B
:105DA0000150DE68D0F80D4021B102462D4B06208F
:105DB000FFF780FF6B7953B14EB101272A7DE96867
:105DC000284D207C3346CDE90075FFF773FE002295
:105DD000E378CDE90722012B8DF8242016D1224843
:105DE00007AD0DF12506002303EBC301415C013330
:105DF000082B42EA0102F7D105F8012BAE4200F16F
:105E0000010001D02A78EEE79DF81C2007A80023A6
:105E1000144D01E010F8012FE9180133092B0A7223
:105E2000F8D149F64041A0786378227803EB40032B
:105E300013440020053301225B00A226042591FBB8
:105E4000F3F4029009490A480491039007AB0596C0
:105E5000CDE90052114664200794FCF72BFC014861
:105E60000BB0F0BDC8070460C42C002068B101006D
:105E700054B10100F0B50546B3B068B3421E022A22
:105E800001D933B0F0BD03AF1C46BC4603F1400E50
:105E9000664620686168A268E368103474450CF1B6
:105EA000100C0FC6F4D15E26389B13AC18685968E5
:105EB0009A68DB680FC4389B186959699A693B4630
:105EC00007C4389A1A49908B2A4620800C6800969D
:105ED00000210120A047D4E70E46144603AF014637
:105EE000BC22384614F009F831683846802213F095
:105EF000F9FF246823AE04F1300C35462068616850
:105F0000A268E3681034644506F110060FC5F4D1A9
:105F100020686168A268BC2407C600220448009477
:105F20003B46046811460120A04733B0F0BD00BFD6
:105F300060E20100F8B50023114C1946236063604C
:105F40003C22104813F0D9FF00F044FA4FF480626D
:105F50000D4B0E490E4E0F4C9B68886030689A605E
:105F60006368851C9847A3680746984739460246E8
:105F7000284613F0B7FF236934689847E080F8BDDE
:105F8000A42B0020282D0020580A00206C2100207E
:105F9000080A002060E201002DE9F04F264C0E4671
:105FA000217885B081420546DDE90E899246DDF80B
:105FB00040B020D0A378AB4202D005B0BDE8F08F4E
:105FC000E378002BF9D09B221C4B00921C49002245
:105FD0006420FCF7B7FB2DBB4FF4F0600121F368A0
:105FE000184C24680E902A460846A446039405B02F
:105FF000BDE8F04F60471F466378002BDAD093224C
:106000000E4B00920E4900226420FCF79BFBCDF85A
:1060100000B04B4608F1100207F110012846FFF7C7
:1060200029FFC7E76B1E022BC7D84FF47070012100
:10603000044C5346D5E700BFA42B0020E0B101007B
:10604000F0B1010060E201002DE9F04F5E4C87B035
:10605000109D64790495DDE91156039614B907B0D3
:10606000BDE8F08F91460290A02288465748002153
:106070009A4613F042FFB8220024554B0092642048
:1060800000225449FCF75EFB05F1FF3BA446524B4E
:106090004E48DFF84CE1CDF814904FE0002A0CBFD9
:1060A000012202224FF487664270029A047032F98C
:1060B0001420049D06FB02F28EFB02761644D217D2
:1060C000C2EBE62240F6241655F82450428038F9F7
:1060D0001420C5F3072706FB02F28EFB0296164436
:1060E000D217C2EBE6228280059A32F81460EAB237
:1060F000BF1AC5F30742C2EB1565AF42C6804FF029
:106100004D024BDD02FB07F7BF1107814581039A62
:106110003AF81450125D85818273029A0CF1010CD9
:1061200032F914201A8038F914205A8001340A2CCC
:10613000197100F1100003F1060335D01BF8011F9F
:106140001A790029AAD1002AF0D04FF48766B3F952
:106150000050B3F9022006FB05F540F6241606FBB5
:1061600002F28EFB05678EFB02964FF00309164480
:10617000D217C2EBE622039E047080F80190365DD0
:106180002F44ED17C5EBE725C18001814181818155
:106190000CF1010C458082808673C7E702FB05F590
:1061A000AA1102814781B2E70C4BCDF840C01B68B1
:1061B00003220293029C02210120A446034B07B054
:1061C000BDE8F04F604700BFA42B0020E817002077
:1061D000E0B101002CB20100282D002060E2010096
:1061E0008100088010B584B003F09CFE174B427903
:1061F0001978914216D04479154AE4B21C7013689C
:1062000003938CB940F21F12124B0092124922469E
:106210006420FCF797FA02210094234622460846A0
:10622000039CA04704B010BD40F21712094B009226
:106230000A4900226420FCF785FA0023022100931A
:1062400008460122039CA04704B010BDDC170020C3
:1062500060E20100E0B10100ACB1010094B10100C5
:1062600010B582B003F05EFE437F93B14FF4987295
:106270000446094B0092094900226420FCF762FAA7
:106280000023074863771A460468009319460220E2
:10629000A04702B010BD00BFE0B101001CB2010078
:1062A00060E20100F0B587B003F03CFE104CC37F04
:1062B00022789A421AD0012200254FF4A277C67F95
:1062C0000C490D4B00920491039311462346059708
:1062D000CDE9015564202670FCF7ECF907492278D6
:1062E0002B460C68009506210220A04707B0F0BDA0
:1062F000DE170020E0B10100CCB1010060E2010036
:1063000030B583B091B1838B028B19491A446E2A40
:106310000B781FDDB0F924001BB30024154A14606C
:10632000013BDBB202200B70106004E00846114A0A
:106330000F4B11601970104C2378834208D0002352
:106340000E49024600930D68207007210220A847DD
:1063500003B030BD0020074A1060002BE0D1106868
:10636000E9E70123034AA0281360F8DD2323D9E7D6
:10637000E4170020E0170020DD17002060E2010094
:10638000002300B583B0019300F024F80378054A98
:106390008DF80430019BC3F30013137003B05DF854
:1063A00004FB00BFDF17002010B582B0FFF758FFD5
:1063B000FFF718FFFFF776FFFFF7E2FF002304491E
:1063C00000930C681A4604210120A04702B010BDBA
:1063D00060E2010000487047881800204FF4806098
:1063E000704700BFF9F74EBF13F07CBD13F085BDB9
:1063F0000F2330B5012583B0054C00930022054BD7
:10640000054964202570FCF79DF903B030BD00BF3D
:106410005A290020D0B20100E0B201003C23F0B5BF
:1064200005460E461446144F8BB0009300223B469F
:10643000124964200994CDE90756FCF783F94FF01F
:106440003F0C0121002004220D4BCDE901100092E8
:106450000393CDE9047C07AB03226420FCF72AF9FF
:10646000003418BF0124074B03EB450203F8156005
:1064700054700BB0F0BD00BFD0B2010074B2010087
:10648000A8B20100A42B0020162310B582B0044648
:1064900000930022134B14496420FCF753F9134B6B
:1064A00040F2F1211A4622F8021B20686168C3F805
:1064B000020051609B7803F03C030C2B09D00022B2
:1064C0000C210B4B09481A7002B0BDE8104003F0D4
:1064D0005DBD03F01BFD0128F1D00122044B1A70B1
:1064E00002B010BDD0B2010054B201006C330020E4
:1064F000881C002000487047FCB201001EF0040F09
:106500000CBFEFF30880EFF309808169004A104760
:1065100041F60000684620F007018D4601B401BC39
:106520008546704772B61EF0040F0CBFEFF308806B
:10653000EFF30980004A1047AD66000072B61EF006
:10654000040F0CBFEFF30880EFF30980004A1047F7
:10655000B166000072B61EF0040F0CBFEFF30880A6
:10656000EFF30980004A1047B566000072B61EF0CE
:10657000040F0CBFEFF30880EFF30980004A1047C7
:10658000B9660000684620F007018D4601B401BCE1
:1065900085467047684620F007018D4601B401BC6E
:1065A00085467047684620F007018D4601B401BC5E
:1065B00085467047684620F007018D4601B401BC4E
:1065C00085467047684620F007018D4619B50723B8
:1065D0002B4CB020237308F0E9FF0021294A2A4BF5
:1065E000A1709A420CD2111D03335B1A23F00303EE
:1065F00026480B4450F8041B42F8041B9A42F9D178
:10660000234A244B9A420CD2111D03335B1A23F008
:10661000030321480B4450F8041B42F8041B9A4220
:10662000F9D11E4A1E4B9A420AD20020111D033393
:106630005B1A23F003030B4442F8040B9342FBD193
:10664000EFF30882174B9A4205D94FF0CD3143F84A
:10665000041B9A42FBD84FF6FF72094B1A8708F0C9
:10666000A5FE08F0AFFE1049002008F051FE0446D8
:1066700000F04EF8844200D0FEE70AF0D1FBFBE7C1
:1066800000001050005600209856002080000000A6
:10669000000000203412002030E3010034120020FA
:1066A000442B0020AC340020FCFB0100704700BFED
:1066B000704700BF704700BF704700BF014B93F8A1
:1066C00021007047C0FB0100014B187E704700BFDE
:1066D000C0FB0100014B587E704700BFC0FB0100AA
:1066E000014B987E704700BFC0FB0100014BD87E74
:1066F000704700BFC0FB0100014B986A704700BFA4
:10670000C0FB0100014BD86A704700BFC0FB01000D
:10671000014B1868704700BFFCFB01002DE9F04FEA
:106720004FEA820B83B00BF10A0525F0070500AF95
:10673000ADEB050D6D463B604B68D1F80080064619
:1067400014468A467B60C0475A462846002113F00B
:10675000D4FB012202FA06FB1BF1FF3B17D37B6837
:1067600098478146BBF1000F00D0C047002CF3DDF5
:10677000AC4600215CF8043B59F8042B013113446A
:106780008C424CF8043CF5D11BF1FF3BE7D2002CC6
:1067900009DD2946002251F8043B0132334194427D
:1067A00041F8043CF7D1DAF80830294620469847EA
:1067B0003A68DAF80C302946204698470C37BD462F
:1067C000BDE8F08F01322DE9F04191FBF2F404FBBA
:1067D000121282B0DDE90A67DDE90C4512B102B0A0
:1067E000BDE8F0812022804600921846DDE90812BB
:1067F000012305F0DBF8B8F1000FF0DD04EB4802EF
:106800000FFA87FE0FFA86FC08E0634655F8041B72
:10681000944203FB101345F8043CE0D034F9023BEA
:10682000B342F2DCBB42B8BF7346EFE72DE9F04F4D
:1068300014469846D31D85B023F0070300AFADEB97
:10684000030D950079608346002168463A6013F095
:1068500054FB05F10A0323F0070341462046EA46AC
:10686000ADEB030DBB6B9847FB6B9847E9460146C0
:106870002A46484613F036FB002C40F388804346F6
:1068800008EB040113F8012B01328B4203F8012CB1
:10689000F8D141463868BB6B9847FB6B9847043D7D
:1068A00004384D44A9F10403514642464FF0FF0C11
:1068B0004FF0010E08E0AB4281F800E01C6001F1EE
:1068C000010102F1010211D050F8044F53F8046F96
:1068D000A642F0DB1478AB4204F1FF3481F800C02B
:1068E000147001F1010102F10102EDD13B685E1E5D
:1068F00056440AF1FF334FF0000A1D46C4461C46B9
:10690000012209E0786888420FDB00228CF8001031
:10691000B4420CF1010C0ED014F9011F0029F7D07C
:106920009CF8000001448B45ECDDB44284F800A0E3
:106930000CF1010CF0D182BBC7E902324146386844
:10694000BB6B9847FB6B9847D7E9023284469E465B
:1069500005E049F82200AC4202F1010215D015F918
:10696000011F0029F7D05CF8220059F82230834239
:10697000EFDB18F80200AC42A0EB010108F80210AE
:1069800085F800A002F10102E9D17346B5E7BB6BBF
:10699000414638689847FB6B98471437BD46BDE8B9
:1069A000F08F00BF2DE9F04F012683B00138B2F11E
:1069B00000080D4600AF9B4606FA00F640F39880AB
:1069C000013B03EB0800F1B203F8011F8342FBD146
:1069D000761000F09D804FEA880AAAF10409C7F8F2
:1069E00004A07C6BD7F830A059464046D047A0475A
:1069F000B8F1000F13DD5B465FFA86FC011F00EB68
:106A0000090E51F8040F1A78A842A2EB0C00D6BF69
:106A1000624418701A70714503F10103F1D17610C8
:106A2000E2D1594640463B6BD7F804A098477B6BB0
:106A300098470AF10A0323F00703ADEB030DB8F101
:106A4000000F02466C465CDD043C161F20463146B2
:106A5000AAF1040A02EB0A0C51F8043F5B1B8C45B7
:106A600040F8043FF8D1D9465B46304602EB0A0EA7
:106A700050F804CF1978AC4501F1FF3CD6BF013185
:106A800083F800C01970704503F10103F0D1594635
:106A900040463B6B7A6098477B6B98477A68924494
:106AA00056F8043F54F8042F5B1B002A83EAE37175
:106AB000A1EBE371B8BF52428A420ADA99F800208A
:106AC000002B02F1FF31D6BF013289F8001089F89E
:106AD0000020B245236009F10109E1D15946404641
:106AE0003B6B98477B6B98470C37BD46BDE8F08FF2
:106AF00076107FF470AF3B6B5946404698477B6BEE
:106B000098473B6B5946404698477B6B9847E5E76B
:106B1000594640463B6B98477B6B98474FEA880A3B
:106B20000AF10A0323F00703ADEB030D02466C469E
:106B30008AE700BF2DE9F04F83B00D9EDDE90F9C81
:106B4000002E40DDDFF88480DF021D0388FB073B59
:106B500088FB05380E9BFF17ED17013B5200C5EB74
:106B60006815002400EB01084FF47A7E41F2301AD8
:106B7000A7EB6B171E44411A01921AE008FB00FBB9
:106B800059F82400019A381890FBF2F00EFB00F03F
:106B900090FBF5F00EFB0BFB0AFB00F00C9A9E42FB
:106BA00002FB10B090FBF1F04CF8240004F101045A
:106BB00009D013F8010F0028E0D19E424CF82400C0
:106BC00004F10104F5D103B0BDE8F08F1F85EB514E
:106BD0002DE9F04F17469A460646850097B02A469B
:106BE000DDE9214908468846002113F086F92A4646
:106BF0000021384613F081F972000021504613F04D
:106C00007CF932460021209813F077F92A4648464D
:106C1000002113F072F9002E40F39980209BCE469C
:106C2000099300230193249B221FC3EBC3730F928C
:106C30005B002A44CDF814A00B9711920E93CDF867
:106C400018800F9B53F8041F0F934FEA116BC1F389
:106C500007435B450C9156D80123249A26989A4005
:106C60000BFB02020292DDE924200BFB02020792D9
:106C7000019A93400A93CBB20093C1F307230D937B
:106C80000D99009B99422FDB079B4FF0010C5E187A
:106C9000DDF82C8005E090065CD4009B01398B4226
:106CA00022DC16F80129019B9A42F4D1029B069C32
:106CB00033F911202368059D01FB023328882360E6
:106CC000D8F8003010440BFB0233C8F8003028809D
:106CD000099803789342E0DAFF2AA8BFFF22009BBD
:106CE00001398B420270DCDD029A0E990C9B0A443A
:106CF00002922499079A0BF1FF3BC3F30743521A00
:106D00005B450792BCDD059BB3F900205AB106999B
:106D10000B685B0293FBF2F30B600B990B685B0251
:106D200093FBF2F20A60019B0F9A01330193059BDA
:106D300002330593069B043306930B9B04330B939A
:106D4000099B01330993119B93427FF47AAF17B0EB
:106D5000BDE8F08F00234FF601701C464A4D16AF78
:106D60002D7847F8040D03952598484D0493149504
:106D700000EB010A02F00F05089245FA03F0C20782
:106D80001AD514AAD056249A584402FB00A013F92D
:106D90000790039A10F809900CFA09F0914540EA1F
:106DA000040009D2A04207D0049A044616A8104451
:106DB000013200F80C9C04920133042BDDD10A9BB4
:106DC000089A1C423FF469AF029B33F911300893D3
:106DD000D30613D49DF804307370069D08982B6871
:106DE000059F01FB00333A882B60D8F8003002443D
:106DF0000BFB0033C8F800303A804EE74FF0000933
:106E0000049B0DF14B005A1E914500EB03070DF159
:106E10004C0A1846CDF840B01CDA09F10109484582
:106E200014DD54469AF800B0039214F8013F9B45D4
:106E30002ABF1D465D465B465EF825200CFA03F32B
:106E40001343A7424EF82530EFD1039A91450AF13A
:106E5000010AE2DB049BDDF840B0032B0BD0042BCE
:106E600005D0022BB9D1089B5B100893B5E7089BAE
:106E70009B100893B1E74AF6AB23089A03FB02F391
:106E80005B140893A9E700BF14B30100000001FFE1
:106E90000288014B1A807047901C00202DE9F041B8
:106EA0004FF4614C4EF2B057184C069E94F8008097
:106EB00094F801E006EB410611F1FF3123D336F9D6
:106EC000024D002CF8D053F8215032F9214068B916
:106ED00005F5807504F58074B8F1000F01D0C5F593
:106EE000F055BEF1000F01D0C4F580440CFB05F550
:106EF00007FB04F42D14241442F8215043F82140D8
:106F000011F1FF31DBD2BDE8F08100BF901C002001
:106F10002DE9F843984604460F46164603F002F85A
:106F2000437A40F6FE72022B14BF0D25002544F271
:106F3000507E49F64E3CC5F57F6108EB04030F31E6
:106F4000A2EB050814F1FF341FD313F8010D00283C
:106F5000F8D037F9140036F914900CFB00F0001447
:106F60009042A8BF10460EFB09F94FEA29494D454A
:106F700020EAE0700BDA4945D8BFC14627F8140073
:106F800026F8149014F1FF34DFD2BDE8F883A94647
:106F9000F4E700BF0288014B1A807047941C002060
:106FA00000231849184A70B41848194E194D1A4C44
:106FB000C1E900330B81C2E9003318491381184A33
:106FC000C6E90033C6E902333361C5E90033154E23
:106FD000C5E902332B61C4E90033C4E902332361FC
:106FE000C0E90033C0E902330361C1E90033C1E9FC
:106FF00002330B61C2E90033C2E90233136133701B
:1070000070BC70470421002054200020D8200020AC
:107010006020002074200020B02000209C20002050
:1070200088200020002100202DE9F04F8BB09DF832
:107030005450854CCDE90450677894F800C0834CD7
:1070400003932478049B15469C4238BF7F4A0E4622
:107050008DF8257038BF1370149F8DF824C0092453
:1070600004F024FF059B0690DFF8F8A1DFF8F89103
:10707000DFF8F8B112352744123603F1120840E068
:10708000734819F804300AAA0A4430F9140012F8B7
:1070900004CC0133DBB201903BF914009C4509F8A4
:1070A00004304FEA44020290C64659D24FF0000322
:1070B000397809F804300AF80410664BBDF804006A
:1070C0009852654BBDF808009852BEF900306048F0
:1070D0008352B6F9003061482BF80230B5F9003020
:1070E0008352039B5E4833F914308352013C631C86
:1070F00007F80119A5F10205A8F10208A6F1020698
:107100004DD0B5F90030002B07DDB6F90030B3F5EE
:10711000007FBCBF00238DF8243005F0CFFC58B1B0
:10712000B5F90030002B07DDB6F90030B3F5007F6C
:10713000BCBF01238DF824301AF804103B788B4231
:107140009ED14FF00003620009F80430404B9B5E73
:1071500001933BF902300293059B03EB020EACE76F
:10716000002BAAD09DF858302BB93B781BB9374B70
:107170001B78012B1AD0BDF80430A8F800303BF979
:1071800002303380354B03989B5E2B80344B9B5EE3
:1071900020F8143019F80430002BA7D1D6E7049B4F
:1071A0000BB92A4A13700BB0BDE8F08F069B132B66
:1071B000E1DC284B28489B5E30F902C013B9BCF1D2
:1071C000000FD8D00198A0EB030E8EEAEE73029860
:1071D000A3EBEE73A0EB0C00772B07902DDD41F6AF
:1071E000CC0C0198A0F1C9039BB26345C3D843F20C
:1071F0004A6C029BA3F291139BB26345BBD841F644
:107200005C2C0EEB4E0303EBD37300EB630E0EF11D
:10721000FF336345AFD8079B029803EB430C0CEB9D
:10722000DC7C00EB6C0343F66A1003F1FF3C844501
:10723000A1D8A8F800E03380A4E703460028B8BF2F
:107240004342772B97DDCAE7941C002000210020E1
:10725000B020002060200020742000209C2000200E
:10726000882000200421002054200020D820002065
:10727000F8B505461A4C0146C022204612F032FEEF
:107280002E1D04F1640C0FCEACE80F000FCEACE85D
:107290000F0096E8070005F1340704F194068CE826
:1072A00007000FCF0FC60FCF0FC697E8070086E87D
:1072B000070005F19407261D0FCF0FC60FCF0FC68D
:1072C00097E807006435343486E807000FCD0FC413
:1072D0000FCD0FC495E8070084E80700F8BD00BF94
:1072E000981C00202DE9F84F90460F461D46044695
:1072F00002F018FE814604F0D9FD99F80920012A10
:1073000040D08246594E05EB440506F1040B14F1BA
:10731000FF3437D335F9023D002BF8D057F824302D
:10732000316E8B4257DA99F80920022A74D1BAF1EA
:10733000010F4FF07F0C30687ADD5B1A0CFB03FC09
:1073400001EBAC1147F8241058F8241081421BDAE5
:1073500099F80930022B72D14FF07F0CBAF1010F6E
:1073600006DC57F82420336E9A42B8BF4FF07F0CEA
:10737000091A0CFB01FC00EBAC1048F8240014F1D6
:10738000FF34C7D2BDE8F88F306BC1F5E0518142C0
:10739000BDDA99F80930022B5CD008B2344904F008
:1073A00071FB58F824108446306BC1F5E051BAF1F6
:1073B000010F06DC57F82420336E9A42B8BF4FF015
:1073C0007F0C091A0CFB01F100EBA110C0F5E05095
:1073D00048F824009BE7D6F89020C3F578539342F1
:1073E00018DA99F80910022932D018B2214904F0AC
:1073F00049FB57F82430D6F89020C3F578539B1AF0
:1074000000FB03F302EBA312C2F57852306847F891
:10741000242099E7306897E718B2174904F032FB47
:10742000BAF1010F8446316E57F82430306884DC9D
:1074300058F82420824210DA4FF07F0C7DE708B222
:10744000594604F01FFB58F824108446306885E73D
:107450007F20D4E74FF07F0CA9E7C2F5E05E326BE6
:107460009645B8BF4FF07F0C67E700BF981C00201F
:10747000CC1C00202C1D0020FC1C00200346997A07
:10748000254A0078012930B410701FD0197C0129D9
:107490000BD009B92148017053F8120F20491B790C
:1074A000C2F812000B7130BC7047D089D98988426C
:1074B00020D0194651F80C0F1A4C8988D060A18051
:1074C0000120022415491C740870E5E71089198908
:1074D000884214D0194651F8025F13484C68098954
:1074E000C2F8025044600181002002240B499C72C2
:1074F0000870CBE7908999898842DAD1E0E7D08893
:10750000D9888842E6D1508859888842E2D190884B
:1075100099888842DED1E7E7581D0020F02B002033
:107520006A1D0020641D00205A1D002010B4314C3B
:10753000314B04FB00F49C4229DB4FF4876202FBD1
:1075400000F02E4AA2FB0032801A02EB5002D20A4F
:1075500040F6241303FB01F1284B294CA3FB010344
:107560002078C91A03EB5103DB0AD0B9A27C002AA8
:1075700036D0B4F813209A4238DCB4F8152010BC89
:10758000C2F5126204329A42B8BF032070471D4A06
:10759000E31782FB04021444C3EBE42404F587627E
:1075A000D6E71949097891B9E18891421BDCA18895
:1075B000914201DD642B19DC218991420DDCA27C12
:1075C000012072B1B4F813209A42D6DD0EE0A189F1
:1075D00091420BDCE1899142F1DD022010BC704741
:1075E000104610BC704761889942E0DA032010BC55
:1075F000704700BFC8FBFFFF1E32DEFF0101100015
:10760000581D002081000880F02B0020F0B49DF868
:107610001840079D022C25D0032C19D0012C02D034
:107620000020F0BC70473B4B5B5D002B41D1092231
:10763000394B3A4EA3F10A0513F8011D022908BF80
:107640009455AB4202F1FF32F6D1F0BC01207047F5
:10765000304B5B5DA3B1324B5B5D023B012B0FD91D
:107660000420DEE72B4E765D86B12D4E765DB71E8B
:10767000012F2DD92B4A042052F82530013314E074
:107680000122264B03205A55F0BC7047264C274E4A
:1076900024F815002648274C20F815300220012335
:1076A00024F815201F4A26F8151042F82530F0BCA2
:1076B00070471B4B5B5D022BC7D11A4B53F825302B
:1076C0002F2BC2DC1C4A1D4B54551C702046A8E7CA
:1076D000032EDBD044F6C466144A134B32F915204E
:1076E00033F91530891A01FB01F1C01A00FB0010B3
:1076F0000C4AB04252F8251001F1010308DD2F2990
:1077000006DC01210D480C4C017061550420CCE7CA
:107710002046CAE7202C0020CA2B00206834002015
:10772000C02B0020982D00205034002074340020FD
:10773000782D0020F42B0020142C0020683300202A
:107740002DE9F04F00248FB0CDE90C23804BCDE91B
:107750000A011C7002F0E6FB437A002B56D17D4BE8
:107760001A78002A4FD0002309931C460A9B189DC3
:10777000A3F102090B9BA3F102080C9BA3F1020BDE
:107780000D9BA3F1020A22E0734A125D022A00F067
:1077900097800023714A13556F4A13552B78704A0E
:1077A0001355BDF814300134A9F80030BDF8183075
:1077B0000A2CA8F80030BDF81C30ABF80030BDF83A
:1077C0002030AAF8003005F8016B00F09180002706
:1077D00039F9023F059338F9023F06933BF9023F1E
:1077E00007933AF9023F0893199B1F555D4BE754E5
:1077F0002E78002E32D15A4B1B5D002BC4D1564A35
:107800001E461355CBE79B7C002BACD10023564A78
:10781000DFF860E1DFF860C1544F524E4E4D504CDE
:107820004E48534902F1140822F8023B42452EF813
:10783000023B2CF8023B27F8023B06F8013B05F817
:10784000013B04F8013B00F8013B41F8043BEBD15C
:107850000023099309980FB0BDE8F08FBDF8181008
:10786000BDF81400FFF762FE0A23199ACDE902045D
:10787000DDE90501CDE90032DDE90723FFF7C6FEAA
:10788000042830D0012804D93E46334B18552B78B4
:1078900085E7314B1B5D022BF7D10128F5D1334B26
:1078A000344933F91430344A08932F4B31F914100A
:1078B00032F9142033F91430069107920593E4E766
:1078C0002B4A52F824202F2A3FF763AF234A125D38
:1078D000002A7FF45EAF1E4609930123199A1355BF
:1078E0001B4A137055E71C4B1B5D022BCDD1D6E70D
:1078F000174B1B78002BADD0DDE90ACEDDE90C89F2
:10790000DDE918AB00230127164A174E194D1A4C12
:10791000164812F8011B11B91BF8031089B136F98A
:1079200013102CF8131035F913102EF8131034F926
:10793000131028F8131030F9131029F813100AF84F
:10794000037001330A2BE4D109980FB0BDE8F08F22
:1079500068330020581D0020C02B00206834002010
:10796000202C0020142C002050340020782D0020E2
:10797000982D002074340020F42B0020014654225E
:10798000014812F0AFBA00BFE80700200021044B05
:1079900003F1780299600C339342FBD1704700BF2A
:1079A000D83300202DE9F04F3F4F85B03C68DDF81B
:1079B0003880012C08BF002200295AD04FEA400A23
:1079C0000AEB0001394D89006E18B4680A2C59DDA4
:1079D000D3F800C00AEB000105EB810149680AEB0E
:1079E00000094FEA8909044655F809001E46D8F8EF
:1079F0000030ACEB0000591A0028B8BF4042002903
:107A0000B8BF4942039203F0E7FF039A834607EBAE
:107A10000217D7E9022379683F69009703F0C6FF90
:107A200005EB090700283BD0326855F8093002FB06
:107A30000BF203FB00230BEB000251100B4493FBF2
:107A4000F2F33360D8F800307F6803FB0BFB07FBD1
:107A500000B0084490FBF2F0C8F8000033685444CA
:107A6000A4002B51D8F800302C44636005B0BDE869
:107A7000F08F0E4B00EB400003EB8000816005B0FF
:107A8000BDE8F08F0134B460012CD3F800C0A1D15F
:107A900045F801C0D8F800107160D3F800C09EE727
:107AA000D8F80000D8E700BFE8070020D83300204E
:107AB00030B40546064C6968AA68EB6800680FC4D4
:107AC00028696969AA69EB690FC430BC704700BFB7
:107AD000701D00202DE9F047DFF8C0800021D8F8A4
:107AE00004208146920012F008FAD8F80430D8F841
:107AF0001020581EA0EB63009047D8F81430984728
:107B0000D8E9006486B3671E002C37D009EB8404E3
:107B1000013ED8F81830984782469FB3D8F8040041
:107B20007D1EA5EB6000D8F810309847FE4202D0C9
:107B3000D8F814309847D8F81C305046984700229F
:107B4000831E3E3033F9021F98420A44FAD154F89A
:107B5000043D2F469A42B8BF1A466B1C2260D8D10A
:107B6000D8F80440002ECED104EBD4706410D8F8BD
:107B70001030C4EB6000BDE8F0471847013EF3D079
:107B8000013EBFE7D8F80420D8F81030501EA0EB13
:107B9000620098474FF0FF35C8E700BF701D002016
:107BA0000E4BF0B45F68022F15DD00EB87070C3F2A
:107BB0000438024600230A4900F10C0652F8045F1B
:107BC00011F9014B964205FB0433F7D11B1140F824
:107BD000043F8742EDD1F0BC704700BF701D00200C
:107BE0007C1D0020DFF868C0F0B4DCF804600024DD
:107BF000002E0ADD01EB8606043E0B1F53F8045FDE
:107C0000AC42B8BF2C469E42F8D1DCF80830461092
:107C1000A34214DA002818DD00236FF00045043970
:107C200051F8044FAC42B8BF1F4603F10103B8BF7F
:107C300025469842F4D1B81B1560F0BC704751F846
:107C400026300020F0BC136070476FF00045F2E76B
:107C5000701D0020F0B40446084E00F13007354690
:107C600020686168A268E3681034BC4206F110061F
:107C70000FC5F4D120683060F0BC7047901D002023
:107C80002DE9F047DFF8E89002EB400599F8303035
:107C900099F8312082B0441E0F468DF804208DF8EB
:107CA00005304E464FF0000A4FF0640800E0013CFA
:107CB000631C17D035F9023D002BF8D0314637F957
:107CC000140003F0DFFEB5F9003098423EDBD9F82E
:107CD0002C2008FB03F302FB00F29342C8BF4FF0D5
:107CE000020AE4E71F4B1878BAF1000F13D11E4ABD
:107CF000C2F800A060B91D4999F832400A68013203
:107D0000A2420A6004DD01221046C1F800A01A70E8
:107D100002B0BDE8F0870546AAF10200B0FA80F093
:107D20004009854217D0104C02A92268014411F87D
:107D3000041C01328A42226011DD00221870226088
:107D400000220A4B1A6002B0BDE8F0870020054B04
:107D50001D788542E7D10022034B1A60F0E72846E0
:107D6000EEE700BF1C210020102100201821002078
:107D7000901D0020014B1870704700BF1C2100208F
:107D8000034B1B781BB9034A136801331360704718
:107D90001C210020182100200278014B1A70704726
:107DA0003C0800200022034B83F8F02083F8E421F4
:107DB000704700BFC02D00202DE9F04F614D97B0F6
:107DC0002C78002C69D000296BD0F42404FB00F43B
:107DD000DFF874811E4608EB040C9CF8F03017465F
:107DE000FF2B68D00133DBB28CF8F030D2F800E022
:107DF000D6F8009004F1D00B012BCDE904E9C3447F
:107E000061D00DF1100900234FF4807A5A460EA874
:107E100008EB040B4946CDE90633039300F096F8CE
:107E20000EAA06A9584600F045F9039B59461A4682
:107E3000CDF800A00123484600F092FA012304F196
:107E400034011A460A904144CDF800A0484600F09B
:107E500087FA04F168010B9041444FF4C873022281
:107E6000CDF800A0484600F07BFA04F19C010C908C
:107E7000414449F640430122CDF800A0484600F0B5
:107E80006FFA06AA0D900AAB594608A800F026FA28
:107E9000DDE908232C783A603360204617B0BDE84E
:107EA000F08FF422284B02FB0033204683F8F010B9
:107EB00017B0BDE8F08F1268336804F1D00BCDE93C
:107EC0000423C3449DE74FF0000A614652465346DF
:107ED0008CF8F1A08CF8F2A00132042AC1F800E07D
:107EE000C1F80C904B600B618B60C1E90533C1E9AF
:107EF0000733C1E90933CB6201F13401ECD1F4213C
:107F00004FF4C863FA2201FB00800DF110090263EF
:107F10004266C0F89820C0F8CC208361C3648365B2
:107F2000C0F88030C0F88C30C0F89430C0F8B4305D
:107F3000C0F8C030C0F8C8304946584600F0A6F82E
:107F400061E700BF3C080020C02D0020F0B413689A
:107F50000F684E685568DC1BAD1B002CB8BF64422F
:107F6000002DB8BF6D422C44C82C84B004DC4EF602
:107F700060251389AB4274D90125C2E90076D1E9A5
:107F80000034341B2E46FF1A002FB8BF7F42002C4E
:107F9000B8BF64423C44134694FBF5F5002123F836
:107FA000086F02F11C0633F8024FA142B8BF214608
:107FB0009E42F8D1937FA942B8BF2946082B02EB15
:107FC00043048CBF0023013305296581937722DDAB
:107FD00027294ADC294B4A1F03FB02F2284BD417FE
:107FE00083FB02531344C4EB631303F2CA34142912
:107FF000009413DD31293DDC6FF0D102143902FB0E
:1080000001F1204ACB1782FB01520A44C3EB221331
:1080100003F28E3304E040F2CA34009440F28E330F
:1080200001934FF42F730146CDE90233164F00F14F
:10803000280601ADC4F57A7287FB02C3A3EBE27395
:108040009BB200F1080220F8023B8242FBD121F8EA
:108050000A4B8E4202D055F8044BEBE704B0F0BC5B
:10806000704701339EB2354695E74FF42F7431299E
:108070000094C1DD4FF42F73D2E700BFF2FEFFFF83
:10808000EBA00EEA898888885655555570B4D1E919
:108090000062034600256424C0E9006200F11C026E
:1080A00023F8085F23F8024F9342FBD170BC0023F2
:1080B000837770472DE9F04F0C469246CFB003907E
:1080C0000146D0221AA8A4F1020B11F00BFF5D4665
:1080D000D6465046A046804F0AF1080600221346B5
:1080E0001AA930F833C00C6B0133042B04FB0C22AB
:1080F00001F13401F5D1B2F5FA6F34BF0122A7FBCB
:10810000023200F1020028BFC2F38F12864225F826
:10811000022FE3D144460023A11D8C46CDE906334E
:10812000CDE908330AF1200A0DF124090DF16808A0
:1081300006AA15464F465C467646D8F8301002929D
:1081400036F8022B34F8020F01FB02F2B2FBF0F218
:10815000A445134445F8043B47F8042F01D02B688D
:10816000EEE70EF1080EF24508F1340809F11009A6
:10817000069BDDD1002108460C461AAD05F1D00C56
:108180002A6B2F68EE683435AC45114407FB024476
:1081900006FB0200F4D194FBF1F490FBF1F1039A99
:1081A00010461460D160934604229046CDE9040342
:1081B00000218C460F460E460C4608460AAB01933A
:1081C00003EB080E1AAA00915EF8103B1168D2F872
:1081D000089001FB0300D168D2F814A001FB03440E
:1081E000516809FB03CC01FB03661169343201FBC2
:1081F0000377009995420AFB03130093E4D11946D3
:1082000006AB53F8083008F1040890FBF3F094FB38
:10821000F3F496FBF3F697FBF3F79CFBF3FC91FB6F
:10822000F3F1B8F1100FCBF83400CBF84040CBF8A5
:108230003860CBF84470CBF83CC0CBF848100BF159
:10824000340BB5D1DDE904430399D0310391002506
:10825000A846AE46AC462F462E46DDF804901AA935
:10826000009359F8100B8B69D1F82CB003FB006612
:10827000CB690BFB005503FB00770B6A03FB00CCBB
:10828000D1E9093A34318A4203FB00EE0AFB008847
:10829000E7D1009B96FBF3F697FBF3F79EFBF3F019
:1082A0009CFBF3FC98FBF3F195FBF3F5019BC4E910
:1082B000066704330193039BC4E908C0C4E90A15A7
:1082C0003434A34204D0029951F8043F0291BEE72E
:1082D0004FB0BDE8F08F00BFD34D62102DE9F043E1
:1082E0008C460C460026DFF87480971E043B06324D
:1082F00037F802EF53F8045FBA4205FB0EF5A8FB0E
:10830000059ECCF8305006EB9E160CF1340CEFD1E4
:1083100001250A46D031136B3432B3FBF6F3002B40
:1083200008BF2B4642F8043C9142F4D100210D468F
:108330000E46236BD4F800C0E7683434A2421944D7
:108340000CFB036607FB0355F3D196FBF1F695FB97
:10835000F1F1C0E90061BDE8F08300BFD34D6210C8
:108360002DE9F04FD2B28BB0012A0192044600F001
:108370005881C0F02881022A00F09D8000234FF42C
:1083800080629C461F461D469E469B461E4698465A
:1083900099469A46CDE907330592039302930693D3
:1083A00004930093039AD4E90004A4EB090406FBA8
:1083B00004290BFB0433A0EB0A0043F3951308FBDD
:1083C00000EE06FB00550BFB007708FB04CC49F3DD
:1083D0009519C1E90493029B4FEAAE2E8B61019B74
:1083E00045F3951547F395174FEAAC2CC1E900E525
:1083F000C1E9027C002B00F0E080009A059B7642E8
:1084000003FB02F3069A002B4FEA822A009AB8BFB8
:1084100003F2FF3306FB02AABAF1000F4FEAA323CF
:10842000B8BF0AF2FF3ACB614FEAAA234B62019B25
:10843000022B00F037810023C1E90A330B6204FBF1
:1084400004F400FB0040A94B984200F3AE80642482
:1084500004FB00F0149BA64A90FBF3F463109342D4
:1084600000F3A38042F21071A24AE41782FB0302D8
:10847000C4EB223201FB12309F4D561C80EAE0749F
:1084800001FB1633A4EBE07435F81600002B00FB5B
:1084900004F035F81220B8BF5B4202FB0300974F8F
:1084A000A7FB0030400B01FB00F0149B90FBF3F0A6
:1084B0000BB0BDE8F08FD1F82090D1E906073D1848
:1084C00009EBD970D1E90ACED1F824A005EB6005FB
:1084D0000EEBDE7809EB0C064FEA68080CEBDC7B50
:1084E0003D4406EB08024FEA6B0B57445544049297
:1084F0005F445D4402EBD27B8A684F4403924A6931
:10850000674409920A687344914605EB6B0507932B
:1085100007EB080300932B4648680AEB4C0A0290CD
:10852000029AF24409EB2219039ACDF818A009EB3C
:10853000621A099AD1E9036006EB201606EB62196C
:10854000002D149AB8BF05F10F0302EB23134FEA75
:10855000851898FBF3F8009A14939601049AC8F5CD
:1085600080634FEA821B149A059396FBF2F69BFBFD
:10857000F2FB029A03FB05F31546099F002B3844D2
:10858000F444039AB8BF03F2FF338001CDF820C052
:1085900003909812099B1544AD01029097019B012D
:1085A0004FEA8A2E4FEA892CFCE642F21070149BA7
:1085B00090FBF3F00BB0BDE8F08FC1E90733C1E9E0
:1085C0000933CB623BE78869149A03441846002BB1
:1085D000B8BF03F10F0002EB20124FEA831898FB9B
:1085E000F2F81492C8F5806202FB03F00023002821
:1085F000D1F800A0D1F80C90B8BF00F2FF3005927E
:108600008212CDE902231F461D469B461E46CDE938
:1086100007330693049300934FEA8A2E4FEA892C7E
:10862000C0E6486AD1E9065605EB460E8644034487
:108630000693734632184D6800920A680F6902EB80
:10864000251ACA68BEF1000F02EB2719149AB8BFA9
:108650000EF10F0302EB23134FEA8E1898FBF3F889
:108660001493C8F5806303FB0EFE0593009BBEF1D7
:10867000000F4FEA8316149BB8BF0EF2FF3E96FB25
:10868000F3F600234FEAAE220292BA01AD01039243
:108690001F469B46CDE9073304934FEA8A2E4FEAE3
:1086A000892C7FE6DDE9042303FB02F3089A002B03
:1086B000B8BF03F2FF334FEA822C9B12049A0B627D
:1086C000079B06FB02C6049A9B020BFB123B002E83
:1086D000B8BF06F2FF36BBF1000FB8BF0BF2FF3B8D
:1086E000B6124FEAAB238E62CB62A8E614AE470106
:1086F0006F110100AD8BDB6820B301005917B7D1B2
:1087000030B40546044C00686968AA68EB680FC479
:108710002869206030BC7047C41D00200268014BEE
:108720001A607047D81D00200146BC22014811F094
:10873000D9BB00BFDC1D00202DE9F0430746032212
:1087400000204FF0010803FB07F6079D104C294459
:108750008E5D94F80090DFF83CE0DFF83CC006F056
:108760000F0646FA02F4E4070CD512F90E4012F98E
:108770000C503C4403FB0414645D4C453CBF08FAB8
:1087800004F4204312F1FF32EBD2BDE8F08300BFC6
:1087900018B3010030B3010038B301002DE9F04FE8
:1087A0008DB0189F0546059097F802B0F878884676
:1087B0008345CDE90832DDF870A04DDC0123B846D1
:1087C0001E9C0BFA03F20AFB024204921D9A97F8D0
:1087D00001900BFB0A2603FA05F28B401343039327
:1087E0004FEA4A030693EBB2CDE90A13079298F8D1
:1087F00000404C450CDD23E0FA0606D4079B83427B
:1088000000F09780002800F0B1800134A14515DB0D
:10881000375DB906F9D51D9B1B9A00932146534637
:108820005846FFF789FF039B8342E5D19DF814303A
:10883000335598F801900134A145E9DA98F803001E
:10884000049B069A0BF1010B1344584556440493BC
:10885000CDDA4746DDF8288019993B680846059A25
:1088600040F8223050F828309400C3F30741B1EBB0
:10887000136F4FEA88003B6019DC94461D9B97F804
:1088800001900AFB01353B7899450BD32B4413F833
:10889000016B464504BF03F801CC97F801905A1BC1
:1088A0009145F4DAFB7801318B425544EBDA1A9B9F
:1088B00008F101011844099B8B420FDD01279C46FA
:1088C0001A9A059D161952F82550026807FA01F305
:1088D000134001311D438C453560F6D100231A9AAF
:1088E000984542F8283040F383800122059F1A986A
:1088F00002FA08F10444BC4602FA07F0CD431646DA
:108900001A9F06E002432A4047F823200133984586
:108910006ED057F823200A42F8D09C45F2DCF2DAF8
:10892000226806FA03FE42EA0E02226057F823206C
:10893000E9E79DF8143008983355049B98F80190A6
:1089400033F91420036804FB02F103EB41230360B5
:108950000BFB02F1169B1B6803EB412316990B607E
:10896000179B1B681344179A13604EE707F00F0319
:10897000CDF860800325984648FA05F3DB072FD52C
:108980001D4B1B9AEF561D4B5F4415F903901D9B21
:10899000A1440093384653464946FFF7CDFE039B5A
:1089A00083421DD11D9B0B9A0AFB0737049B07F8D6
:1089B0000920325533F91420089804FB02F10368AA
:1089C00003EB412303600BFB02F1169B1B6803EBD7
:1089D000412316990B60179B1B681344179A136069
:1089E00015F1FF35C8D2DDF8608098F801900CE7EA
:1089F0000DB0BDE8F08F00BF30B3010038B3010007
:108A00002DE9F04F814291B00546DDE91A760C461A
:108A10000B92984601DB04460D4636F9140057F8D0
:108A2000243058F8241003FB00F336F915E001FB5D
:108A300000F957F825100EEB000A01FB0E3C1D9BB8
:108A4000CDE90DCA53F8241058F825208C4653F868
:108A5000253002FB0E99D8B25FFA81FE864588BFA9
:108A600060F3070CC1F3072EC3F30720864538BF18
:108A700060F30F2CC1F3074EC3F30740209A8645DD
:108A80004FEA136388BF60F3174C0692B3EB116F84
:108A90001F9A88BF63F31F6C229B05921E9A08934E
:108AA000219B04921D9A0FA80EA907930DABCDE947
:108AB0000110039200930B9A0CAB29462046CDF887
:108AC0003090CDF83CC0FFF769FE0CA90EC991FBB0
:108AD000F3F192FBF3F24FEA84094FEA440B48F8B2
:108AE000091047F8092026F80B301C9A1C9B115DD1
:108AF0005B5D00228B4238BF0B461C994FEA450A4A
:108B00000B5526F80A2011B0BDE8F08F2DE9F04F83
:108B1000DFF8C8B08BB09BF80C40002C5BD000286D
:108B200059DD00251F4637F9153005F1010A002BE4
:108B300091468846064654464BDD564503DC4AE0DE
:108B40000134A6423DD037F91430002BF8DD59F836
:108B5000243059F8250058F82510C01A4EF2B053A9
:108B600058F82420891A0029B8BF494203FB01F1B3
:108B70004FF461430028B8BF404203FB00F00914E2
:108B8000001402F029FFDBF814308342D8DD1A9B71
:108B900021460893199BCDF800900793189B324605
:108BA0000693179B28460593169B01340493159B47
:108BB0000393149BCDE901734346FFF721FFA642BF
:108BC000C1D1554637F9153005F1010A002B54463D
:108BD000B3DC5645F5DC0BB0BDE8F08FDC1D0020A2
:108BE0002DE9F04F99B09E4C0AAF657B6C4605B1FC
:108BF00020B9A5463C37BD46BDE8F08F83467C6072
:108C000090464400C21DFB6122F0070204F10803F4
:108C1000ADEB020D23F007030DF1280AADEB030DB8
:108C20005A460AAD0E465046FF21BD6011F065F967
:108C300022462846FF2111F060F97A6E002A40F39F
:108C4000A6803A6FFB69786E911E9A1E01EB400375
:108C5000FB621319FA607B6342464FF0000933460A
:108C60008846C7F824A0C7F818B038F9021F0029B1
:108C700040F38180B869B96F002851F829107ADD76
:108C80004FF0E17C0E0EC1F30744C1F307205FFAF9
:108C900081FE74490CFB06F601FB00F00CFB04F4AA
:108CA00001FB0EF13614241400140914C83EC83414
:108CB000C838C8313E63C7F82080D7F80CA000251B
:108CC000BC62786139611E46904603E07B6B0135DA
:108CD00053454CD03AF9021F0029F7DD4FF46143A8
:108CE00058F8254056F8251003FB04F44EF2B05313
:108CF00003FB01FBBB6E241433F91900FB6E001B50
:108D000033F919104FEA2B4BA1EB0B010028B8BF28
:108D100040420029B8BF494202F05EFE3B6BA342CD
:108D2000D4DDBB6AA342D1DA7B695B45CEDD3B690A
:108D30005B45CBDA7B6F33F91940494B04EB4404B4
:108D40009969C4EBC404A142A8BF21468842BDDA98
:108D50007B6A595DFF297DD0BB6833F815108142CD
:108D6000B4DD7A6A23F8150002F80590AEE73346C1
:108D70004246D7F82080F96A09F1010941457FF49C
:108D800074AF1E469046D7F824A0D7F818B0BBF1B0
:108D9000000F59DD00254EF2B0590BF1FF333B6354
:108DA0006B1C7B631C463B6B9D4203D14CE0013442
:108DB000A34547D058F8243058F8250056F8251018
:108DC000C01A4FF4614356F82420891A0029B8BF0D
:108DD00049420028B8BF404203FB00F009FB01F103
:108DE0000014091402F0F8FD40F647539842DEDC07
:108DF0001AF805201AF804309342D8D1FF2BD6D0A8
:108E0000D7F8903021460893D7F88C305A4607930C
:108E1000D7F8883028460693D7F884300593D7F8DA
:108E200080300493FB6F03933B6E0293FB69CDE9A3
:108E300000833346FFF7E4FDFF230AF804300134D2
:108E4000A345B7D17D6BABE7D7F804D03C37BD461F
:108E5000BDE8F08F03F80590BB6823F8150035E7EF
:108E6000DC1D00200060CB012DE9F04F644C93B075
:108E7000247C34B3002824DD1F4690468A46814670
:108E80004FF0000B37F91B30BBB158F82B2020995D
:108E900002F58072521201FB02F65AF82B3021992A
:108EA00003F5807331445B12C95C56485945057817
:108EB00022D0A94209D388066FD40BF1010BD94502
:108EC000E0D113B0BDE8F08F7746229BCDF800804B
:108ED0000893219B4A460793209B584606931F9B65
:108EE00005931E9B04931D9B03931C9BCDE901736B
:108EF0005346FFF785FDE0E74FF0FF306FF0FE1EB1
:108F0000844603243E49CDE90A578968CDF844E0F8
:108F10000E913D490DF1400E1091229901EB460151
:108F20000D9159000C9111AE1CEB020C18442CD47D
:108F300000282ADB1F99614527DD2099814224DD25
:108F400001FB0CFC21990A9D6144095CA9421CD2D9
:108F50000C9F8B4507EB4C0C17D06427229D35F9ED
:108F60000C500F950D9D35F913C00F9D07FB05F5AE
:108F70000E9F07FB0CFC654507DD64250D9F37F947
:108F8000100005FB00F0604537DC24B1013C14F90A
:108F90000EC0A057C8E70B9F8FE71D9850F82B0015
:108FA000C0F307249C4224D0C0B298420BBF0324D4
:108FB00001244FF0020C4FF0000CBE4601F00F00F0
:108FC00021990B4440FA04F1C9070DD50F49209FA0
:108FD00061560F4E114407FB0131A657895DA94226
:108FE00002D259457FF470AF013C6445EADA774616
:108FF00063E703244FF0020CDFE70B9F65E700BF38
:10900000DC1D002018B301000101FFFF30B3010097
:1090100038B301002DE9F04F83B0DDE90D4704FBC3
:1090200002FE07EB0E04E65C864245D08E4243D03A
:1090300016F0200549D000250324AA464FF0010B65
:10904000DFF8A4C006F00F069CF80090019307EB30
:10905000030C46FA04F7FB0715D5214F214BE757C0
:1090600014F903800D9B174403FB07C717F808800A
:109070000BFA08F7C84547EA050704D2AF421CBF00
:109080003D460AF1010A14F1FF34E2D2012202FA4C
:1090900000F002FA01F10843A842019B19D02840D0
:1090A00010D05B0003EB4E0E0F9B33F90E0090FBCC
:1090B000FAF003B0BDE8F08F5B0003EB4E0E0F9BA0
:1090C00033F90E0003B0BDE8F08F284603B0BDE8C9
:1090D000F08F934003EB4E0E0F9B33F90E00F1E738
:1090E00030B3010038B3010018B301002DE9F04F8F
:1090F000B54CABB0E47B1C94002C00F00E81002832
:1091000000F0038118930023CDE91A121093431E37
:1091100014901F93109B1F9A934280F2FE80369BFF
:10912000109A194651F82230511CCB404FEA820266
:109130001D9115920F9300F05581149B19461D9BAC
:10914000994240F34F810E930023109A1E93189B6F
:1091500003EB420319930BE00E9B0F9A0133520865
:109160000E930F9200F03A81149A9A4200F03681E1
:109170000F9BDB07F0D51A9B15991C4658581B9B73
:109180000E9A1D4654F82240595855F82230051BB6
:109190000C940D93CC1A85EAE573A3EBE573169353
:1091A00084EAE473A3EBE4731793189E199B36F9D2
:1091B0001220B3F90030002C40F0FB80002D40F06D
:1091C00014814FF4007BDDF870800C9E0D9F3446B7
:1091D0003D4604FB03F402FB004405FB03F5134486
:1091E00094FBF3F402FB015595FBF3F5359B159ABF
:1091F0009C469A5822941446CDE9236100260E9B82
:1092000021905CF82330D0B2D9B2814238BF61F3EB
:109210000704C2F30720C3F30721884238BF61F374
:109220000F24C2F30740C3F3074188424FEA136398
:1092300088BF61F31744B3EB126F88BF63F31F64F9
:109240002595230EC4F307459D422697CDE9276651
:10925000299600F3D08001331193E3B21293C4F343
:109260000723139327AF129C139A94425CDC9DF85A
:1092700040306E020B933346464698469DF838A020
:1092800002F101093A9B2A460393399B5146029306
:10929000389B0B980193379B00932346FFF7BAFE48
:1092A00000283DDDDDE90C324FEA442C0221ACEB15
:1092B000030E0EB30BFB0EF3A2EB6323A3EB080329
:1092C000002BB8BF5B42B3F5007F09DAC3F500732A
:1092D00000FB03F357F8212002EB632347F821300A
:1092E000F1B1013921AB53F8213024AA52F82120E1
:1092F000ACEB030E002EDDD1A8EB02020BFB02F259
:10930000A3EB6223A3EB0C03DAE76FF000432F4CCF
:109310002F49304A23600B6010602BB0BDE8F08FFE
:1093200001344C45AED1B046119B01359D429AD1D6
:10933000DDE92842DDE91601279B64259A42A8BF92
:109340001A4605FB04F4154602F07EFB2D2801DDCC
:10935000C0F15A001C4A0CCA03FB00F3C0F12D00F7
:1093600002FB00321C4B83FB0231D3170A44C3EBD0
:10937000621305FB03F3A342BFF6EEAE3A9B149AC9
:109380000893399B0E990793389B10980693379B47
:109390000593369B0493359B0393349B0293189B50
:1093A00001931B9B00931A9BFFF72AFB1C9B1E93A8
:1093B000D2E6DDE91667BE4217DA6D0295FBF4FBD3
:1093C000DDF8708001E700BFDC1D00206008002090
:1093D0006408002038210020B7600BB61E9B002BCC
:1093E0007FF498AE1D9B109394E6640294FBF5FB0A
:1093F0004FF00008E9E6DDE9160102F025FB2D2813
:109400007FF7AAAE00252C46A2E700BF2DE9F04F5A
:10941000B74CADB0A47B002C00F02A82002800F0ED
:109420002782934600260A93023B189303EB4003DE
:109430000B9011930E91B246CDF848B005E00AF1B9
:10944000010ABAF10A0F00F069811F2200211CA84D
:1094500010F053FDA74B4FEA4A0233F91A300C9231
:10946000002BECDDA44B33F91A30B3F5967FE6DA26
:109470000B9B002BE3DD13464FF000089F4ADDF8FD
:1094800060909A1814929E4ACDF840A01344CDF8EB
:109490005C801593CA4605E0119B08F1010853450D
:1094A00000F0B4803AF9023F002BF5DD129E149DC6
:1094B000159F0E9B56F82820B5F90010B7F900004B
:1094C00053F82830891AC01A02F086FA662303FB83
:1094D00000F08C49821237980D9251F8042C10F844
:1094E0000800A1F12004139202F0CCFA04F14C011F
:1094F0000F90BDF9340002F0C5FA0E9B56F82820F3
:10950000B5F9001053F828301690B7F90000891A01
:10951000C01A0029B8BF49420028B8BF4042D4E968
:109520001E9502F091FA04464FF0660B40F2EC4CA7
:109530002D2CC8BFC4F15A0404FB05F5C4F12D0459
:1095400009FB0459369C704D34F9184085FB0965B8
:109550000BFB04FB6D4E109CDFF8BCE1345D109EEC
:1095600028941EF806E00C9C634ECDF814C036F922
:1095700004C0674F674C0497039401270024CDE98A
:10958000017404270D9C0097379F4D4417F808601D
:1095900024944FEAE9790F9C24AB08226820C9EB98
:1095A000651501214FEAAB27CDE92954CDF8ACE090
:1095B000CDE925C72796F9F77DF80C9C4E4B0F9AFD
:1095C0001B5F0D9C02FB04F0139A80111A4405FBEB
:1095D00002F5B0EBA51FBFF65FAF454AD2F8802079
:1095E00082427FF759AF169A9A42BFF655AF4FF0B5
:1095F00001021CAB03F80820179B08F10108013396
:10960000DBB21793119B53457FF44CAF179BDDF8EA
:1096100040A0012B7FF613AF9DF87020002A40F088
:109620009B811CA913460B9C04E011F8010F002834
:1096300040F0808101339C42F7D1199B0E999F0025
:1096400001EB070B12995B0001EB070838990F44F7
:109650000A9901EB03093699CB180D930026CDF832
:109660003CA0CDF83080DDF82CA0DDF8648024AC7F
:109670001BAD002A34D0B04532D03D9B52460893F2
:109680003C9B314607933B9B404606933A9B059390
:10969000399B0493389B0393379B02930A9B019356
:1096A000129B00930E9BFFF7ABF938680C9AB9F93F
:1096B00000301268DBF8001002903D98CDE90054AC
:1096C00006903C9805903B9804903A980390404649
:1096D00001F09CF924991B9802F07EF90D9B1880EB
:1096E0000136B24500F023811CAB9A5DC1E700BF93
:1096F000DC1D0020B02C0020A4330020DC2B002037
:109700007C330020FC1D0020B7600BB68C2D0020A0
:1097100094B301008CB30100CC2B00200B9BDDF82F
:1097200038A0002BDDF848B040F3A2804FF00009CC
:109730000A9B33F91930002B40F394804FF0000856
:109740005D4602E00A9B33F91930002B40F3838019
:109750000A9B33F91830002B7DDDC8457BD055F8C6
:1097600028205AF8283055F829105AF82900891A63
:10977000C01A02F031F95AF8282055F828305AF862
:10978000294055F82970A41AFF1A379B002CB8BF3E
:1097900064420C90002F764913F80900B8BF7F424D
:1097A00002F070F9379B0646714913F8080002F081
:1097B00069F9704B39460D902046D3E92DB402F07B
:1097C00043F940F23B5E4FF0000C012104272D28A5
:1097D000C8BFC0F15A0000FB04F4C0F12D000BFB20
:1097E000004B654B0D9C83FB0B235B444FEAEB7BEB
:1097F000369ACBEB631B5F4B32F91900D3F88430F8
:1098000006FB00F60D935D4B32F9182004930D9B77
:1098100004FB02F403EBA616594BCDF814E00393B6
:10982000379BCDF808C006EBA41613F80940CDE924
:10983000007106FB0BFB0C9F13F80860CDE9247048
:10984000269224AB05224D2027942896F8F732FF64
:10985000B7EBAB1F0FDB0B9B08F1010843457FF40F
:1098600071AFAB460B9B09F101094B457FF460AF2B
:109870002DB0BDE8F08F3D9B0A9C08933C9BCDE941
:10988000005407933B9B0B9A06933A9B41460593E2
:10989000399B48460493389B0393379B0293534666
:1098A000FFF7AEF8C84520DD3D9E389834F91930F1
:1098B00055F829205AF8291050F8290006963C9EA0
:1098C0001BAC05963B9E04963A9ECDE902061AA86B
:1098D000CDE90004484601F099F8DDE91A0102F0EB
:1098E0007BF8369B23F81900B5E73D9E0A9B389814
:1098F00033F9183055F828205AF8281050F8280065
:1099000006963C9E1BAC05963B9E04963A9ECDE97E
:1099100002061AA8CDE90004404601F077F8DDE917
:109920001A0102F059F8369B23F8180093E7DDF886
:109930003CA084E50E989F00590019930A9B00EB08
:10994000070B129803EB0109369B00EB07083898C8
:109950000B4407440D9381E6369B389F0D930023FB
:10996000DDF82890DDF84880DDF838B0199375E609
:10997000641E0020DC1D0020B7600BB694B301000C
:109980009CB3010084B038B5174D04AC84E80F00D7
:10999000202240F21461154804AC00F087F80FCC87
:1099A00028606960AA6003CC182228616961284692
:1099B0004FF4B871EB6000F079F80D494FF4606036
:1099C00000F0C2F80B494FF4905000F0BDF864204D
:1099D00000F0C6FC632000F0C3FCBDE83840602006
:1099E00004B000F0BDBC00BF782B00203C2100205B
:1099F000380A0020480A002084B030B402AC84E861
:109A00000F000A4B9DF808209DF80A109DF812508F
:109A10009DF813401A7099709D72DC7230BC184624
:109A200018224FF4B87104B000F06AB8782B002007
:109A300070B40446174D00686168A268E368164E6A
:109A40000FC520696169154A03C57368A569207F40
:109A500051692B4373600870A37F657FCB71E17FF1
:109A600093680F480570197094F820000D495870DC
:109A700094F821500C489D7094F82250DD70D36802
:109A8000A28DD4E909651A811E605D60086070BC12
:109A9000704700BF102D0020880C0020100C002003
:109AA00084210020D82B002065A00000F8B5134BBE
:109AB0000C0A53F824606EB1F468CFB2013C05E0A3
:109AC00073681B5DFB1A002B05DA2C46631C04F13E
:109AD000FF35F5D1F8BD1546B368326833F8143058
:109AE000014652F824002A46184410F0FBF9B368E6
:109AF00033F814202A4423F81420F8BD680A002003
:109B0000104BF0B40C0A53F824706FB1FB68CEB25E
:109B1000013B05E07C68E45C341B002C06DA2B4634
:109B2000591C03F1FF35F5D1F0BC7047BC683968AA
:109B300034F8134051F82350A41A01462819F0BCF8
:109B400010F0D0B9680A0020044B000A53F8202016
:109B50001AB9142898BF43F820107047680A0020EB
:109B600000232DE9F043036069B3CE68D2B206F159
:109B7000804C06F100470CF1FF3C013F06F1FF3E2F
:109B8000B342A7EB0308AEEB0305ACEB030915D01A
:109B90004C680133645D141BF2D40D6855F82990AC
:109BA000B9F1000F07D08D6835F818502D1B002D26
:109BB000E6DD0560A1444846BDE8F0834FF00009AA
:109BC0004846BDE8F0838946F5E700BF0023B1F5BC
:109BD000704F70B4C1F30724036028DA132C1FD927
:109BE000144D06466A68E86889B2431E02EB4002DB
:109BF00004E032F8020D081A07D52346581C03F179
:109C0000FF34F6D1002070BC7047AA68296852F86A
:109C1000232051F82330121A3260184470BC704768
:109C2000054B8AB253F8241070BCFFF799BF184651
:109C3000E9E700BF580A0020680A002000B583B099
:109C4000014601A8FFF7C2FF044B186008B1019B51
:109C50001844034B186003B05DF804FB7821002022
:109C60007C21002070B50E4E024635681DB10D4BAB
:109C70001C68A54206D314460846002110F03DF9A1
:109C8000204670BD641B8442A8BF04460846224695
:109C90002946254410F026F93560204670BD00BFE6
:109CA000782100207C21002070B50B4E35681DB155
:109CB0000A4B1C68A54202D30024204670BD641BD9
:109CC0008442A8BF044628462246254410F00AF9DB
:109CD0003560204670BD00BF782100207C21002027
:109CE000B0F5C06F16D0B0F5047F03DC0F4B5B6995
:109CF000B3B118470E4B1B7803F07F0303F50473D1
:109D00008342F3DB42189342F0DA10B500F036F8E4
:109D1000012010BD0029E9DB064B1A78A02A01D0EA
:109D200000207047052201201A707047102D002076
:109D3000CC210020080B0020024B1B6903B11847FF
:109D400018467047102D0020084B094A5B78DBB29B
:109D5000012B137006D0022B03D10122054B5A7040
:109D600070477047044B1B68184700BF1C0B00204E
:109D7000C4210020080B0020102D002008B50A4B3C
:109D80001B78012B0CD0022B02D10022074B5A70FA
:109D9000074A137803F080036FF3C713137008BDED
:109DA000044B5B689847F3E7C4210020080B0020B0
:109DB000CC210020102D00202DE9F843254EDFF89E
:109DC000A8903378244DDFF89C80244F012B06D0D7
:109DD000022B1BD06A78934238D1BDE8F883D8F8BB
:109DE000083098470446B9F1000F28D1D8F804305C
:109DF0009847D8F800309847DFF870906B78327841
:109E0000DBB2934209D1002CE0D1E6E71A467C7818
:109E10006B78E4B2DBB29342F5D0012A12D0022A69
:109E200002D100220D4B5A700D4A697813783170B7
:109E300003F080036FF3C7131370BDE8F88309F1D3
:109E4000FF39DBE7074B5B689847EDE71A46012AC5
:109E5000E5D1F7E7C42100201C0B0020080B0020EF
:109E6000CC210020102D0020FF2C0100FE2C010031
:109E700038B5194C2378012B17D0022B0CD0174A78
:109E80005278934206D0164A137803F080036FF39A
:109E9000C7131370002038BD124B104A59785278FE
:109EA000022AF7D000225A70EDE70F4DAB689847B1
:109EB00018B16B6898472B6898470A4B0749227876
:109EC000587849789142E5D0012A02D16B689847C9
:109ED000D9E7022AE6D0D6E7C42100201C0B0020D7
:109EE000CC210020080B0020102D0020A023034AC5
:109EF00013701378A02BFCD0704700BF080B002014
:109F0000014B1878704700BF1C0B0020014BD8781C
:109F1000704700BF1C0B0020014BD870704700BF7A
:109F20001C0B002000487047200B0020014B987844
:109F3000704700BF1C0B0020014B9870704700BF9A
:109F40001C0B002008B5FFF793FF08B9014B186000
:109F500008BD00BFC82100200A46F8B5094F0A4CC9
:109F60003B6826689B79B51803EB830103EB41033B
:109F70009D4200D9FFDE0146B86830440FF0B2FFC1
:109F80002560F8BD5C0B0020C821002070B50D468F
:109F90000646FFF711FF094A094C1378094963F097
:109FA0007F0365F306038D80A5681370A660FFF735
:109FB000CBFEFFF701FFA56070BD00BFCC210020E4
:109FC0005C0B0020680B0020F0B50D46002185B029
:109FD0002E79CDE9011103919DF828C0044638B3CC
:109FE0005EB31F4E3178814224D09DF80510600881
:109FF00060F300019DF80470C4F3800E64F38201E5
:10A000006EF3C30162F303070A466CF307176EF39E
:10A01000041201A80C21ADF809308DF805208DF847
:10A020000470FFF799FF012334702B7105B0F0BD68
:10A030002EB90B4E347005B0F0BD094ED5E79DF832
:10A04000043001A862F303036CF307130C218DF8AD
:10A050000430FFF781FF024E2C71347005B0F0BD63
:10A060001A2200202DE9F04F89B099469DF85C40F6
:10A070009DF8603006460F46904602933CB1FFF7CC
:10A0800061FF002800F0DD8009B0BDE8F08F754B5E
:10A090001D460393FFF790FE2C600024A642CDE9F5
:10A0A0000544079440F3AE80DDF850B04FF0010A4C
:10A0B0006D4D68E037F914E038F9140021B1B5F9B5
:10A0C0000030734500F0C0809DF81610159A4FEAD5
:10A0D0002E2C6CF303018DF817E08DF8180012F8A0
:10A0E00004E00012129A60F307119DF8143004F195
:10A0F000010C8DF8161032F914106CF30303FE29CD
:10A100006AF307138DF81430C8BFFF239DF815C0FC
:10A1100039F81400C8BF8DF81B30139B4CF0010CAC
:10A12000ADF8190053F824006EF3410CD8BF8DF838
:10A130001B108DF815C0C1B2C0F3072CC0F3074344
:10A14000ACEB0101C3EB106399424FF04D024FDDC0
:10A1500002FB01F189118DF81E108DF81F300C21C2
:10A1600005A8FFF7F9FE37F914309BF800102B8093
:10A1700038F914306B800134A64229710BF1010BC0
:10A1800005F106053ED09BF800302979002B91D1CE
:10A190000029F0D0B5F900109DF815C09DF8160003
:10A1A0009DF814E063F3000C0B1263F30300631CCF
:10A1B00063F3030E7346159AB5F902E08DF8171094
:10A1C0008DF818E0115D4FEA2E2E6EF3071061F343
:10A1D000410C6AF307130C218DF8160005A88DF8C1
:10A1E00015C08DF81430FFF7B7FE9BF80010C2E7DA
:10A1F00002FB03F3ACEB00009B118DF81E308DF8D1
:10A200001F00ACE70222194CB9F8143002980092F2
:10A2100017490B22FFF7D8FE2378DBB9039B1B6895
:10A22000002B3FF431AF134913480A78838002F0C2
:10A230007F0263F306020A70FFF786FD09B0BDE8EE
:10A24000F08F084B039328E7B5F9023083427FF47F
:10A250003BAF90E70C210948FFF798FE00232370DD
:10A26000DCE700BFC8210020D0210020881C00208E
:10A2700014220020CC210020680B00206C33002029
:10A28000092300B583B08DF80500022101A88DF8DF
:10A290000430FFF77BFE03B05DF804FBF0B4224C02
:10A2A00082B025788DF80720854202D002B0F0BC3C
:10A2B0007047FF261D4802AD076B15F8012DBF68DA
:10A2C0001B4892000361C0E902151A4B3A81069AB5
:10A2D00026701A608A7822B30B7908784E7902FBCF
:10A2E000003006F07F06144B06FB00F09F683860D4
:10A2F0008B795BB10022013B01EB83056D89013B4A
:10A300002A445D1CF8D102FB06023A60A0230B4AE6
:10A3100013702378FF2BFCD00523137002B0F0BC20
:10A3200070474A78D8E700BF1C220020680A002046
:10A33000880B00206C210020580A0020080B002008
:10A34000014BDB6858817047100C0020034B1879D3
:10A35000A0F10100B0FA80F0400970472C220020E3
:10A3600000B583B00146202268460FF097FD012317
:10A370000099064A019802EB8102D2F80510834049
:10A380000B43C2F8053003B05DF804FB2C2200201B
:10A39000014B1878704700BF840C002070B4184A35
:10A3A000184B90601960827802B94278037901787D
:10A3B000457902FB013105F07F05134B05FB01F1E7
:10A3C0009E68316083795BB10022013B00EB83041E
:10A3D0006489013B22445C1CF8D102FB0512326007
:10A3E000A024FF2309480A4A04700A49137002E0B6
:10A3F0000B78022B02D11378FF2BF9D070BC704779
:10A40000780C00206C210020580A0020080B002046
:10A41000840C00201C0B00200246024B006851688F
:10A4200003C37047981E0020002330B40C490D4A26
:10A430000D48C1E90033C1E90233C2E90033C2E982
:10A440000233C0E90033094D094C0B6113610381EC
:10A45000C5E900332B81C4E90033238130BC704748
:10A46000C4200020EC2000205022002044220020A4
:10A470002C2100202DE9F04F374C85B02579247828
:10A4800083460294092335480395354C354EDFF851
:10A49000D890DFF8D8A00A3200913DE007783BF968
:10A4A0001350002F3FD039F91380F75CA5EB080E4D
:10A4B00071460029B8BF494201914FEA430C002F71
:10A4C00044D00399E75C8E460299092F98BF8E46C7
:10A4D000774601998F422EDD009931F913E03AF960
:10A4E0000C10AEEB010EBEF1000FB8BFCEF1000EA6
:10A4F000774520DD2BF813803AF90C50009921F8AC
:10A500001350E55C092D01D80135E5541578013B60
:10A51000591C00F801591BD012F8015D002DBDD166
:10A52000E5549D55F2E7009929F8135031F913507D
:10A530002AF81350E5E7009929F80C5031F9135027
:10A540004FF001012AF80C50F154DAE7029FC0E7FE
:10A5500005B0BDE8F08F00BF981E00203521002017
:10A560005022002044220020C4200020EC200020A3
:10A5700030B40546044C00686968AA68EB680FC4EB
:10A580002869206030BC7047A01E0020014B18785D
:10A59000704700BF5A220020014B1868704700BF67
:10A5A0005C2200202DE9F04F6FF000444FF0000EC8
:10A5B000A446F2464FF0640987B03D4ECDE9031240
:10A5C0003C4ADDF84880146072680092B2680192DB
:10A5D00032690292F268059210F1FF304AD3347862
:10A5E000002CF9D033F91050009A95424CDD109AA6
:10A5F000019932F910208A4246DD4FF00101A2464E
:10A60000119A115458F82070C7F307215FFA87FB9D
:10A61000C7F30742A1EB0B01C2EB17620132013114
:10A620009142B5BF09FB01F109FB02F291FBF2F285
:10A6300092FBF1F271786245BCBFA64694460029B0
:10A64000CAD002998D42C7DD039951F82040049980
:10A65000A4F50074A4B2B4F5705F51F8201018D9B5
:10A6600005999142B8DD4FF00101119A115410F192
:10A67000FF30B4D2BEF1000F15D150460E4B83F817
:10A6800000A007B0BDE8F08F4FF00001119A1154FF
:10A69000B8E7A1F5007189B2B1F5D05F9CD90599F1
:10A6A0009142E0DC98E7034BC3F800C0E5E700BF48
:10A6B000A01E00205C2200205A2200202DE9F04F2D
:10A6C000C3F307461C0E8BB0A642DDF85090DDE9BF
:10A6D00017E856DC06FB09FC12B2A2EB46220292F6
:10A6E000621CDDB209920AB2079505926544159A7B
:10A6F000C3F307276B1ED3180193169B089703EB30
:10A700004C0C4FEA490301370693079B08998B428B
:10A710002ADC029A019D002AB8BF5242039204E04B
:10A720008A0631D40133BB421ED015F8011F814285
:10A73000F6D13CF91340002CF4DD059AA2EB43213D
:10A7400081EAE172A2EBE172DEF80010013304FB52
:10A750000211CEF80010D8F800200399BB4201FB8B
:10A760000422C8F80020E0D1069B01369C44019BDE
:10A770004B440193029BA3F500730293099B9E42F5
:10A78000C3D10BB0BDE8F08F0022159C01F00F0182
:10A7900004EB030B049341FA02F4E3070BD5094CD5
:10A7A000094B145712F903A0344409FB04B414F8FC
:10A7B0000A40A04204D00132042AECD1049BB1E744
:10A7C000049BB6E734B301003CB30100F0B4044687
:10A7D0000F46134E00F1300C354620686168A268C0
:10A7E000E3681034644506F110060FC5F4D13D4608
:10A7F00020686168A2680B4F07C605F130063C4629
:10A8000028686968AA68EB681035B54207F1100737
:10A810000FC4F4D128686968AA6807C7F0BC7047FC
:10A82000602200209C2200202DE9F04F824693B048
:10A830001F46BDF98C30840007939DF89030884600
:10A840009146002122461C9806930FF056FB2246A3
:10A850001D9800210FF051FBBAF1000F72DD0024AA
:10A86000DFF8A4B102E00134A2456BD037F914300F
:10A87000002BF8DD0025229E1E9B12A853F82430E1
:10A8800059F8242058F8241040F8245D0296219E9F
:10A8900004900196209E08A80390009620460895F3
:10A8A000FFF70CFFDDE9083237F9141093FBF1F3E1
:10A8B00092FBF1F11C9A42F824301D9B43F82410BE
:10A8C000069B012B41D058F824005946C0F30800DC
:10A8D000B0F5807FC8BFC0F5007001F0D3F8064620
:10A8E00059F824004549C0F30800B0F5807FC8BF7F
:10A8F000C0F5007001F0C6F81D9B054653F8241002
:10A900001C9B53F8240001F067F8DBF830308342D9
:10A910004FDC4020064637F914C0DDE9082302FB6E
:10A9200006F603FB00F34FEA8C1C96FBFCF693FB48
:10A93000FCF31C9A42F824601D9A42F8243001343A
:10A94000A24593D113B0BDE8F08F1C9B58F824208A
:10A9500053F8240059F82430C2F30802C3F3080363
:10A96000B2F5807FC8BFC2F50072B3F5807FC8BF63
:10A97000C3F50073CDE90B010D920E930A9401F01B
:10A980002BF8B3250026012104220F901C481D4BF3
:10A99000CDE9040537F91450CDE90116079E009260
:10A9A000039308220AAB6420CDE91065F7F782FE15
:10A9B00059E7DBF82C30079A37F914C09A4202DCC9
:10A9C00040200646A9E7C6F14003DBE90D126046C8
:10A9D0000093002300F0EAFF084B37F914C0D3E9D5
:10A9E0000D12C5F14003009306440023604600F0B9
:10A9F000DDFF37F914C028448FE700BF9C220020F8
:10AA0000B0B30100B8B30100602200202DE9F04787
:10AA1000002688B01C1EDDE91087C8F800603E6083
:10AA20004FDD8A46169D08AB43F8046D0295159DCF
:10AA30000DF1180C0195149DCDE903C30095129BEF
:10AA400091460696FFF73AFE1F4ECAF30800B0F58E
:10AA5000807FC8BFC0F50070314601F013F8DFF801
:10AA60006CA0C0F14003716BDAF838200546009302
:10AA70002046002300F09AFFC9F30809B9F5807F4A
:10AA8000C8BFC9F5007905441049484600F0FAFFEF
:10AA9000DAE90D12C0F14003064600932046002378
:10AAA00000F084FFDDE90623304403FB00F302FBE2
:10AAB00005F0A40193FBF4F390FBF4F4C8F8004014
:10AAC0003B6008B0BDE8F087602200209C22002097
:10AAD000F0B40446094E00F130073546206861683D
:10AAE000A268E3681034BC4206F110060FC5F4D129
:10AAF00020686168A26807C6F0BC7047B41E0020D9
:10AB00002DE9F04F061E83B026DD9946904601914F
:10AB100000244FF0640ADFF84CB0114F02E001341A
:10AB2000A64219D01BF80450002DF8D038F91400B3
:10AB30000B4900F0A7FF019B3D6B33F9142005FB87
:10AB400000F00AFB02F28242B4BF0020012009F8A3
:10AB500004000134A642E5D103B0BDE8F08F00BF88
:10AB6000B41E0020082C00202DE9F047061E1FDD32
:10AB7000DFF840A04FF064085746941E04EB4606E9
:10AB8000A1F102095D1E34F9020F394600F07AFF87
:10AB9000DAF82C2039F9023F02FB00F008FB03F33E
:10ABA0008342B4BF00230123B44205F8013FEAD138
:10ABB000BDE8F087B41E002000283BDD2DE9F043FE
:10ABC000002637468C1E04EB4008951E34F902EF30
:10ABD00035F902CF7745B8BF77466645B8BF6646B8
:10ABE0004445F3D100254FF06408A946124CD4E93E
:10ABF0000DC404FB06F60CFB07F7079C013C04EBB5
:10AC0000000E14F8010F78B131F915C008FB0CFCE7
:10AC1000BC4505DB32F9150008FB00F0B04203DA51
:10AC200084F8009003F80590A64505F10105E8D1E8
:10AC3000BDE8F083704700BFB41E0020034610B487
:10AC4000034C59689A680068DB680FC410BC7047F1
:10AC5000F01E00200023F0B42E492F4D2F4C304A17
:10AC6000304F3148314EC5E90033C5E902332B611D
:10AC7000C1E900332E4DC1E902330B61C4E9003351
:10AC80002C49C4E9023323612B4CC2E90033C2E9E9
:10AC9000023313613B60294A7B603B81C0E900338A
:10ACA000C0E902330361C6E9003325483381C5E9B1
:10ACB0000033244EC5E902330B604B602B618B607F
:10ACC000214DCB600B61236020496360A360E3608A
:10ACD00023611F4C136053609360D3601361336032
:10ACE0001C4A736033812B606B602B81036043606F
:10ACF0008360C36003610B604B608B60C4E9003309
:10AD0000CB600B61136053609360D3601361238148
:10AD1000F0BC70472C230020182300204023002083
:10AD200004230020082C002054230020EC220020C3
:10AD3000D8220020642D0020A4330020903300206E
:10AD4000B02C0020CC2B00208C2D00207C33002048
:10AD5000F8220020DC2B00202DE9F04F460006F100
:10AD600008058BB0044625F00705073020F00700E2
:10AD700000AFADEB050DE846D7E91EABADEB000D1E
:10AD800068467D6FF961E91D21F007017B61D7F805
:10AD90009030ADEB010DBA61002122467B62C7F80D
:10ADA000088078600FF0A9F82A464FF0FF31684616
:10ADB0000FF0A3F83246F96E4046C7F810D00FF0F6
:10ADC00091F8002C7B6A6CDD3A6E002602F1FF39A7
:10ADD00009EB04027A62C7F890305A46D34603E082
:10ADE0007B6A0136994558D019F8011F0029F7D020
:10ADF000FB6E002D33F916A0584B596801EB4A0A37
:10AE0000EEDD4FF0FF333B62D7F88030C7F80C908F
:10AE10000024A3F10208914602E00134A5421BD0B0
:10AE200038F9023F002BF8D0BB6E59F8241033F9E3
:10AE300016C07B6EA1EB0C0133F916005BF82430D1
:10AE4000181A00F0C9FD5045B8BF3C6204F1010476
:10AE5000B8BF8246A542E3D13B6A4A46591CD7F89F
:10AE60000C90BDD03969C9564B1C6CD0BB6833F906
:10AE700011008245B4DA4FF0000C4FF0010E7C68EF
:10AE800023F816A004F801C03B69396A04F806E00B
:10AE90005E547B6A01369945A6D1DA469346D7F8C7
:10AEA0009030002D4BDDD7E9216C00221046396926
:10AEB000013D0D44D7F88CE04C1E7D6214F9011F52
:10AEC0004D1C38D05AF822505BF82280A946FD6903
:10AED00025F81190BD6925F81180D7F880501CF82D
:10AEE000028035F912907D6925F8119036F912909B
:10AEF0003D6D25F811907D6D05F801801EF80280EA
:10AF0000BD6D05F801803D6F6A54FD6DA84653F88C
:10AF1000225048F82150D7F880104AF822004BF808
:10AF2000220021F8120026F812000CF802000EF898
:10AF3000020043F82200796A0132A142BED12C37C7
:10AF4000BD46BDE8F08F0121BB68386A23F816A022
:10AF50003B691E547B68995542E700BFF01E0020F4
:10AF60002DE9F04F044699B006AFD7F8805007306E
:10AF7000073525F00705ADEB050D20F0070006AD00
:10AF8000ADEB000D0DF1180BC7E90C215846224618
:10AF90000021BD6098467B600EF0AFFF0022D7F81D
:10AFA0008010FA63914252DDC44EC7F82CB006E01F
:10AFB000FA6BD7F8803001329A42FA6345DAD7F853
:10AFC0008C3033F91230002BF2DD0023D7F8B82093
:10AFD0009C42C7E91023FA6B40F36C814FF0FF39B4
:10AFE00004E07B6C0133A3427B6420DA38F9131050
:10AFF0000029F6DD786B396B31F9131030F9133015
:10B00000D7F8880050F82250D7F88400691A50F811
:10B010002200C01A00F0E0FC3B6C0546834200F3BE
:10B0200005817B6CFA6B0133A3427B64DEDB4FFA54
:10B0300089F30121B8688354FB6A013203F80910CF
:10B04000D7F88030FA639A42B9DBD7F82CB0002CDD
:10B0500040F3E8804FF00009013C0BEB0402D7F805
:10B060008030FA60BA68013B0BF1FF3BD318CA4647
:10B07000FB62D84605E0FB6809F10109984500F03C
:10B08000D18018F8013F002BF5D07B6833F919E027
:10B090007B6B33F919203B6B0EFB02F233F919304D
:10B0A000FA610EFB03F33B623B6F33F919307B62AD
:10B0B000BB6F13F80930BB627B6F13F809B0FB6FED
:10B0C00053F82900D7F88030002B40F38680C7F86A
:10B0D00000800023D846F346BA68013A12F9011FEE
:10B0E000894572D1D7F88C00FD6930F913C0D7F8C3
:10B0F0008400E34450F82360D7F8880006FB0C5620
:10B1000050F823003D6AB861FE61BE69F96F06FB25
:10B110000C553D62D7F8945051F82940EE5CE0B2EE
:10B12000BE617E6A3861B446D7F89000D7F898506F
:10B1300030F91300ED5C78617E692046B444BE6945
:10B1400051F8231048EA0608BE6A5FFA81FEAE4253
:10B15000B8BF2E463D69BE627545C4F30726C1F3EC
:10B16000072588BF6EF30700AE4238BF65F30F2096
:10B17000C4F30746C1F30745AE424FEA116188BFE9
:10B1800065F31740B1EB146F88BF61F31F60D7F808
:10B190008410C7F824C041F823A0D7F8881041F8DC
:10B1A00023A0D7F88C1021F813A0D7F8901021F81D
:10B1B00013A0D7F8941001F803A0D7F8981001F85D
:10B1C00003A0D7F89C1041F823A0F96A01339142FB
:10B1D00084D1DE46C346D7F80080FB693A6A93FB08
:10B1E000FEF392FBFEF2796821F819E0796B21F801
:10B1F00019303B6B23F819203B6FBA8C23F81920C8
:10B200007B6F03F809B0BB6F1A4697F8283002F835
:10B210000930FB6F43F82900FB6809F101099845E3
:10B220007FF42FAF4C37BD46BDE8F08F40F2273298
:10B2300000920022334622496D2093464FF0040AC3
:10B240003D64D7F844900125F7F77CFA4FF44A7330
:10B250001C4A0593039229462A4607F13C030496AB
:10B26000CDE9015BCDF800A06420F7F723FA40F2A6
:10B270002933154A2946039205932A4607F14403C8
:10B28000CDE9015BCDF800A004966420F7F712FA2F
:10B2900040F22A300D4B05900393CDE9015BCDF8C8
:10B2A00000A004962A46294607F140036420F7F7D8
:10B2B00001FAB6E64FF0FF339946BAE6C4B301008F
:10B2C000D0B30100DCB30100E0B30100E4B301003E
:10B2D0002DE9F04F071E83B040F3A98092469B46AC
:10B2E00089460025B8463BF91530002B40F39B807A
:10B2F0004FF0FF360024169FA54213D03BF91430BF
:10B30000002B0FDD5AF825105AF8242059F8250093
:10B3100059F82430891AC01A00F05EFBB842BCBF4D
:10B32000074626460134A045E6D1731C7BD03BF985
:10B33000160059F826203BF9151002FB00F359F8C6
:10B3400025200C1802FB013292FBF4F249F825206B
:10B350005AF826305AF8252003FB00F302FB01328D
:10B3600092FBF4F20C9B4AF825200C9A2BF815401E
:10B3700032F8161033F815300D9A0B440C99925D83
:10B3800021F815300D9B71005A550E9B0E9A9B5D4E
:10B39000525D0191934238BF13460E9AB100535546
:10B3A0000F9B53F8252053F826301046DFB23C4659
:10B3B0000D9F5FFA82FE07EB060C0E9FA6453E44EA
:10B3C000C2F3072EC3F3072788BF64F30700BE4507
:10B3D00038BF67F30F20C2F3074EC3F30747BE45DC
:10B3E0004FEA136388BF67F31740B3EB126F88BF50
:10B3F00063F31F600F9B4FF0000243F8250000230A
:10B4000049F801304AF80130019B01982BF80320DC
:10B410000C9B1A524FF000038CF8003033700F9BD6
:10B420001A46002353500135A8457FF45CAF03B0A2
:10B43000BDE8F08F2DE9F04FB0F1000B83B0DDE9EE
:10B4400011C9DDE918A843DD00264FF0FF34DFF80D
:10B4500088E002E00136B3453AD01EF80600002825
:10B46000F8D1013408EB040002E00134A4452FDDDB
:10B47000077805460130002FF7D06445019527DA9B
:10B48000139859F8247050F8240021F8167022F807
:10B49000160014980C9D30F914701698005D23F86E
:10B4A0001670159F37F9147025F816700D9D0F9FB3
:10B4B000A85517980E9D005DA8555AF8245001987C
:10B4C000007847F82650109DA8550136B345C4D1E1
:10B4D00003B0BDE8F08F00BF082C00202DE9F04F2D
:10B4E0001D464FF01F339BB004460E46904614AFE6
:10B4F0007960DFF894C16049C7E90333D7E9129A4C
:10B50000CDE9061CB96EBB820391796E07F10C037D
:10B51000089302913B6C396E584A59480D9301913A
:10B520007B6CF96DCDE90E390592BB6D7A6DCDE975
:10B530000946CDE90B85CDF840A00091396D049006
:10B540000A20FFF709FC4F4AD7F88400D2E90232FB
:10B5500000210092642200F029FA00284FD03B6FAE
:10B56000002B4CD0FB6F002B49D083463B6FCDE9BD
:10B570000568CDE90BA37B6C07F10C0609933B6CC6
:10B580001196CDE90753BB6ED7F8806003937B6EAD
:10B590001096FE6F02933B6E0F96BE6F0193FB6D8C
:10B5A0000E967E6F0093396DD7E915230A20CDF8EA
:10B5B00028900494CDF848B00D96FFF7D1FCD7F849
:10B5C0008430E3B107F10C030993D7F88030CDF84C
:10B5D00028B00893FB6FCDF808900793BB6F4246E5
:10B5E00006937B6F796805933B6F2046CDE903A3F3
:10B5F0007B6C01933B6C00932B46FFF769FEE31DC8
:10B6000023F00703ADEB030D002C0DF1500C10DD02
:10B61000AA1E7E6802EB44000DF14F0132F9023F91
:10B62000002BD4BF00230123824201F8013FF5D152
:10B630007E607B6C396D0A933B6C0A20CDE9085320
:10B640007B68CDE90CACCDE90543FB6ECDF82C90C1
:10B650000493BB6ECDF81C8003937B6E02933B6E0C
:10B660000193FB6D0093D7E91523FFF7E3FE1C3729
:10B67000BD46BDE8F08F00BF5423002040230020CA
:10B68000082C0020F01E0020D82200202DE9F04FC9
:10B690004FF0000883B001928246894644460D9DD2
:10B6A0004F4E504ADFF854B125E0002323540029BF
:10B6B00059D13AF914104C4F22F8141039F91400EA
:10B6C0004A4B27F814003AF9140049492BF81400A2
:10B6D00039F9140023F81400019B33F914002B7876
:10B6E00021F8140031190B7008F1010801340A2CFB
:10B6F00005F1010533D02B78311900913D48315DBA
:10B70000002BD2D13B48DFF8E4C0DFF8F4E0002999
:10B71000ECD0215C3BF81470013149B2DEF800E056
:10B72000215422F814703CF814002F4F714527F86B
:10B730001400DBDD30482E4927F8143022F814308D
:10B7400037192BF814302CF8143020F8143021F865
:10B75000143001340A2C3B7005F10105CBD1404671
:10B7600003B0BDE8F08F204F32F9143039F914C01E
:10B7700037F914103AF91400ACEB0101C01A009229
:10B7800000F02AF91C4B3BF914C023F814003AF9D5
:10B790001430009AA3EB0C0C144903EB6C0322F851
:10B7A000143039F9143031F914C01148A3EB0C0CE2
:10B7B00003EB6C0327F814303AF9143095F800C005
:10B7C0002BF8143039F9143021F81430019B311959
:10B7D00033F9143081F800C020F8143084E700BF3A
:10B7E000082C002040230020542300202C2300207C
:10B7F00004230020EC220020D8220020182300205F
:10B80000F01E00202DE9F04F4FF0000983B0CDE984
:10B8100000129846594D5A4B824695E8070003C3DB
:10B820004C460D9EDFF880B11A8034E00021544F61
:10B830009E42DFF864E1DFF868C15248524A395548
:10B840005DDB3AF91410514FA35CE9530099504F56
:10B8500031F91410E9533AF914104E4F25F80B1032
:10B86000009931F9141025F80E10019931F91410CE
:10B8700025F80C1038F9141079530C99095D2154EE
:10B880000C99095D8B4238BF0B46A35409F101099D
:10B8900001340A2C2FD038F914203E4BB2424FEA23
:10B8A000440533F91430C1DC9E423B4A3B49EFDA90
:10B8B000334F35F80B003B5D096801335BB23B55F4
:10B8C000324F35F802C0E85331488B4225F800C0AA
:10B8D000DEDD0023AB522E4A2A49AB522D4A3048B6
:10B8E0005353294A6354A35401340A2C25F80B30CE
:10B8F000EB532B52CFD1484603B0BDE8F08F244B19
:10B90000009FEA5E214B37F91410EB5E3AF9140000
:10B91000891AC01A00F060F8224B35F90B10585301
:10B920003AF914301C4A591A03EB61031749A85E0F
:10B930006B5237F914301A49181A03EB6003144894
:10B940002B523AF914300F4825F80B3037F91430E0
:10B95000104FAB52019B0C4A33F914306B5238F93B
:10B960001430A15C7B530C9B1B5D23540C9B1B5D13
:10B970008B4238BF0B46A35488E700BFEC2200205F
:10B98000F82200208C2D0020CC2B00207C330020BE
:10B99000DC2B0020B02C002090330020F01E002073
:10B9A000A4330020D8220020642D0020884210DB20
:10B9B000904210B40ADA441A0198521AC01A04FBD1
:10B9C00000F494FBF2F210BCD0187047019810BC40
:10B9D00070471846704700BF81EAE173A3EBE1733B
:10B9E00018B30028B8BF4042F1B198421FDA820173
:10B9F00092FBF3F2402AA8BF402211498A5CC2F1AF
:10BA00005A028AB10F4910B4C2F15A0431F8122017
:10BA100031F8141003FB02F300FB01F01B1403EBDD
:10BA20002043184610BC70470346184670479A01D9
:10BA300092FBF0F2402AA8BF402201498A5CE0E76D
:10BA4000D4B4010018B5010088420ADB40B1890175
:10BA500091FBF0F04028A8BF4020094B185C7047CC
:10BA6000704751B1800190FBF1F14029A8BF4021FE
:10BA7000034B595CC1F15A0070470846704700BF3C
:10BA8000D4B4010070B40E680C89022E25DDA042EA
:10BA900023DB0B460125013E02E0844206DC15460D
:10BAA0006A1C96429C8903F10403F6D101EB8505DB
:10BAB000AE88ED88A6420DD001EB8201CB88001B39
:10BAC0005D1B00FB05F0A41B90FBF4F41C4420B2AA
:10BAD00070BC704728B270BC704700250122E5E7B2
:10BAE0007F280CDC402824DA0F2824DC082827DAF9
:10BAF000022829DB0428B4BF012002207047B0F5DA
:10BB0000806F08DAB0F5007F1CDAB0F5807FB4BF33
:10BB1000072008207047B0F5805F05DAB0F5006FA8
:10BB2000ACBF0B200A207047B0F5005F0CDA0C2088
:10BB30007047062070472028B4BF042005207047B6
:10BB40000320704709207047002070472DE9F04F0F
:10BB5000056889B01446ADB1394D3A4F3A4E4FF4AD
:10BB600080722B460092394600226020F6F7EAFDEB
:10BB700040F201122B460092314622466420F6F72D
:10BB8000E1FDECE7314A81461368084601338A46F5
:10BB900013600EF097F9C9F8000020B12C4B00EBB0
:10BBA0000A029A423CD9264F0025B846DFF8B0B0C9
:10BBB00040F20B1243460092264900226420F6F719
:10BBC000C1FD0426012240F20F13D9F800001146EE
:10BBD00000EB0A0C0593069006ABCDE903B7CDE95F
:10BBE000015500966420CDF81CC0F6F763FD0122D4
:10BBF0004FF4887318490593CDE9025107AB1146FC
:10BC00000096049701956420F6F754FD40F2111256
:10BC100043460092214600226420F6F793FDC7E7D1
:10BC20000E4A2B46114602E00133322B05D051F863
:10BC3000044B002CF8D142F8230009B0BDE8F08F86
:10BC40007CB4010084B4010088B4010030240020D9
:10BC5000AC440020A8B40100C8B40100682300204F
:10BC6000BCB401002DE9F04F8046006889B08946D8
:10BC7000C0B12F4D00232A4602E00133322B1DD0E4
:10BC800052F8041B8142F8D1002445F823400EF0FD
:10BC900021F9284AC8F800401368013B136009B035
:10BCA000BDE8F08F4FF491730A4600932249234B6D
:10BCB0006420F6F747FD09B0BDE8F08F1F4E002461
:10BCC0003746DFF880B0DFF880A04FF497723B462C
:10BCD00000921B4900226420F6F734FD042501225E
:10BCE0004FF49873D8F8001064200791059311461B
:10BCF00007ABCDE903B6CDE901440095F6F7DAFCD0
:10BD000040F231123B460092494600226420F6F789
:10BD100019FD4FF499730A2205930095CDE903A606
:10BD2000CDE901441146024B0020F6F7C3FCCCE7F5
:10BD3000682300203024002020B401007CB40100DE
:10BD400040B40100CCB4010068B40100134B1B687F
:10BD5000002B22DD2DE9F041114C4FF00008274661
:10BD6000104E114D86B040F23F123B4600922946DC
:10BD700000226420F6F7E6FC01224FF4A0710423B0
:10BD800005910093CDE90364CDF808800192114636
:10BD9000024B6420F6F78EFCE5E770473024002064
:10BDA0007CB40100ECB50100D0B5010010B504462B
:10BDB000FCF7BAFC04F1F80104F1BC00FEF706FD43
:10BDC00004F59A70FBF754FA04F5FA70FBF760F883
:10BDD00004F5FC70FEF7CCFB04F50370FBF73AFFAB
:10BDE00004F51070FEF774FE04F51F70FEF726FFD1
:10BDF00004F52370FCF792FC04F2053001F038FBE7
:10BE000004F29220FBF7C8FF94F892320BB9FBF7CB
:10BE1000C9FF04F52570FBF7B1FD04F53A70FEF794
:10BE2000FBFA04F53C70FCF76BFC04F5427000F083
:10BE30003DFE0023044C194623604FF47072BDE8A8
:10BE4000104002480EF059B814210020A82F0020FD
:10BE500038B9064A136801338B4205DD10600120B2
:10BE6000704700231846014A1360704714210020D0
:10BE700008B5FBF795F8FEF7D7FAFEF7EBFEFBF7F0
:10BE800091FFFBF783FDBDE8084001F0E9BA00BF70
:10BE90000022014B1A60704734240020024A1368C4
:10BEA00001331360704700BF34240020014B186831
:10BEB000704700BF34240020014B33F81000704756
:10BEC000FCB5010038B500240A4B0B4D21464FF458
:10BED0002072C3E90044C3E902441C6107482C6096
:10BEE0000EF00BF82146BDE838404FF49672044836
:10BEF0000EF003B8902B00203C24002040240020AA
:10BF0000C02600202DE9F04F00261F460D4691B0B7
:10BF10000DF1200881461446314640462022CDE9E5
:10BF200005660496CDF81B600DF0E7FFBB10DFF847
:10BF300008B10A2BB8BF0A23B542CBE90066CBE9AA
:10BF40000266CBF8106060DDCDE9016604AF4FEA10
:10BF5000490AC9EBC97E039607EB050C04EB0A02FC
:10BF60004FEA4E0EB9F1000F14DD00210EEB020076
:10BF700030F9024B9C4207DD3E7811F8085001363B
:10BF800001353E7001F808501F2901F1010131DD32
:10BF90009042EDD1013767455244E3D1019BBBBBD1
:10BFA0009DF820509DF81030002630463746314627
:10BFB0000DF111020DF11F040BB1012630448B422B
:10BFC000C4BF19460127944202D012F8013BF3E79F
:10BFD0007FBB5EBB00210B460DF125020DB1012197
:10BFE0000B44904502D018F8015FF7E7D9B911B0BA
:10BFF000BDE8F08F039DA542B8BF254603950125F6
:10C000000195029D25440295C2E733463546CBE7AC
:10C01000029B9DF82050CBF80C30039BCBF81030DE
:10C020009DF81030C0E7CBF80830E0E7CBF800000F
:10C03000D0E7CBF80410CCE7AC2B00202DE9F04F73
:10C0400097B000AFC7E90432D7E920CED7F89C30CB
:10C050000028BB61D7F8A030F961D7F8C040D7E914
:10C060002E517B607862386240F37281C04EC14BC2
:10C070003068994603EB8013786A023A4000B86052
:10C08000023B02EB000832F9020F904523F8020F41
:10C09000F9D12368FB60FB69002B19DD3B6932682D
:10C0A000A3F102084346B448C2EB021200EB42027D
:10C0B000F869023A08EB400633F9020FB34222F85E
:10C0C000020FF9D13B6A002B40F36481A94B9946DA
:10C0D0000022C7F8C04047F6FF764C46C7F8BC10B0
:10C0E000DFF8AC8279697A6200234FEA420B786A02
:10C0F00004EB0B09C34439F940ABCB455344FAD1A7
:10C10000824678629D4880FB0309DB17C3EBA903D5
:10C110001BB2002B21F81230994602DD504618441C
:10C1200078629E42A8BF1E469C450CDAB5F808907E
:10C130002B6809F10109A5F8089031F91290A9EBD3
:10C140000C0A53442B60CE450CDDB5F80A906B68A1
:10C1500009F10109A5F80A9031F91290A9EB0E092D
:10C160004B446B60022A40F329813B6A01329342BF
:10C17000BADCD7E92F14FA68AE811546804B786A8D
:10C1800083FB0553A3EBE2732360E3683A6AFB6029
:10C19000FB6990FBF2F0002B40F3E4803B69A3F1D4
:10C1A0000208002247F6FF7C96464646724DDFF8AD
:10C1B000CC81D7F8049038612846002305F5967B9A
:10C1C00030F91EAB83455344FAD188FB03A0DB173B
:10C1D000C3EBA0031BB29E45B869B8BF9E469C4501
:10C1E000A8BF9C46834226F8023F0CDD0B890868F5
:10C1F00001330B817862B6F90030B869A3EB000A0D
:10C20000786A50440860994509DD4B8948680133D4
:10C210004B81B6F90030A3EB090A50444860012A6B
:10C2200023EAE37002DD0E2A40F0C3806369034411
:10C230006361FB690132934205F10205BCD13869A3
:10C240000FFA8EFE0FFA8CFCBD68A1F80EC02B46CB
:10C25000083323F00703ADEB030DFB69A1F80CE0F5
:10C26000A3F1040C3B6A6946002B38DD7B6900268C
:10C270009A1E154440F24458A946A1F1020E32F923
:10C2800002AF256AAAEB000323EAE3731BB2AAF10B
:10C29000970AAB421FFA8AFAC8BFC4E90763C245CE
:10C2A0002EF8023F06F1010602D8A3690133A3610B
:10C2B0009145E4D1B1F90030002B10DDA36A3A6A50
:10C2C0001A441046013304E031F9022F002A40F3EA
:10C2D000988098421D4603F10103F5D1A06247F60C
:10C2E000FF70FB680326984293FBFCF1B8BF184629
:10C2F0000023244AC7E90F33C7E91133C7E91333D1
:10C300007B65214D214BA16000B207F12C01C7E9EB
:10C310000D23C7E90B65FFF7B5FBE2686369012AE6
:10C320001146B8BF01219B0193FBF1F323EAE373AC
:10C33000984209DAE369B34206DD41F287339A4253
:10C3400002DC012384F824305C37BD46BDE8F08F61
:10C350002368FB60FB69002B41DD3B6A044E5B00F8
:10C36000BB609BE647F6FF7C4FF0000E6CE700BF1A
:10C370003C24002040240020C0260020676666661A
:10C3800056555555E8034000F4013200D0074000EF
:10C39000C026002047F6FF72AA81FA681A4B1046A1
:10C3A00083FB0003A3EBE2732360E3680020FB60E0
:10C3B000F7E6FB680344FB60E3603AE731F912906B
:10C3C000F868D7F8C030B9F1000FA8BF48445B68DF
:10C3D000F8609944D7F8C030C3E90009C5E647F6CC
:10C3E000FF70FA69084BA2F1040CFA68A88183FB7C
:10C3F0000263E068A3EBE273044A2360F860CA605A
:10C400006DE7A5626BE700BF565555550000FF7FED
:10C410000020F0B4384E8C1E186058609860D860C8
:10C42000186104311D1F34F9020F002821DD87B285
:10C4300007F1FF3CBCF1090F11D9A7F10B0CBCF1BE
:10C44000090F1CD9A7F1150CBCF1090F1FD800EB7F
:10C4500040004000A6FB0070C008033080B2A1423B
:10C4600045F8040FDFD1F0BC2449DA600A791A617B
:10C4700070470020A14245F8040FD4D1F3E74010E3
:10C48000053080B2A14245F8040FCCD1EBE7A7F10B
:10C490001F0CBCF1090F0BD9A7F1290CBCF1090F36
:10C4A00011D8C000A6FB0070C008043880B2D6E7DF
:10C4B000C0EBC000A6FB0070A1424FEAD00045F8D7
:10C4C000040FB0D1CFE7A7F1330CBCF1090F0BD9A2
:10C4D0003D3F272FC3D8C0EBC0004000A6FB007033
:10C4E000C008263880B2BAE700EBC000A6FB007097
:10C4F000C008093880B2B2E7CDCCCCCC902B00205C
:10C5000084B02DE9F047002482B081460BA880E872
:10C510000E00524D9DF85070DFF86C81504EDFF8E0
:10C520006CA115F8013BD3B9119B122B02DCB9F1B8
:10C53000000F34D04FB340F2851233460092494980
:10C5400000224920F6F7FEF8002305F8043C0134E8
:10C55000032CE6D102B0BDE8F04704B0704708EB09
:10C560004403DB880B9A9A4202DD0D9B1E2B3BDCB9
:10C570004FF4CC7233460092514600224920F6F720
:10C58000E1F8002305F8043CE1E740F28912334664
:10C59000009235493A464920F6F7D4F8D7E74FF4E8
:10C5A000B6722F4B009231494A464920F6F7CAF835
:10C5B000129B062BCBDD002F44D1109BB3F57A7F65
:10C5C00036DD159B052B33DC139BB3F5FA7F2FDA91
:10C5D0004FF4BC723346009225493A464920F6F79B
:10C5E000B1F805F8047CB2E74FF4C7721C4B009217
:10C5F000204900224920F6F7A5F8012305F8043C5C
:10C6000067B14FF4C972334600921B49002249209A
:10C61000F6F798F8002305F8043C98E740F29512E5
:10C620003346009215493A464920F6F78BF88EE7D3
:10C6300040F27D1233460092114900226420F6F741
:10C6400081F884E740F27112334600920D494A4660
:10C650004920F6F777F805F8049C78E7932B00203B
:10C6600024B70100E4B7010020B8010038B7010089
:10C6700088B7010054B8010070B80100A0B80100EB
:10C68000ACB7010060B70100FCB50100B0B8010013
:10C6900082B000B583B0069A0593012A23D0E8B191
:10C6A000591001EB4301914202DCD91E032926D91E
:10C6B000023A032A12D8079A012A0FDD023B032B04
:10C6C0000CD84FF4E472134B009213490022492016
:10C6D000F6F738F80022114B5A709A7003B05DF8E3
:10C6E00004EB02B07047042BD9DC4FF4DC72094B29
:10C6F00000920B4900224920F6F724F8EAE74FF4AC
:10C70000E072044B0092074900224920F6F71AF81C
:10C71000E0E700BF24B70100F4B60100902B002031
:10C7200088B60100C8B6010084B0F0B587B00CAC83
:10C7300084E80F000D9B002B45DB40F2EB13284DE6
:10C74000009300222B4627494920F5F7FBFF4FF4C1
:10C75000F6722B460092244900224920F5F7F2FF99
:10C760000124002640F2ED120427204BCDE90452AB
:10C7700021462246039364200DABCDE90146009784
:10C78000F5F798FF4FF4F770194B22460590039385
:10C7900004951AABCDE90146009721466420F5F7D0
:10C7A00089FF40F2DC530C9A9A4207DC43F6982347
:10C7B0001A9A9A420F4BCCBF9C709E7007B0BDE88E
:10C7C000F04004B0704742F210731A9A9A4203DDA7
:10C7D0000122084B1A70B0E70022064B1A70ACE732
:10C7E00024B7010020B601003CB6010054B6010098
:10C7F0006CB60100902B00202DE9F043204C214F16
:10C80000DFF88490DFF8848083B0E61CE07814F8C9
:10C81000015BB8B9E5B163790133DBB20A2B63710F
:10C820000BD940F2092301250246009360713B4673
:10C8300041466420A570F5F785FFB442E6D103B008
:10C84000BDE8F08345B10023B4422372DED1F6E7A0
:10C85000B4426571DAD1F2E7237A0133DBB2282BD7
:10C860002372EAD940F213223B46009249462A46F7
:10C870006420A570F5F766FFB4422572C6D1DEE7E5
:10C88000902B002024B70100ECB80100DCB80100B7
:10C8900000212DE9F047984601270B468CB025482A
:10C8A000DDF850A0179D199E234C914601808170A0
:10C8B000C21C12F8011B31B934F813108D4202DD8D
:10C8C0001E2EC8BFC7540133032BF2D16C461AADDC
:10C8D0000FCD0FC495E80F0084E80F006C4617AF2A
:10C8E00097E80E004046FFF70BFE23AB0FCB8DE819
:10C8F0000F0014AE52464146484656F8383FFFF7FF
:10C90000C7FE0FCE0DF11C0CACE80F0033681BAD59
:10C91000CCF800300FCD0FC495E8070084E807007D
:10C9200097E80F00FFF700FF0CB0BDE8F047FFF7F6
:10C9300063BF00BF902B0020FCB501002DE9F04F34
:10C94000A3B00025DDE93D876E4681468A4617ACD7
:10C95000159220462C2200219B460DF0CEFACDE9FF
:10C960000F74CDF838800DF1D80C0DF11C0EBCE819
:10C970000F00AEE80F009CE807008EE807000DF1FD
:10C98000BC0CBCE80F00C8F80050C8F80450C8F848
:10C990000850C8F80C50C8F810503D607D60BD606C
:10C9A000FD603D610FC69CE807002E9B86E80700EE
:10C9B000314E2D9A514648460EAFFFF73FFB0FCE42
:10C9C0000FC736680FCC3E6003AE0FC60FCC0FC644
:10C9D00094E8070086E807002E99284E02912C99CA
:10C9E0005B4600912D99159A019148465146FFF7F3
:10C9F0004FFF33682D9901330A2B14BF1C462C4678
:10CA000048463F9B179A3460FFF702FD3F9B1C4A44
:10CA1000D9684098D37881828DF85B50E3B9117959
:10CA200018465279F1B91ABBF8B9012240F27A21BD
:10CA30000023144C14480591CDE90133CDE90304DA
:10CA4000009211460DF15B036420F5F733FE9DF86B
:10CA50005B0023B0BDE8F08F0120117903465279C5
:10CA60000029E0D043F0020312B98DF85B30DCE717
:10CA700043F00403F9E700BFAC2B00203C24002066
:10CA8000902B002024B70100A0B7010030B9064B5D
:10CA9000187810B10138C0B2187070471423024AD8
:10CAA00018461370704700BF3824002001464FF429
:10CAB000A87201480DF016BA001F0020014B18782B
:10CAC000704700BFF52700202DE9F04F4FF0000818
:10CAD000C146D5B014AD029200218022284634AE62
:10CAE0000393629C0DF009FA8022002130460DF07C
:10CAF00004FA05A83C2200210DF0FFF9631E019302
:10CB00004A4BDFF830C193F9024093F801A005AF1A
:10CB1000CDF80080019B13F801EF0193002301E0A1
:10CB2000202B28D03CF91320A24207DA55F8231015
:10CB3000501D014409F1010945F8231092450BDA13
:10CB400056F823003968A2F1050B5844594408F1FE
:10CB5000010846F823003960BEF11F0F03F10103FD
:10CB6000DED1A242DCDA61990029D9DD0099202BBF
:10CB700011440091D6D10437BD420CF1400CC9D10B
:10CB800000210F46294BDDF800E09C88B3F90660D0
:10CB9000B3F908C053A833AB53F8042F002A08DDBB
:10CBA000A24206DA55F82120B24202DAF445B8BFB3
:10CBB0000137984201F10101EED1029BB3F57A6F82
:10CBC0001BD9B8F1500FD4BF0021012140F2EE2350
:10CBD000059A9A420FDD13989842D4BF0020012095
:10CBE00017B1B8F1050F0ADC00231846104A13608C
:10CBF00055B0BDE8F08F0020F2E70021E6E7B9F17B
:10CC00000A0FF1DD039B052BEEDD0029ECD1002896
:10CC1000EAD1064B064A1978639C1368214499426D
:10CC2000CBBF0133106013600120E1E7001F00203B
:10CC3000EC270020A82F002070B588B09DF8685020
:10CC40009DF86C60C0B9B9B9354C2178C9B1132AC7
:10CC500047DC0D9A632A44DC133342DB0C9B092B1F
:10CC60003FD8304B304AD9691368994251DD0121D0
:10CC70000B44136021701BE00022294B1A7008B08E
:10CC800070BD1999104604911799CDE90556039185
:10CC90001699029115990191149900911946DDE9AF
:10CCA0000C23FFF711FF207010B12048FAF7F0F8BD
:10CCB000FDF738F924780546FCB11D4C1D4E23883C
:10CCC000327801331BB22380002AD8D1632BD6DD02
:10CCD0000220FDF7D5FA01236422AB77337022805E
:10CCE000CDE7104B0D99B3F918209142BADC002220
:10CCF00001210D4B21701A60DAE70E4E0C4A337891
:10CD00001480002BBBD00320FDF7BAFAAC77347047
:10CD1000B5E70023084813602370FAF7B9F8C7E7AE
:10CD2000F5270020001F0020F027002006DE01006C
:10CD3000F6270020F4270020A0DC0100054A92F825
:10CD40005030834204DA8B42B4BF00200120704788
:10CD500001207047001F00204B28CCBF002001207D
:10CD6000704700BF2DE9F04F013883B000280191D2
:10CD70006CDD012872D04FF000094FF0010C09EB77
:10CD8000000303EBD3735B1032F9131032F9104038
:10CD90004500A14204DD22F813400C4622F8101091
:10CDA00032F919104FEA490BA14202EB0B0A04DDDC
:10CDB00022F81940515332F9191032F913408C42BC
:10CDC00005DD22F8131022F80B4032F91340064615
:10CDD0000BF10201555E02EB4C0E22F81350545237
:10CDE00032F90B503EF9028F0CF1010CA845F9DB2A
:10CDF000711E02EB410301E00E4601391F4633F973
:10CE00000249AC42F8DC8C4507DCAEF80040A7F8DC
:10CE100000800E46BAF90050E4E7019B22F80B406F
:10CE20008B423D8018DBE14616DD48450EDD09F1F9
:10CE3000010C8445A3D102EB49094000B9F9003047
:10CE4000115E8B42C4BFA9F800101352019B32F946
:10CE5000130003B0BDE8F08FB01EE6E79146022054
:10CE6000ECE700BF2DE9F04F013800EBD07383B041
:10CE70005B10002801936CDD012872D04FF000098F
:10CE80004FF0010C09EB000303EBD3735B1031F996
:10CE9000132031F910404500A24204DD21F813406F
:10CEA000144621F8102031F919204FEA490BA2420B
:10CEB00001EB0B0A04DD21F819404A5331F919201E
:10CEC00031F91340944205DD21F8132021F80B407D
:10CED00031F9134006460BF102028D5E01EB4C0E58
:10CEE00021F813508C5231F90B503EF9028F0CF19E
:10CEF000010CA845F9DB721E01EB420301E0164666
:10CF0000013A1F4633F90249AC42F8DC944507DC8C
:10CF1000AEF80040A7F800801646BAF90050E4E7E2
:10CF2000019B21F80B4093423D8018DBE14616DD62
:10CF300048450EDD09F1010C8445A3D101EB4909F7
:10CF40004000B9F900300A5E9342C4BFA9F800203E
:10CF50000B52019B31F9130003B0BDE8F08FB01EF6
:10CF6000E6E789460220ECE7831A042B10B413DDB0
:10CF7000DC1EB1F90430002A0B804B8031F91430EB
:10CF800008DD4000A0EB42020A44014421F8023DC2
:10CF90008A42FBD110BC70475C1E032C08BF9C1E4C
:10CFA000E7E700BFF0B40446049E0846DDE90551FA
:10CFB000A642DDF81CC019DD04F10044AF1E013C9F
:10CFC00007EB460705EB44058E1C06E09C42B8BF04
:10CFD0001C46BD4226F8024F08D035F9024F944254
:10CFE000F4DD1446BD4226F8024FF6D1F0BC62468D
:10CFF000FFF7BABFF0B400280F46DDE90561DDF8A0
:10D000001CC014DB013006EB40048D1C06E0984286
:10D01000B8BF1846B44225F8020F08D034F9020D03
:10D020009042F4DD1046B44225F8020FF6D138469E
:10D03000F0BC6246FFF798BF2DE9F043B1F90090CC
:10D0400002284FEA4918DDE90767C2E90088DDE9EF
:10D0500009CE21DD8C1E5B0176017F01043204EBD9
:10D060004000023103E0A84631F9029C0432B1F9D4
:10D070000050B1F9024006FB05F503FB04541568A6
:10D0800002310CFB054407FB094408FB0E448142B6
:10D090004FEAA4245460E6D1BDE8F0832DE9F041C5
:10D0A000884684B04C00083404AFBD6B24F00704FC
:10D0B000ADEB040DBE690395FD6904AC01950096C6
:10D0C00002947D6BFFF76EFF3B6B21460293FB6A78
:10D0D00003950193BB6A40460093D7E90823FFF705
:10D0E000ABFFBD46BDE8F0812DE9F041884684B034
:10D0F0004C00083404AFBD6B24F00704ADEB040D05
:10D10000BE690395FD6904AC0195009602947D6BA0
:10D11000FFF770FF3B6B21460293FB6A0395019377
:10D12000BB6A40460093D7E90823FFF785FFBD4659
:10D13000BDE8F0812DE9F04F8FB00AAF7D6D9A46C2
:10D140001B1A023300F103088B465919FB6B18EBCD
:10D15000050804461646FB6000F0AA804FEA8809DD
:10D16000002934D109F10A0929F00709C7F808D0C4
:10D17000ADEB090D08953E6D0DF128090796FE6C83
:10D1800013460696BE6C5A4605967E6C414604963A
:10D190003E6C0396BE6BCDF80890CDE900A6FFF774
:10D1A000A3FF002C0DDBFE680235013409EB850975
:10D1B00006EB440459F8043B5B1124F8023DA642F7
:10D1C000F8D1D7F808D01437BD46BDE8F08F8B00F2
:10D1D0000A3323F00703C7F804D0ADEB030D08951D
:10D1E0003A6D0AAB0792FA6C09F10A090692BA6C19
:10D1F00029F0070905927A6C04923A6C0392BA6B93
:10D20000CDE900A2BB605A4602933346FFF746FFC2
:10D21000ADEB090D0895396D0DF128090791F96CF1
:10D2200033460691B96C5A460591796C20460491B3
:10D23000396C0391B96BCDF80890CDE900A1414656
:10D24000FFF752FF631C9A4511DDFE68BA68E91CBE
:10D25000B31E02EB810103EB4A0A06EB440251F8CC
:10D26000043B5B1122F8023F5245F8D1FE60002CCE
:10D270000DDDFE68E91C09EB810106EB440251F863
:10D28000043B5B1122F8023D9642F8D1FE60BB6878
:10D29000023559F8252053F825301344FA689B11BC
:10D2A00022F81430D7F804D01437BD46BDE8F08F0B
:10D2B0008B000A3323F00703E946ADEB030D089515
:10D2C0003E6D0DF128080796FE6C13460696BE6C5F
:10D2D0005A4605967E6C04963E6C0396BE6BCDF85E
:10D2E0000880CDE900A6FFF7D9FE544512DAFA68A6
:10D2F00004F10044013C0335931E02EB440608EBA5
:10D30000850803EB4A0A58F8043B5B1126F8023FF4
:10D31000B245F8D1CD461437BD46BDE8F08F00BF09
:10D320002DE9F04788B099464FEA430808F1080410
:10D3300024F0070408AFADEB040DD7E90D563C6BA4
:10D34000CDE90656BD6AFE6A059403953C6A7D6A7E
:10D35000049608AECDE901650094FD6BFFF7EAFE87
:10D36000B9F1000F10DD023CA044A6F1020A34F925
:10D37000023F3AF9022F9B1AAB42CCBF5B1B03EA78
:10D38000E37344452380F2D1BD46BDE8F08700BF7A
:10D390001E232DE9F041264E86B00D4680460093AF
:10D3A00024493346642014460022F5F7CBF90027C0
:10D3B0004FF01F0C012204211F482B46CDF814C04A
:10D3C00000910390114664200496CDE90177F5F7AA
:10D3D00071F94FF0240C0120184AA5EB0801490906
:10D3E000009003920496CDE901774346CDF814C02E
:10D3F00020226420F5F75EF9294651F8043BA34248
:10D40000FBD02B2700220124C5F11F030C4819442F
:10D41000CDE901220390049649092B460597009413
:10D4200020226420F5F746F906B0BDE8F08100BF80
:10D43000FCB8010008B901001CB9010028B90100BD
:10D4400040B901000B68934209D070B50D461446EF
:10D450000646224629463046FFF79AFFF9E770470D
:10D460000022024BC3E900221A8170477028002075
:10D470000278014B1A70704750200020314B1B7806
:10D48000002B5AD02DE9F04F16462F4A87B0894617
:10D49000804600242D4F1368DFF8B4B0DFF8B4A045
:10D4A000013E14E03D5D38F91410022D2BF81010E8
:10D4B00005F1010E39F914109CBF5FFA8EF53D5548
:10D4C000032D2AF8101017D001340A2C0CD04FEA83
:10D4D000440C0CEB0401C81816F8011F0029E1D117
:10D4E000395501340A2CF2D10133022BC8BF002375
:10D4F000136007B0BDE8F08F0CEB04035B000BEB8F
:10D5000003010868534402901868B1F804C09B886E
:10D51000049002A928460192ADF81430ADF80CC071
:10D52000FFF7A0FC04A928F814002846FFF79AFC8E
:10D53000019A29F814001368C6E7044AC2E90033C7
:10D5400013817047502000207C2800207028002084
:10D55000F827002034280020F0B483000A3323F099
:10D560000703002800AFADEB030D30DD6B4600264E
:10D570000439B20002F1804292F880C292F88152DE
:10D5800092F8824292F883225FFA8CFCEDB2E4B208
:10D59000D2B2013683F800C05D709C70DA70BCF1C5
:10D5A000000F03D00CF1FF3C83F800C01E2D9CBF80
:10D5B00001355D700CB1013C9C700D2A9CBF01329D
:10D5C000DA7053F8042BB04241F8042FD1D1BD4694
:10D5D000F0BC704792F83230002B43D1F0B50028F0
:10D5E0008BB00E460546144610DD936A42189A42E7
:10D5F00010DB00231A4684F8313094F8243093422B
:10D600009CBF012384F830300BB0F0BDF1D1D36A58
:10D610008B42EEDD2E2294F83130134F013384F823
:10D62000313012493B46009264200022F5F78AF817
:10D630004FF0340C0020012104220D4B049794F884
:10D640003170CDE90110009203930322CDF814C08C
:10D6500007AB6420CDE908650797F5F72BF894F838
:10D660003120CAE7704700BF54B9010068B9010012
:10D6700090B901002DE9F04F98468DB0DDE91653C1
:10D68000012DA946B8BF4FF00109012B9C464FF070
:10D690000004B8BF4FF0010C189E09923788B6F805
:10D6A00004E01268D8F8006005FB072503FB0E664E
:10D6B000002895FBF9F596FBFCF6CDE90A442ADD36
:10D6C000A446A146A246023901EB40000894CEF1DF
:10D6D000000B079031F9023F5A1B22EAE2723344F1
:10D6E00003EAE37397420EEB030403DC0120D21B31
:10D6F000089092445B4505DC4FF0010C002CB8BF4C
:10D700006442A144079B9942E4D1089B002B49D174
:10D71000BCF1000F49D10124002604255C22244FCE
:10D72000DDF82490234B059221462246CDE90337AC
:10D73000CDE901464B4600956420F4F7BBFF5D2020
:10D740001D4B224621460590039304974346CDE99D
:10D75000014600956420F4F7ADFF5F20174B224689
:10D7600021460590039304970AABCDE90146009545
:10D770006420F4F79FFF6020114B2246059003932D
:10D7800004970BABCDE90146009521466420F4F7E0
:10D7900091FFDDE90A23C9F80020C8F800300DB078
:10D7A000BDE8F08FCDF828A0B2E7CDF82C90B2E715
:10D7B00054B90100A0B90100B0B90100C0B901001D
:10D7C000D4B9010070B19A4215DC0F4A1368C72B17
:10D7D00001DC013313600D4B187808B181F00100B2
:10D7E00019707047084B1A68C72AF4DD1860074B98
:10D7F0000120197070470022034B1A60034B187800
:10D800000028EDD0EAE700BF8428002090280020FF
:10D810002DE9F04FBD48ADF2AC4D1893DDF8E8446A
:10D820000378CDE915121993002C00F07A850DF1DB
:10D83000E40AD0AD3C220021504631AE12950CF0E6
:10D840005CFB78220021284613960CF056FB1E2222
:10D85000002130460CF051FB002326AAC2E9003318
:10D86000ADF8A03001232046294617921E93FFF7FA
:10D8700073FEDDF8E84420220F23DDF8E014CDE943
:10D8800003320691DDF8E414B2AB059112992046FB
:10D89000019113990293009194AA76A95346F9F73E
:10D8A00097F9DDF8E804002840F3F185002253469B
:10D8B00014460AEB400133F9022B02B101348B42CA
:10D8C000F9D11F940A2420260F25DDF8E0340194B5
:10D8D0000C93DDF8E4348E4C0B93B2ABDFF848C206
:10D8E000129F8C498C4A08930694139B8B4CCDE96C
:10D8F00002C2CDE90414009394AA534676A907976F
:10D90000CDE90956FBF76CF940F22F2000240123E2
:10D910000590DFF818B282483246294600930390FA
:10D92000DDF8E4346C20CDE90144CDF810B0F4F713
:10D93000C1FEDDF8E024139B0692DDF8E424DDF857
:10D94000E8040592B2AACDE901720093CDE903562D
:10D95000534694AA76A9FBF787FADDF8E804A042BB
:10D9600008DD53460AEB400133F9022B02B10134C2
:10D970008B42F9D1209420250F24DDF8E034129E4B
:10D980000693DDF8E434139F0593B2AB0293CDE91F
:10D990000345534694AA76A901960097FBF7A6FB88
:10D9A000DDF8E034CDE903450693DDF8E434DDF835
:10D9B000E8040593B2ABCDE901630097534694AAFE
:10D9C00076A9FBF7A3F8DDF8E844002C40F3638563
:10D9D0000022534610460AEB440133F9022B02B1F0
:10D9E00001308B42F9D12190EEAE782200210DF565
:10D9F000866530460CF081FA7822002128460CF02A
:10DA00007CFA20210F22474B20461C68DDF80C359C
:10DA10006478B3F924300894DDF8E044CDE90321BB
:10DA20000694DDF8E44407930594129C534601954F
:10DA30000096029494AA76A9FCF7F6FEDDF8E83485
:10DA4000002B40F32085002448AF149755F8041BA1
:10DA500056F8040BFDF7C0FFDDF8E8340134A342AB
:10DA600027F8020BF2DC0F252026DDF8E014DDF8A4
:10DA70000C25149FB2F924200791DDF8E414184610
:10DA80000691B2A903911299CDE904560291139916
:10DA900008920191534694AA76A90097FBF7B6FC29
:10DAA000002440F28F20012329461D4D3246059067
:10DAB00000936C20DDF8E434CDF810B00395CDE987
:10DAC0000144F4F7F7FD534694AA76A9DDF8E8047B
:10DAD000F9F708FC2046DDF8E814CDF800A094AB77
:10DAE00076AAF9F7DBF9DDF8E804A04220DD3A4632
:10DAF000662407EB4001B2F9003004FB03F39B12EC
:10DB000022F8023B8A42F6D112E000BF5D160020E7
:10DB1000A8280020B02C0020DC2B00209428002016
:10DB2000E8B90100340A00207C33002054B9010018
:10DB3000129B94AA0293149B76A9009329AB01939C
:10DB40005346FCF72FFDFCF7EDF91C90FEF7B6FFEE
:10DB5000002835D1199B022B1C9B9B7928D0DDF81E
:10DB6000142503F0FF0102F510721A92002B40F009
:10DB70002E84199B012B20D11C9BDB7FEBB128222B
:10DB800067A80CF0BAF94FF4AF720A23642046215B
:10DB9000022566ACC4E90B01E28020466281238144
:10DBA0002560C4E90D330DF5AE79FCF791FF0AE06D
:10DBB000002B40F00A84AD4B1A931A98FCF788FFAB
:10DBC0000DF5AE7966AC0026DDF8E8342660B34288
:10DBD0004EDDCDF86890DFF8AC82DDF850904FF460
:10DBE0003F7243460092A24900227020F4F7AAFD3A
:10DBF000012540F2FD2204239E490592CDE90261F0
:10DC00002A462946009370202346CDF810B001958E
:10DC1000F4F750FD022740F2FE202368964A294679
:10DC2000CDE9026205902A4609EB43037020019575
:10DC3000CDF810B00097F4F73DFD40F2FF202368C7
:10DC40008E4A0590CDE902620AEB43032A46CDE9EC
:10DC50000075CDF810B029467020F4F72BFD23682D
:10DC6000DDF8E8242B4493422360B8DBDDF86890AC
:10DC7000012240F2013100250420814BCDE904B19D
:10DC8000009003936D20CDE9012511460DF59D63AC
:10DC9000F4F710FDDDF8E804A84236DD149F56467F
:10DCA000DFF8F48103E0DDF8E804A8422DDD4FF44D
:10DCB000427337F9020BB6F900C0002200934146C7
:10DCC000C4E900506F4B4120C4F808C0F4F73AFD96
:10DCD00036F9023B0135002BE5D040F20A30002234
:10DCE00001214FF0040C684B05900393CDE901121C
:10DCF0004120CDF810B0CDF800C023460322F4F740
:10DD0000D9FCDDF8E804A842D1DC0F262027B2AB0D
:10DD10000C93DDF8D434169A0B93DDF8DC340592BD
:10DD2000159A0A93179B0492129A0993DDF8D83436
:10DD3000DDF828550392139A0893DDF8D034029247
:10DD4000119529AADDF8E05407930192189B149AC3
:10DD50001095DDF8E45406930092534694AA76A9F0
:10DD60000D96CDE90E75FDF7B9FB002540F2233085
:10DD700001233146454E3A4605900093CDF810B048
:10DD80000396CDE90155DDF8E4346C20F4F792FCFC
:10DD9000DDF8E824AA422CDD189BDDF8D0149F1E84
:10DDA000DDF8D434AA46A1F102085E1E01E0AA42C1
:10DDB0001FDD38F9023F37F9021F636016F8013F93
:10DDC0002560A1600135002BF1D040F229320121FC
:10DDD0000423CDE904B22E4ACDE90031CDE902A2F7
:10DDE000234603224120F4F765FCDDF8E824AA422B
:10DDF000DFDC1423189E179DDDF85880159FCDE9B0
:10DE00000053DDF8D024334641463846FDF7FAFC8E
:10DE10003146DDF8D434DDF8D0240A20FCF7A4FE26
:10DE20003146DDF8D434DDF8D0240A20FCF768FE52
:10DE3000DDF8D43432460093DDF8D014DDF8D83460
:10DE40000A20FCF7B9FEDDF8D4343246CDE90053A0
:10DE50004146DDF8D0343846FDF718FC0023179012
:10DE60000C49DDF8D054DDF8DC6424E07CCA010004
:10DE7000F0B90100DCB3010008BA010014BA0100D6
:10DE800020BA010054B901003CBA0100E8B9010010
:10DE90004CBA0100B02C00202CBA010035F9130057
:10DEA000A84F56F8232027F81300A74840F823204E
:10DEB00001330A2B0CD031F9022B002AEED1A148F4
:10DEC00020F81320A04840F8232001330A2BF2D178
:10DED000169F159D3946DDF8D4242846FFF7CEFA63
:10DEE000FEF7ECFD199B0026022B08BF40F0010055
:10DEF000C3B21D93AB1E1393BB1E1293DDF8D474F3
:10DF000024ABDFF84C82DFF84CA214931B94139AD5
:10DF1000129932F9023F1498139231F9022F239388
:10DF20001291397825930260C9F800203C460029F7
:10DF300049D06FF4E17541F69C00A3F1E10C2B444C
:10DF4000824D844515F806E041F2D86002D8E42AF3
:10DF500000F30C82834230D843F2D450A2F5E6732A
:10DF60009BB283428CBF00230123BEF1000F00F05F
:10DF7000118243B34FF00000744A5AF8263090558E
:10DF8000B200199233BB0F22704BC8F800209B5D82
:10DF9000002B00F087800A2325AAC8F800303046FD
:10DFA0004B46F9F709FF00BB39780246CDF80090DF
:10DFB00025AB3046F9F7F6FC17E0BEF1000F02D1B1
:10DFC0000123624A93555AF82630B20019920BB9D0
:10DFD0000029D8D1D8F800300E2B63DC4B4625AA97
:10DFE0003046F9F7E9FE0028DED0149D217823ABF6
:10DFF000009500223046F9F7D5FC1B9DDFF858C18B
:10E000002C46BCE80F000FC4BCE80F000FC4BCE8EE
:10E010000F000FC49CE80F0084E80F0058F8040BB1
:10E02000D9F8003055F82040259DC0F10F0103FBC1
:10E0300001F31A95239A149D02FB04F22D6805FB47
:10E0400004331A9D05FB0122214492FBF1F293FB5C
:10E05000F1F3139C17F8011B2280129A138041B32D
:10E06000179B022B00F34881384B9B5D002B40F03F
:10E0700077811D9B002B00F04C810E2840F33E81E0
:10E08000179B012B00F34981304B9B5DABB91D9B66
:10E090009BB958F8043C002BC4BF03F1FF3348F888
:10E0A000043C0AE04B4625AA00213046F9F784FEDD
:10E0B0009BE71D9B002B40F07181199A179B4AF832
:10E0C00002101BB948F8043C4AF80230002E00F058
:10E0D00011810225159B1B9C5F19169B5E19DDF8AB
:10E0E000D43403F1010837F9020F36F902CF18F8DA
:10E0F000011F4B4600940022C9F80000C4F800C07C
:10E100002846F9F74FFC0135D9F8002023680A2D7D
:10E110003A803380E7D1179B002B40F348810025DC
:10E120002822002148460BF0E8FEDDF8E8242560AF
:10E13000AA4252DDCDF848904FF4737A2B46DDF8B1
:10E14000DC9410E094280020A828002080280020DB
:10E15000D02800208828002020A101002368013356
:10E160009342236036DADDF8D414CB5C002BF5D073
:10E17000012600274FF00408CB4B32463146CDE94B
:10E180000273019623466D20CDE904BACDF80080D4
:10E19000F4F790FA40F2CD30236831460096C34E32
:10E1A0004246059009EB83036D20CDE90177CDF858
:10E1B00010B00396F4F77EFA2368DDF8E82459F8E6
:10E1C000231012980133934240F82510236005F183
:10E1D0000105C8DBDDF84890EDB24FF475730127F7
:10E1E00000269DF88020CDE904B3B14B9DF85C007A
:10E1F00003938DF895209DF87C309DF88420394656
:10E20000CDE9016600978DF894308DF8962025AB06
:10E2100004228DF897006D20F4F74CFA40F2D530C7
:10E22000A44A3946CDE901660097DDF80C35059022
:10E2300003926D209A22CDF810B0F4F73BFA40F229
:10E24000D73102229C4BCDE90176CDE904B1009291
:10E2500003932022DDF8E0340F216D20F4F72AFA31
:10E260004FF47672954BCDE90166009703930592C2
:10E27000DDF8E43420220F216D20CDF810B0F4F742
:10E2800019FA31463E220DF5CD700BF036FE2027EF
:10E2900042F20F0C8226DDF8E034214600932A4634
:10E2A0004B460320A4F800C0A7706671FBF7F6FF89
:10E2B0001C9B159C5A792046CDE90152169DDDF82C
:10E2C000D424DDF8D03400922946189AF8F7ACFE31
:10E2D000DDF8D42429462046FCF7CCF8DDF8D43408
:10E2E0002A4621460A20F8F713FE1E980DF2AC4D7F
:10E2F000BDE8F08F01260AE60E280EDC013048F852
:10E30000040C00293FF4D9AE179B012B7FF7BCAE5C
:10E3100003E0179B022B7FF4BCAE199B4AF8031055
:10E32000D4E60DF1E40AD0AD3C22214650461295C8
:10E330000BF0E3FD31AB2846782221461E461393AD
:10E340000BF0DBFD26AB1D4630461E2221461793FF
:10E350000BF0D3FD1E942C606C602C81FFF78BBA00
:10E360000E28CBDD179B022BD7D0A6E6834220D800
:10E3700043F2D450A2F5E6739BB283428CBF0023D4
:10E380000123BEF1000F7FF4F4AD43F68700824213
:10E390007FF719AE01224A488255EAE50E283FF779
:10E3A0008CAE013048F8040C0029ADD185E600257B
:10E3B0007EE7BEF1000F7FF406AE43F687039A4274
:10E3C0007FF701AE0123AB55FDE53E4B1A93524654
:10E3D0001499DDF8E804F9F753FC4FF028081B9076
:10E3E0004246002158A80BF088FD82220DF5AE7937
:10E3F000A9F80620A9F80A204FF00C02A9F80C2071
:10E400004FF00F0219214FF4FA73A9F810204FF0C2
:10E41000FA02A9F818104FF49671A9F81620A9F875
:10E420002230A9F82630642246230A270926A5258A
:10E43000E12410204FF4C87C4FF0370EA9F81A10D1
:10E440004FF03801C9E90B23199BA9F81C80022B56
:10E45000C9F80060A9F80E50A9F81240A9F81400F4
:10E46000A9F81EC0A9F820E0A9F82410A9F808709E
:10E47000C9E90D7728D066AC1B9B83B14846FCF7F1
:10E4800027FBFFF7A0BB48AA1492FFF7ECBA0023C2
:10E490001F93FFF717BA00232193FFF7A5BA1A9825
:10E4A000FCF716FBFFF78FBB64BA010068BA0100E6
:10E4B0007CBA010080BA010080B60100E8B9010011
:10E4C000802800207CCA01004246002167A80BF08A
:10E4D00014FD4FF00C0166AC21814FF00F01A181BA
:10E4E0004FF0FA01A4F81880E1824FF06408462149
:10E4F000C4E90B81072121604FF0140150232182D0
:10E500004FF49B72A0204FF032014FF0D20C4FF02D
:10E510001E0E26464D46C4E90D77E081A4F812C0D0
:10E52000A4F814E0A183E38063816283E2830FCEC9
:10E530000FC50FCE0FC50FCE0FC596E8070085E8B3
:10E54000070099E72DE9F04FC7B2C0F3072883B061
:10E55000474501900C992BDC9DF806A052000AF16A
:10E5600000499DF807B009F1FF390AFB023301EBBE
:10E57000490901EB4B0C0D9908F1010801EB470E1D
:10E58000DA4518D849461C460C4D34F9170031F9C4
:10E59000026F8542B8BF05468642B8BF08808C45E9
:10E5A0001444F2D12DB2013747452EF8025BE7D172
:10E5B00003B0BDE8F08F014DF5E700BF0080FFFF1D
:10E5C0002DE9F04F05468FB04FEA410A08AF1846D3
:10E5D0007A608846524600216C00BB60D7F84490B0
:10E5E0000BF08BFC2246386C00210BF086FC002DD2
:10E5F00064DD0AF108033E6C23F0070B4FEAA80321
:10E600003B617B683119F9609C1EC7F814D0ADEBF3
:10E610000B0D08ABA51C1846294652460BF062FCB0
:10E62000396902464046FEF79DFBB8F1000F0146EE
:10E6300050DD00202246034632F902CF8C4508BF48
:10E64000184601339845F7D10522ADEB0B0D152384
:10E6500040F23E6C4FF0290E07926FF42472009541
:10E6600008ADCDE901530692CDE903E3A1F11E0205
:10E67000CDF814C03C314346FEF75CFDBA68023D5C
:10E680000AEB040134F9023F35F9020F1B1AA3EB20
:10E690000903002B238006DD10889BB218441080EC
:10E6A0003088034433808C4202F10202EAD1FB68D5
:10E6B00002369E42D7F814D00C46A6D100237A68C1
:10E6C000C8EBC8084FEA48081C3722F80830BD4696
:10E6D000BDE8F08F6FF424724FF0050E152340F261
:10E6E0003E6C2920ADEB0B0DCDE9062E08AA039058
:10E6F000019204930293A1F11E0200953C31CDF8E2
:10E7000014C043460020FEF715FD04EB0A01CEE7D6
:10E710002DE9F04F9FB08A0008AF7A61083222F0ED
:10E720000702ADEB020DB8614E0008A8002979631D
:10E73000B860FE6119DD4FF4004E47F6FF7C0025FE
:10E74000B11ED7F884200144D7F88C00023A9619FC
:10E750000DF11E04023822F8025FB24221F802EFE6
:10E7600020F8025F24F802CFF5D1B969786B4A002E
:10E7700000FB02F2083222F00702ADEB020D08AAFC
:10E7800000297A6040F3E3807A6400223A6300EB68
:10E79000D07222F00102043B0A32D7F88010BB632A
:10E7A00022F007033B617B690439CB18F9603B65B4
:10E7B0003B69C7F82CD0ADEB030D08AAADEB030DF8
:10E7C00008ABBB647B6BFA64002B40F33981D7F84C
:10E7D00090200023013A144647F6FF797A6290466A
:10E7E000D7F88C209A46951E7A6CC7E90F33CB4632
:10E7F000FE68D7F838E0A2F1020C3C620BE0FC6C3A
:10E800004A4524F8130002DA01468146FB633A6D5B
:10E810000133964221D056F8040F5EF8042F35F8E4
:10E82000021FC2EBA0121144298018F8014F10B248
:10E83000E4072CF8020F4946C7F854B0DFD4BC6C8B
:10E840005A4524F81A0003DA83467865C7F840A0D1
:10E850003A6D0AF1010A9642DDD1C7F828A01525C4
:10E860004FF0000B05266FF4247840F23E694FF01C
:10E87000290AFA6C3C6A0092F86B6431CDE9066BA8
:10E880000395CDE9015A4FF00042CDE90498FEF717
:10E8900047FDCDE902A5CDE9066BCDE904980195C8
:10E8A000BE6C4FF000420096796DBB6A6431386CE3
:10E8B000FEF736FD796B7B6AFD6C0B4459461846B2
:10E8C0007B6C14F8012F0233D2074BBF35F81B20A5
:10E8D00036F811200BF1010B0131844223F8022C90
:10E8E000EFD17A6CF9693B6B0A447A647969BA6B47
:10E8F00001330A44BA63BA693B639A42D7F82CD011
:10E900007FF456AFD7E90C897A68FB69A2F1020C53
:10E91000BA6800269E4692469D1E1544B9F1000F26
:10E9200011DD29466046AAF1020230F9023F31F9B1
:10E93000024F9C42B8BF0B8032F9024F9C42C8BFC5
:10E940001380AA42F1D101364645F444E6D17B6BEF
:10E95000002B71DDBB68D7F888109C1E2646FA692B
:10E96000881ED7F88C10A2F1020CD7F81880023953
:10E9700003EB0C0500EB020E35F8023F36F8022FD0
:10E980009B1A20F8023F31F9023F704593FBF8F3E0
:10E990000B80F1D1D7F88430991E0A46BB6803EB8F
:10E9A0000C0534F9023F32F9020F002BB8BF5B426D
:10E9B000984200DA1380A542F3D1BB68084663444D
:10E9C0009C46FB690B441A463CF9023F30F9024F62
:10E9D000002BB8BF5B429C42B8BF03809042F3D18A
:10E9E0006FF00044D7F890302646581E7B6B0344E6
:10E9F0009C46034604E09442A8BF14469C450AD0B6
:10EA000013F8015F31F9022FED07F4D49642A8BF45
:10EA100016469C45F4D1D7F8842010F8015F118880
:10EA200015F0010FA1EB04050ABF891B15801180A9
:10EA3000834202F10202F0D15C37BD46BDE8F08F9F
:10EA40000024152505266FF4247840F23E694FF026
:10EA5000290AFB6C2046009307942346CDE90586DE
:10EA6000CDE90359CDE9015A4FF0004248F2630164
:10EA7000FEF756FCCDE90664CDE90498CDE902A580
:10EA80000195BB6C204600934FF00042234648F2AC
:10EA90006301FEF745FC24E7002824DDF0B40025DF
:10EAA0008E1EAC464FF0FF3700E01D4636F9024F90
:10EAB0006B1C944203DD6445C4BFA4462F469842B4
:10EAC000F3D17B1C11D07B0031F917001FB1CA189C
:10EAD00032F9022C1044AF4203DA1944B1F9023082
:10EAE0001844F0BC7047002070470020F0BC70470D
:10EAF00070B40024061E1C6020460EDD023901EBB6
:10EB0000460631F9024F944202DD1D6801351D6051
:10EB1000A042B8BF2046B142F3D170BC704700BFDD
:10EB20002DE9F04F82461646524600258BB000AFC5
:10EB30008846386D520000213C6E9946BB61C7F88B
:10EB400008A00BF0DAF90AEBDA7323F001030A33B9
:10EB500023F00703ADEB030DC7F820D0AA45ADEBBA
:10EB6000030D2561C7F81CD025606560A560E560D0
:10EB700084F811A0257440F3F980504647F6FF7ED3
:10EB80007A6DCC46013A7A609246321F02EB8003DE
:10EB90007B613B6DAB467146A8F10408A3F1020905
:10EBA0007D623C6611E07345A8BF7346D7E908450E
:10EBB00024F81500A8BF18467C6A86467869013497
:10EBC00090427C620CF1010C31D0B86952F8043FDC
:10EBD00020B19CF8000000FB0333DB1158F8040F50
:10EBE000BD6DC3EBA01347F6FF708342A8BF034679
:10EBF00061480E468342B8BF034618B229F8020F97
:10EC00001AF8014F2C57002CCDD18B42A8BF0B46D0
:10EC1000FC691E4624F81B00A8BF18460146786907
:10EC2000734690420BF1010B0CF1010CCDD1D7E9E9
:10EC300018429342A8BF13469642A8BF16461BB27D
:10EC4000524236B29342B8BF13469642B8BF1646F8
:10EC500032464FF0000C4FF00040FE60FE6D7968C8
:10EC6000D6E900E9BE683B610E44B346B7F91060CF
:10EC700012B27E61E0464E4663466FF00045BA61CF
:10EC80007862D7F8509041E03A6A786932F91820F2
:10EC9000002A5ADB002802DB3869121A12B229F85E
:10ECA000132008F10108724518DDB4F808A02268A5
:10ECB0000AF1010AA4F808A039F913A094F9110087
:10ECC000AAEB0E0A5244226094F910209842C8BF61
:10ECD00063749A42B8BF237439F9132096420ADD4F
:10ECE000628960680132628139F91320A2EB060A59
:10ECF0008244C4F804A0786A01339042B8BF104639
:10ED00009542A8BF15468B45786227D011F8012F90
:10ED1000B86D8256002AB7D1FA69B86932F91C2059
:10ED2000002A09DB002802DBF868121A12B229F85F
:10ED300013200CF1010CB6E70028F5DA121A02EAEA
:10ED4000E27212B229F81320F3E70028A4DA121AAB
:10ED500002EAE27212B229F81320A2E72DB203B23E
:10ED60002C37A381E581BD46BDE8F08F2B464FF0DF
:10ED700000404FF0FF35F3E70080FFFF2DE9F0473B
:10ED800086B08246DDE9129816461C460D46149F51
:10ED9000F3F756F91423159A0397CDE90423D0F815
:10EDA00001300F98153332462946CDE9010300940E
:10EDB0000E9B5046FFF7B4FE00254FF02E0C0121AC
:10EDC00002271848184E2346CDE90306524669200B
:10EDD000CDF814C0CDE901150097F3F76BFCAA45F7
:10EDE00028460FDDA31E03EB4A0A33F9021FA1EBED
:10EDF0000902002AC8BFAD18B1EB080148BF40188E
:10EE00005345F2D1109BAB4207DB119B8342D4BF29
:10EE10000020012006B0BDE8F087012006B0BDE863
:10EE2000F08700BF80B6010098BA0100002820DDFD
:10EE3000F0B48E1E06EB4006B14218D0571C38467F
:10EE40000B46B1F9004033F9025FAC4207DD0D809B
:10EE50001C8092F9004090F9005015700470B34284
:10EE600000F10100EDD10231B1423A46E6D1F0BCE9
:10EE7000704770472DE9F04F8046450005F10804C2
:10EE800085B000EBD07A24F0070407302AF0010A9D
:10EE900000AF20F00700ADEB040D08F1090424F0E9
:10EEA0000704EB46ADEB000D0AF10A0020F0070065
:10EEB0006E46ADEB040D6C46ADEB000DE946C7E9BF
:10EEC00002210AF1020A08F102021F2120467B609A
:10EED0000BF013F85246484600210BF00EF8B8F13B
:10EEE000000F7B6807DD324606EB0800911B02F835
:10EEF000011B8242FAD14FF0FF3A2A46F968584680
:10EF00007B600AF0EFFF594632464046FFF78EFF1E
:10EF1000023D08F1FF3E7B6806EB0E01AB44013E6B
:10EF2000B14218D03BF9025911F901299D4202F171
:10EF3000010C10DBA05C22441F28927860D01E28B0
:10EF400060D81E2A96BF4FF0FF3204F80C0004F878
:10EF50000C20B142E6D1B8F1020F04F1010113DD3A
:10EF60000B46FF20A64402E0013373450CD05A78CB
:10EF70001F2AF9D11A781E2AF6D89A7801331E2A48
:10EF800098BF18707345F2D1B8F1000F2EDDFB6801
:10EF900004EB0806F96004E00134A64203F1020321
:10EFA00023D06278FF2AF7D1257894F802C039F887
:10EFB000150039F81CE08346704528BFF346B3F9C5
:10EFC0000020B96B0A449345E6DA704538BF7046B5
:10EFD000013465458CBF29F81C0029F81500A642AC
:10EFE0000AF1FF3A03F10203DBD1F9684246B8683F
:10EFF0000AF078FF0AF101001437BD46BDE8F08F32
:10F000001F2A06D01E2A88BF6FF0690204F80C2060
:10F0100086E70AF1010A04F80CA029F81A507FE7E4
:10F02000FFF728BF0048704798080020014B036095
:10F0300020207047B8BA0100014B03600F207047D1
:10F04000D8BA0100014B03600F207047A8BA010035
:10F0500030B44FF0804300220E211F2020250F24C2
:10F0600083F8082183F80A2183F8090183F80B113A
:10F070001A739A735873D9731D725C72DA7793F8A6
:10F08000211041F0010183F8211093F8211062F35F
:10F09000410183F8211030BC704700BF10B44FF01D
:10F0A000804485B00DF1100C0CE90F00BDF8003064
:10F0B0002382BDF802306382BDF90430A382BDF91A
:10F0C0000630E382BDF808302383BDF80A3063833D
:10F0D000BDF80C30A38305B010BC70474FF08043DF
:10F0E000988370474FF08043988B70474FF0804370
:10F0F00083F82000704700BF0123002110B50A4AA1
:10F100000A4C2377917210B94FF08042D3704FF0C0
:10F1100080430122987000211A700A2000F094F9AF
:10F120000022024B1A7710BDD82800200000105092
:10F1300001234FF08040102110B4034A034CA37206
:10F14000436010BC11607047A40C0020D828002038
:10F1500001234FF08040102110B4044A044C637224
:10F16000C0F8043110BC1160704700BFA40C00202F
:10F17000D8280020E022002101480AF0BEBE00BFCE
:10F18000800100402DE9F04105461F4B1F4886B025
:10F190006A1E13F8011B834202F8011FF9D10124F2
:10F1A0002B464FF0A90C002702262868184AC117E1
:10F1B00082FB00E2DFF8648002441648C1EB2222A1
:10F1C00043F8242B2146CDF814C02246CDE903088C
:10F1D000CDE9014700966220F3F76CFA4FF0AA0CD4
:10F1E0000D48CDF810800390CDE90147009605F158
:10F1F000260322462146CDF814C06220F3F75AFABE
:10F2000006B0BDE8F08100BF280000405400004077
:10F210008988888848E10100ECBA0100E8BA010059
:10F2200070B5E022064600210B480AF066FE002475
:10F2300001234FF08042094D09492B770A208C7237
:10F2400093702146137000F0FFF82C773046BDE82C
:10F250007040FFF797BF00BF8001004000001050D2
:10F26000D828002010B50446FFF78CFF2E234FF05E
:10F27000804004F14E0203F1600150F82110013B7F
:10F280001F2B22F8021DF6D14FF0804004F19602A8
:10F2900003F1600150F82110013B22F8021D591CB6
:10F2A000F6D110BD4FF0804270B5037909B201FB71
:10F2B00003F1948B8B11A342B8BF23460125002490
:10F2C000022106889BB24380A2F80C61A2F80E319D
:10F2D000074E084B357709205C7282F8035182F89B
:10F2E00002112146A2F8005100F0AEF8347770BD4B
:10F2F00000001050D82800204FF0804393F81401EC
:10F30000704700BF4FF0804393F81701704700BF6C
:10F310000023094A82F832305064916472B60123A6
:10F3200082F8403000BFB2F852309BB2002BFAD0C6
:10F3300062B6B2F850007047000010502DE9F04757
:10F3400050221020202130244FF0400A4FF0600955
:10F350004FF001084FF4807E4FF4007C4FF480673B
:10F360004FF400660825104B83F8000383F804135C
:10F3700083F8084383F8034383F805A383F809233C
:10F3800083F80A2383F80B2383F80F93C3F80080D4
:10F3900018601960C3F800E0C3F800C01F601E6069
:10F3A0001D60BDE8F08700BF00E100E04FF40042BF
:10F3B000034BC3F88020BFF34F8FBFF36F8F7047AD
:10F3C00000E100E000220121034BA3F86E20A3F826
:10F3D0006A20A3F8681070470000105010B5174C51
:10F3E00084B094E80300029002A88DF80C1000F09D
:10F3F00061F800F069F8FFF7A1FF62B600F014FAB7
:10F40000A36804A840F80C3D00F008FA00F050FA98
:10F4100000F05EF900F0C0FA094B1A6922F004020C
:10F420001A61BFF34F8F0721064A82F824105A69E8
:10F4300042F010025A6104B010BD00BF60A101008B
:10F4400000ED00E00000105008B500BF72B6084A99
:10F45000135C3BB900BF30BF62B600BF72B6135C2D
:10F46000002BF7D00023135401B1884762B608BDC2
:10F47000D828002000200A4B0A4913F8012B104419
:10F480008B42C0B2F9D1064B1A78AA2A01D00020CB
:10F490007047DB7B181AB0FA80F04009704700BF54
:10F4A000800040008F0040004FF0A04301225A74BA
:10F4B000704700BF0246034B0068127918601A714A
:10F4C000704700BFE828002070B5FFF7D3FF012286
:10F4D0000021334BD9705A72DA7200285CD0314A5D
:10F4E000D278D2B21A72002201242F492C4B8D7887
:10F4F0009A725A731D734D780E781E751D77CD78EC
:10F50000097983F8215083F820105A749A741C7476
:10F510009A7018B3234A51781A78C9B2D2B28A4283
:10F5200008D08A42B4BF013202F1FF32D0B28A421F
:10F530001870F6D11B4B1A491A794B78D2B2DBB24C
:10F540009A420AD09A4203F1010096BF03F1FF33B9
:10F55000C3B2DBB29A424B70F4D170BD1A78D2B20A
:10F56000B02A08D0AF2AD4BF013202F1FF32D1B2A3
:10F57000B02A1970F6D10A4A5378DBB2082BECD0C6
:10F58000072B03F101018ABF03F1FF33CBB2DBB2DA
:10F59000082B5370F4D1E0E7E0221A72A3E700BF12
:10F5A0000000105080004000E828002007490B7838
:10F5B000DBB2834208D09842CCBF013303F1FF3362
:10F5C000DAB283420A70F6D1704700BF00001050D3
:10F5D00008B5FFF74FFF18B1024B5878C0B208BD0D
:10F5E000B02008BD80004000014B1878704700BF74
:10F5F00000001050084A5378DBB283420AD0984288
:10F6000003F1010196BF03F1FF33CBB2DBB28342BA
:10F610005370F4D1704700BF00001050014B587870
:10F62000704700BF0000105010B50446FFF73CFFC4
:10F630004FF0A04320686168A26807C310BD00BFF7
:10F6400038B54FF0A044E37DDBB2042B28D0082B63
:10F6500019D0022B09D00123184A137000BF4FF0B4
:10F66000A042137300BF537338BD154D154960791F
:10F67000FAF71AFB61792868FAF75EFB62792B6862
:10F6800013442B60E7E7104BD0E9051259609A60EC
:10F69000236A5BBA0A4A18461360FAF7CFFADAE728
:10F6A000074D0A492079FAF7DDFA21792868FAF737
:10F6B00017FB22792B6813442B60CCE7D828002055
:10F6C000F028002020000050842100202400005059
:10F6D000274B0022D3F8801041F00101C3F88010BD
:10F6E000196C21F001011964196841F001011960D8
:10F6F000D3F8801021F00201C3F88010196C21F0BA
:10F7000002011964196841F002011960D3F88010F0
:10F7100041F01001C3F88010196C41F01001196418
:10F72000196841F010011960D3F8801021F0200110
:10F73000C3F88010196C21F020011964196841F098
:10F7400020011960D3F8801021F04001C3F8801027
:10F75000196C21F040011964196841F040011960E9
:10F76000C3F80821C3F80421C3F80021704700BF83
:10F7700000000250034BD3F8C03018420CBF0120E8
:10F78000002070470000025038B54FF0405401256A
:10F79000642084F8245000F0D1F900F07FF90023B0
:10F7A0004FF47A7084F8253084F8815000F0C6F95F
:10F7B000BDE8384000F072B910B501234FF0405455
:10F7C000642084F8253000F0B9F900F067F90023CF
:10F7D00084F8243084F8813010BD00BF1420012249
:10F7E000002130B50A4D89B02D780A4C05900A48A1
:10F7F00008AB03F8015DCDE90111CDE903040092E6
:10F8000011466420F2F756FF9DF81F0009B030BD85
:10F81000B700400000BB010008BB01000268014BBB
:10F820001A607047F428002038B5FFF723FE0F2335
:10F83000F0B94FF040524FF00104D9B2013B072B11
:10F8400082F82B1082F8284082F82800F5D1042392
:10F8500082F82F304FF040530121002283F8281006
:10F8600083F828204FF47A70BDE8384000F0F6B9EC
:10F870004FF04051012500240C4806E081F82B2070
:10F88000013B81F8285081F82840027A0E2A8EBF69
:10F890000F22027AD2B29342DAB2EFDA4FF040523C
:10F8A000024B5B7ADBB282F82F30D3E78000400056
:10F8B000F8B5FFF7DFFD4FF040540125002607465D
:10F8C00084F825604FF47A7084F8205084F827502B
:10F8D00000F0C4F9642084F8255000F0BFF984F8E2
:10F8E0002450642000F0BAF984F8256007BB062391
:10F8F0001C4D84F82730EB7884F826302B7884F878
:10F9000042304FF0405401230022697840F24C40CD
:10F9100084F8461084F8442084F8453084F8413057
:10F9200084F8403000F09AF9AB7884F84430F8BDA0
:10F93000FFF754FF0C4B9B7A88B94FF04052DBB273
:10F94000084D84F82730E978074B82F82610DB7AD7
:10F9500029780B440B3BDBB282F84230D1E7053B00
:10F96000EBE700BFF42800208000400020B9064AE1
:10F97000064B10601860704703490548034B054A61
:10F9800008601A60704700BFFC280020F82800209B
:10F9900089F70000B9F700004FF04053F0B4062497
:10F9A000012200250A26FF2083F8D64093F8D710BD
:10F9B0000F2764F3030183F8D710042183F8D8607C
:10F9C00083F8402183F8D00083F87F5093F88C00AF
:10F9D0004FF0050C104383F88C0093F88C00072639
:10F9E00040F0020083F88C0093F8910064F3030068
:10F9F000032483F8910083F8901083F88D1083F826
:10FA0000A02093F8A10065F3010083F8A10083F81A
:10FA1000947093F88800104383F8880093F8890065
:10FA2000104383F8890083F8F12083F8874083F836
:10FA30008E4083F8D22083F8D52083F8ABC083F8BA
:10FA4000AD5083F8AC4083F8AE1083F8AF1093F854
:10FA50008B1041F0700183F88B1083F8936083F86A
:10FA6000B020F0BC704700BF00220521034B0448C2
:10FA70001A6058609A601960704700BF10E000E09B
:10FA8000FFFF0F000022044B98681A60C0F57F202A
:10FA900000F6FF70704700BF10E000E0002382B066
:10FAA00000280193B8BF0730019BC010984206DDC3
:10FAB00000BF019B01330193019B8342F8DB02B03D
:10FAC000704700BF054A0649937CD27801335B003A
:10FAD000934000FB03F091FBF0F0704700001050E2
:10FAE00000B4C404054A937AD27ADBB20AB1013376
:10FAF0009840034B93FBF0F0704700BF000010509C
:10FB000040420F00054A937AD27ADBB22AB1012231
:10FB1000134402FA03F390FBF3F070470000105017
:10FB2000054A00EB8000937CD27801335B00934060
:10FB3000000190FBF3F0704700001050124B00EBF7
:10FB400080001B7B0001DBB25A1E062A0DD9082B50
:10FB500012D0092B15D0A3F10B02032A0ED90F2BBB
:10FB60000CBF01234FF0FF3300E00133064AD27887
:10FB7000934090FBF3F070470A23F7E7063B9B00A6
:10FB8000F4E70C23F2E700BF00001050034B044AD7
:10FB90005B7C03F0010352F823301847000010503B
:10FBA00014BB0100034B044A5B7C03F0010352F8D1
:10FBB00023301847000010500CBB010008B5044B5F
:10FBC0001868FFF7EFFFBDE8084000F0A1B800BFDC
:10FBD0000429002038B50C4B054693FBF1F00C4688
:10FBE000FFF7ACFF3A2303FB04F39B1103FB00F088
:10FBF00090FBF5F0834203DB462404FB00F4A411E0
:10FC0000024B1C6038BD00BF40420F000429002099
:10FC100070B5012200244521042688B008AB43F8C2
:10FC2000040D0B4D0B48CDE901240591CDE90305E9
:10FC3000114600966420F2F73DFD074B07985C7172
:10FC400000F042F821460520FFF7FEFB08B070BD2A
:10FC50001CBB010024BB0100D828002008B5FFF719
:10FC600095FFBDE80840FFF7D3BF00BF08B5044BC0
:10FC70001860FFF797FFBDE8084000F00DB800BF1F
:10FC800004290020002000F049B800BF012000F046
:10FC900045B800BF00F030B8012830B44FF0000282
:10FCA0004FF0020438BF01200121054B054D1A70A9
:10FCB0002A719C709860DA605A70197030BC704775
:10FCC00000000850D828002001284FF000024FF013
:10FCD000010138BF012010B4054B064C1A70627147
:10FCE00099709860DA605A70197010BC704700BF44
:10FCF00000000950D8280020012000220249034BAF
:10FD000008711A70704700BFD82800200000085002
:10FD1000014B9860704700BF0000085010B40B4AB8
:10FD20000B4983B0CDE9001202AB03EB800353F81B
:10FD3000082C9378DBB2012B04D10021054C043050
:10FD40002354117003B010BC704700BF000009506D
:10FD500000000850D8280020034AD2F8803023F051
:10FD60000103C2F88030704700000250034AD2F805
:10FD7000803043F00103C2F8803070470000025029
:10FD8000034BD3F88000C04300F00100704700BF70
:10FD900000000250002822DDF0B5DCF804600024E9
:10FDA00096F80EE00CE0DCF800703F5D07FB0333D3
:10FDB00005FB03F35B1242F824300134A0420DD05E
:10FDC00051F8043B356ABEF1000FECD103FB05F39B
:10FDD0009B1042F824300134A042F1D1F0BD7047AD
:10FDE000002822DDF0B5DCF80460002496F80EE06F
:10FDF0000CE0DCF800703F5D07FB033305FB03F309
:10FE00005B1242F824300134A0420DD051F8043B7B
:10FE1000356ABEF1000FECD103FB05F39B1042F8ED
:10FE200024300134A042F1D1F0BD7047002822DD1A
:10FE3000F0B5DCF80460002496F80EE00CE0DCF885
:10FE400000703F5D07FB033305FB03F35B1242F8D1
:10FE500024300134A0420DD051F8043B356ABEF184
:10FE6000000FECD103FB05F39B1042F82430013462
:10FE7000A042F1D1F0BD7047002822DDF0B5DCF8DA
:10FE80000460002496F80EE00CE0DCF800703F5DA2
:10FE900007FB033305FB03F35B1242F82430013404
:10FEA000A0420DD051F8043B356ABEF1000FECD1F1
:10FEB00003FB05F39B1042F824300134A042F1D13A
:10FEC000F0BD7047DCF80830F0B49C7BBCB900286A
:10FED00013DDDCF80430D3F80D301B681E89DD8893
:10FEE00051F8043B013403FB06F393FBF5F3A04206
:10FEF0004FEA831342F8043BF2D1F0BC704700286C
:10FF0000FBDDDCE90043D3F80D30013C1B682044E5
:10FF10001F89DE8814F8015F51F8043BA04205FBFD
:10FF2000033307FB03F393FBF6F34FEA630342F853
:10FF3000043BEFD1F0BC7047704700BF00280BDDD9
:10FF400010B4002451F8043B01349B01A04242F854
:10FF5000043BF7D110BC7047704700BF00232DE968
:10FF6000F041DCF80C5088B00793D5F80920002840
:10FF7000644617680EDDDCF80820D2681618013ECA
:10FF8000013A12F8011F795C96420B440793F8D1AD
:10FF900093FBF0F3606807934288002A53D00689E8
:10FFA000921B11029B1B91FBF3F3B3F5DC7FA8BFFF
:10FFB0004FF4DC730362D5F80D504FF0020E29891F
:10FFC000002603FB01F31912FF29A8BFFF2101221C
:10FFD0004FF0AB081E4FDFF884C0698100EB0E03C1
:10FFE000CDF800E0CDE903C71146CDF81480CDE986
:10FFF00001666420F2F75EFB01254FF00408AC2295
:020000021000EC
:10000000144B059229462A460393049707AB0296A0
:100010000195CDF800806420F2F74CFB4FF0AD0C59
:1000200063680D4804970390CDE90156CDF8008030
:1000300020332A462946CDF814C06420F2F73AFB53
:1000400008B0BDE8F0814FF480730362B3E700BFEE
:1000500028BB010050BB010058BB010034BB0100AC
:1000600000232DE9F041DCF80C5088B00793D5F857
:1000700009200028644617680EDDDCF80820D268E5
:100080001618013E013A12F8011F795C96420B44A2
:100090000793F8D193FBF0F360680793C288002AB6
:1000A00052D08688921B11029B1B91FBF3F3B3F590
:1000B000DC7FA8BF4FF4DC730362D5F80D504FF01E
:1000C000020E2989002603FB01F31912FF29A8BF9C
:1000D000FF2101224FF0F4081D4FDFF880C0698135
:1000E000831DCDF800E0CDE903C71146CDF814809B
:1000F000CDE901666420F2F7DDFA01254FF004082E
:10010000F522144B059229462A460393049707AB20
:1001100002960195CDF800806420F2F7CBFA4FF0FB
:10012000F60C63680C4804970390CDE90156CDF8AE
:10013000008020332A462946CDF814C06420F2F707
:10014000B9FA08B0BDE8F0814FF480730362B4E7F8
:1001500028BB010050BB010058BB010064BB01007B
:1001600000232DE9F041DCF80C5088B00793D5F856
:1001700009200028644617680EDDDCF80820D268E4
:100180001618013E013A12F8011F795C96420B44A1
:100190000793F8D193FBF0F3606807934288002A35
:1001A00054D00689921B11029B1B91FBF3F3B3F50C
:1001B000DC7FA8BF4FF4DC730362D5F80D504FF01D
:1001C000020E2989002603FB01F31912FF29A8BF9B
:1001D000FF2101224FF4C5781E4FDFF884C06981EA
:1001E00000EB0E03CDF800E0CDE903C71146CDF8D2
:1001F0001480CDE901666420F2F75CFA01254FF026
:10020000040840F28B12144B059229462A460393A8
:10021000049707AB02960195CDF800806420F2F7B1
:1002200049FA4FF4C67C63680C4804970390CDE903
:100230000156CDF8008020332A462946CDF814C057
:100240006420F2F737FA08B0BDE8F0814FF480730C
:100250000362B2E728BB010050BB010058BB01009C
:1002600034BB010000232DE9F041DCF80C5088B0CC
:100270000793D5F809200028644617680EDDDCF8DE
:100280000820D2681618013E013A12F8011F795C65
:1002900096420B440793F8D193FBF0F36068079301
:1002A000C288002A53D08688921B11029B1B91FBA7
:1002B000F3F3B3F5DC7FA8BF4FF4DC730362D5F82A
:1002C0000D504FF0020E2989002603FB01F319128D
:1002D000FF29A8BFFF21012240F2D3181E4FDFF8EB
:1002E00084C06981831DCDF800E0CDE903C71146C4
:1002F000CDF81480CDE901666420F2F7DBF9012521
:100300004FF004084FF4EA72144B059229462A462E
:100310000393049707AB02960195CDF80080642003
:10032000F2F7C8F940F2D51C63680D4804970390B2
:10033000CDE90156CDF8008020332A462946CDF874
:1003400014C06420F2F7B6F908B0BDE8F0814FF4AC
:1003500080730362B3E700BF28BB010050BB0100FC
:1003600058BB010064BB010000232DE9F0411C468D
:10037000DCF80C2088B0D2F809206646D76801F571
:10038000F06501F5006C0793043F57F8041FA5F5CD
:10039000F062890952F8803B5B1A95421C44F9D1FE
:1003A0000435AC450794F0D194FBF0F4B36807949E
:1003B0005A88002A54D09988521A1202641A92FB61
:1003C000F4F4B4F5DC7FA8BF4FF4DC741C627268EF
:1003D00040F23A2ED2F80D204FF0020C10680025A2
:1003E000C188012204FB01F42112FF29A8BFFF21CB
:1003F0001D4F1E4C01816344CDF814E0CDF800C0C0
:100400001146CDE90347CDE901556420F2F752F9D1
:1004100001244FF0040840F23B22154B059221467F
:1004200022460393049707AB02950194CDF8008010
:100430006420F2F73FF94FF40F7CB3680D4804973E
:100440000390CDE90145CDF80080203322462146B6
:10045000CDF814C06420F2F72DF908B0BDE8F081A2
:100460004FF480741C62B2E728BB010080BB01001E
:10047000A4BB0100B0BB010030B595B02022002123
:100480000CA809F03AFD294C29492A4D2A48CDE902
:100490000854CDE90A01294A294B0E9293F881208C
:1004A00002AC8DF83C2093F881308DF83D30F6F7A2
:1004B00005F98DF83E00F6F707F98DF83F00F6F7DD
:1004C00009F98DF84000F6F70BF98DF84100F6F7C1
:1004D0000DF98DF84200F6F70FF91190F6F712F9C1
:1004E0001290F6F715F9ADF84C0008A8F9F7A0FA44
:1004F000F6F70EF9F9F724FF0023022202930120F8
:10050000A382C4E90133C4E903338DF81D20FBF74E
:10051000D3FC06ABADF81E0093E803008DE80300A2
:1005200094E80F00F9F72EFA15B030BD6DFD00000C
:100530005DFC000059FD000081FD00006E00167892
:100540000000105070B5002301223F2148260825E5
:10055000022484B001A8CDE9013303938DF807602C
:100560008DF808508DF809208DF80F208DF80A407D
:100570008DF80D10FFF758F804B070BD02FB01F2C2
:100580001212FF2AA8BFFF22028070472DE9F04215
:10059000224E92B0224D0DAC05AF994606910892BD
:1005A00096E80F0084E80F0018ABC4E902752046F6
:1005B00011A91193EFF764FE96E80F00194E09ADEB
:1005C00085E80F00C5E9027621462846EFF758FE78
:1005D000089B069A44F001041169D3F801200591A3
:1005E0000792D3F80D2010491089189E5081CDE94B
:1005F000021445F0010501960495D3F809308022D4
:100600005B690021184609F078FC2022034601A905
:100610004846F6F783F812B0BDE8F0826CA10100FD
:100620005DFF000095FD0000DD5900002DE9F0425E
:10063000224E92B0224D0DAC05AF9946069108921C
:1006400096E80F0084E80F0018ABC4E90275204655
:1006500011A91193EFF714FE96E80F00194E09AD9A
:1006600085E80F00C5E9027621462846EFF708FE27
:10067000089B069A44F001041169D3F80120059102
:100680000792D3F80D2010491089189E5081CDE9AA
:10069000021445F0010501960495D3F809303C2277
:1006A0005B690021184609F028FC0F22034601A9C6
:1006B0004846F6F733F812B0BDE8F0826CA10100AD
:1006C00061000100E1FD0000415A00002DE9F04207
:1006D000224E92B0224D0DAC05AF9946069108927C
:1006E00096E80F0084E80F0018ABC4E902752046B5
:1006F00011A91193EFF7C4FD96E80F00194E09AD4B
:1007000085E80F00C5E9027621462846EFF7B8FDD7
:10071000089B069A44F001041169D3F80120059161
:100720000792D3F80D2010491089189E5081CDE909
:10073000021445F0010501960495D3F80930802292
:100740005B690021184609F0D8FB2022034601A965
:100750004846F5F7E3FF12B0BDE8F0826CA1010056
:10076000610101002DFE0000F55900002DE9F04265
:10077000224E92B0224D0DAC05AF994606910892DB
:1007800096E80F0084E80F0018ABC4E90275204614
:1007900011A91193EFF774FD96E80F00194E09ADFA
:1007A00085E80F00C5E9027621462846EFF768FD87
:1007B000089B069A44F001041169D3F801200591C1
:1007C0000792D3F80D2010491089189E5081CDE969
:1007D000021445F0010501960495D3F809303C2236
:1007E0005B690021184609F088FB0F22034601A926
:1007F0004846F5F793FF12B0BDE8F0826CA1010006
:100800006502010079FE00009D5A00000269054B57
:100810000548013A12F8011F013303F8011C834215
:10082000F8D1704700008360E00183602DE9F0415A
:10083000234E92B0234D0DAC05AF9846CDE906107E
:10084000089296E80F0084E80F0018ABC4E902751F
:10085000204611A91193EFF713FD96E80F001A4EE9
:1008600009AD85E80F00C5E9027621462846EFF775
:1008700007FD069B4FF4F062D3F8093000211B6995
:10088000124F184609F039FBDDE906210969104EBF
:100890000591D2F80D200346126844F00104D18876
:1008A00045F00105118140464FF4F07201A9CDE9F0
:1008B0000345CDE90176F5F731FF12B0BDE8F081CF
:1008C0006CA1010069030100C5FE0000994200000F
:1008D000453C000030B4D0F80D30D0F809001B685A
:1008E000C068DC8801F1800504FB02F21212FF2AC5
:1008F000A8BFFF221A8192B251F8043B03FB02F316
:1009000093FBF4F38D4240F8043BF5D130BC7047C3
:10091000F0B50F46D0F80D30D0F809201B68D46828
:10092000DA8885B01A81F3F7B7FCF3F781F920462E
:100930008022002109F0E1FA074A0849084E094DD2
:10094000009201912346384620226946CDE902658E
:10095000F5F7E4FE05B0F0BD99420000313C00001F
:1009600039FF00003DFF0000002825DD2DE9F003E0
:100970009046043982B04FEAE27901EB800051F8E9
:10098000042FD317CDE90023DDE9002302FB09FC86
:10099000A2FB086708FB03C3B40B1F4444EA874467
:1009A000BD13CDE90045DDE9002388420A60E6D1A8
:1009B00002B0BDE8F0037047704700BFF0B50026F5
:1009C00085B0FFF759FDF5F7B5FA1E491E4F3346BE
:1009D00032460C68022001210096A0473C46FFF7F2
:1009E000B1FDFEF71FFBF3F769F9FEF7F7FCFEF721
:1009F0002FFB164B164DA3F868600FCD0FC40FCD1B
:100A00000FC40FCD0FC43B682A680133226006D0A3
:100A1000082304A800F8043D0121F9F7B7FA0122E0
:100A20000A4B0C4CA3F86820F9F77CFA00F06CFB39
:100A30002568FEF7D9FDA8702468FEF7EFFDE07089
:100A400005B0F0BD60E201009021002000001050D0
:100A500000FE0100340A00200246034B5168006882
:100A6000926807C3704700BF082900202DE9F04FA6
:100A7000964683B0544E9DF834709DF830C0984629
:100A8000009763460D46B6F90620B6F904100446F1
:100A900070469DF83870FAF789FF3378800290FB32
:100AA000F8F0002B4BD0A91C96F801904B002A4679
:100AB00004EB030E03F10208B9F1000F50D13EF828
:100AC000069C05F1FF3C24F80890A3F108053EF8C8
:100AD000043C254424F811306189238961802380F6
:100AE000531ED2B31A4602F1010B4FEA4B0104EB3D
:100AF000010A063134F801903AF8028C34F81B30C0
:100B0000C84407FB08F9BAF8048096F903B04344D7
:100B10000BFB0398BAF8023096F90290624509FB84
:100B200003834FEAA31300FB03F34FEA234363520B
:100B300046D0012AD4D1E38800226380D3E765B18F
:100B4000A91C04EB4101043431F8022D00FB02F230
:100B50008C424FEA22428A80F6D103B0BDE8F08F82
:100B600000236380238024F8113024F80830002DFE
:100B7000F3D07F0004EB450131F802E996F9035008
:100B8000B1F808C00B88CA889C4538BF9C4696457A
:100B900038BF96460CFB07F36A000EFB02338D88C4
:100BA00096F902208C4205FB02324FEAA21200FBAA
:100BB00002F24FEA22420A81DED103B0BDE8F08F93
:100BC0002B88AEF800308BE708290020F0B50546E9
:100BD0002C4C426994F9033094F90270C3F120035C
:100BE000E07AC7EB4307A37A85B0C7F34707CDE99F
:100BF0000107009305F12C0020230E460F21FFF77B
:100C000035FF617A237A05F152046A692046CDE9FD
:100C10000117009320210F23FFF728FFFEF7AAFA00
:100C200020462E234FF0804403F1600230F8021D6D
:100C3000013B1F2B44F82210F6D14FF0804405F100
:100C40009A0232F8020D03F16001013B44F82100E1
:100C5000591CF6D10120FEF74FFA2846FEF792FA0A
:100C6000B4F84C301BB2336094F85030337294F8BF
:100C70005130737294F85230B37294F85330F37267
:100C800005B0F0BD0829002038B504220125144B19
:100C9000144C1D712260FEF7F5FFFEF78FFFF9F788
:100CA00041F9837E43B9104B1B682BB10F4A126880
:100CB00012B90F4A157098470E4BD3F8002112074E
:100CC00008D5002208250C480C49C3F88051027051
:100CD000C1F8402101211023094AD160236038BDA9
:100CE000D8280020A40C0020981700208C1C00207D
:100CF0009717002000E100E0A00C00200000025047
:100D0000000008500122052138B50D4B0D4C5A71D9
:100D10002160FEF7BBFF0C4BD3F80021120708D56A
:100D20000022082509480A49C3F880510270C1F819
:100D3000402101211023074AD160236038BD00BF44
:100D4000D8280020A40C002000E100E0A00C002026
:100D500000000250000009500121032238B50B4B5E
:100D60000B4DD9700B4C2B7822601BB1FEF78AFE1D
:100D7000094B186001232B70FEF776FE002110232B
:100D8000064AC2F84011236038BD00BFD8280020B1
:100D9000A00C0020A40C002000290020000002501C
:100DA00001234FF06050102110B4034A034CE3724A
:100DB000836210BC11607047A40C0020D82800206A
:100DC0000F21124A124B11605B6F84B00193019B9B
:100DD00023F4FF6323F007030293019B23F07F03B7
:100DE0000393029BB3F5800F0AD0039A094B9A42F2
:100DF00006D0019A084B9A4202D20122074B1A7080
:100E00000122034BA3F86C2004B07047A40C00200F
:100E10000000105080FF010000FC01001429002098
:100E200008B5FFF7CBFD00F0D5FD002008BD00BFE1
:100E3000704700BF08B54FF0CD3203490348FCF7B7
:100E4000A7FA002008BD00BFAC440020AC3400204D
:100E5000704700BF08B5F1F707F8D0F80930986877
:100E600008BD00BF40F215132DE9F0431C4A1D4D8B
:100E70001D4C83B012682146009363202B46F1F786
:100E800061FCF0F7EDFF8146F0F7EEFF80460027AA
:100E9000D0F80960F3F798F84846F2F7E7FF4046C4
:100EA000F2F7E4FF08F0C8FFF760F1F70DF83760DC
:100EB000F0F7DEFF064601460120F2F7C7FF314694
:100EC0000220F2F7C3FF4FF49770084A2B461268CE
:100ED000214600906320F1F735FC03B0BDE8F083B4
:100EE0004C070020F0BB0100E0BB010050070020D0
:100EF00051222DE9F041304B82B000921A682F49FF
:100F00002F4B6320F1F71EFCFEF78CF80546F0F737
:100F1000AFFF044601462A460120F2F749FF2A4660
:100F200021460220F2F744FFF0F79AFF0746F0F758
:100F30009BFF044608F06AFF804608F06BFFC7F885
:100F40000D0008F06BFF2946C4F80D003846D4F8B0
:100F50000960F2F7B3FFF2F7DBFF29462046F2F70C
:100F6000ADFFF2F7D5FFF36803B33368DBB120467A
:100F70000221FFF7CDFC3946022322464046FFF707
:100F800055FCD8F82020F1682046FFF7A3FC7A2210
:100F90000C4B00921A680949094B6320F1F7D2FB08
:100FA00002B0BDE8F081F0F785FFE0E708F03AFF16
:100FB00008F04AFFF060D8E74C070020C0BB0100F2
:100FC000F0BB0100500700202DE9F047A8B0F0F772
:100FD0004BFF064607A8D6F80940FEF727F8D6F8D3
:100FE0000D30079A5968A36809780492276818ADEC
:100FF000CDE9025708AA0192E268C5B200920846FC
:101000001A222946FDF784FB65B1236803EB4501ED
:101010000239023B33F9022F002AB8BF52428B42F9
:101020001A80F7D101274FF0040AAB200621DFF820
:1010300080901C4AE3680590CDE90171CDE9032950
:1010400039462A46CDF800A06220F1F733FB4FF075
:101050000008AD20D6F80D20A3685168124A09781F
:10106000CDE904900392CDF800A02A46CDE901888D
:101070007220F1F71FFB02264FF0AF0C0B482368DC
:101080002A460390CDF81090CDE901783946CDF885
:1010900014C000966920F1F70DFB206828B0BDE868
:1010A000F08700BFD4C50100ECC5010004C60100F3
:1010B000F0BB010008B50220F3F7B0F8BDE8084026
:1010C000F3F73CB930B5044687B0FEF781FA8321C7
:1010D000012200230334094D0444059108480949BD
:1010E000CDE901330490039100922B461146642010
:1010F0002C70F1F7DFFA07B030BD00BF8407002085
:10110000F0BB0100FCAD01000148F6F7D1BC00BF07
:10111000400800202DE9F04F8FB006AFFEF758FAD7
:1011200001244FF00009D2220426DFF8B0C29E4D00
:1011300007F1200343F8140D21460592CDE903C5BC
:10114000CDE90149224600966420F1F7B3FA032263
:101150004FF0D40C954807F12003DFF8848243F860
:10116000102D214603900495CDE9014900962246B1
:10117000CDF814C06420F1F79DFAD8F80410FB688C
:10118000CA1D22F007023869ADEB020D034406AA1E
:1011900049457A60FB600DDD01EBD170A3EB600384
:1011A0001046DBB2084402F8013B824203F101031E
:1011B000DBB2F8D189000A3121F00701ADEB010D56
:1011C0000DF118094846F6F785FCDF22764B0092B0
:1011D000774900226420F1F7B5FA494607F1180271
:1011E000D8F804000124F6F7FDFC00264FF0040BAC
:1011F000E422704B07F1200A049521464AF8040DB9
:101200000592CDE9026322466B4B6420CDE900B420
:10121000F1F750FAE523D8F804200593674B2146EF
:10122000039364207B680495CDE901660094F1F78F
:1012300041FAE6236249D8F804206420059303911B
:101240004B4621460495CDE90146CDF800B0F1F7B3
:1012500031FAE82305935B4B22460393214607F1BD
:10126000180364200495CDE90146CDF800B0F1F7EC
:1012700021FAE923544A2146059303925346224614
:1012800064200495CDE90146CDF800B0F1F712FADB
:101290004846F6F785FCEE23324600934B49424B15
:1012A0006420F1F74FFAD8F804304946023B18465B
:1012B00007F11402C7E90563F6F794FC00B10138A1
:1012C000012400264FF0040BF822F861404807F192
:1012D000180305922146224603900495CDE9014664
:1012E000CDF800B06420F1F7E5F9F920334BD8F8D8
:1012F00004202146039305907B68CDE901660094A4
:1013000004956420F1F7D6F9FA202D4BD8F8042083
:101310002146039305904B46CDE90146CDF800B038
:1013200004956420F1F7C6F9FC20264B224603936E
:10133000214607F114030590CDE90146CDF800B030
:1013400004956420F1F7B6F9FD2040F201181E4B18
:1013500022460393214653460590CDE90146CDF838
:1013600000B004956420F1F7A5F9F969FB68194A02
:10137000DFF870E012680B4417485FFA83FC82F8CC
:1013800002C073460390CDE9016600940495CDF840
:1013900014802246214664208EF800C0F1F78AF9B5
:1013A0002437BD46BDE8F08FF0BB01000CBC010046
:1013B0001CBC010048BC01004408002054BC0100D2
:1013C00060BC01005CBC01006CBC01007CBC010085
:1013D000B4BC0100340A0020FCAD010000BC0100D7
:1013E000400800208407002040F2091330B50D4A60
:1013F0000D4D0E4C83B012682146009363202B469E
:10140000F1F7A0F9FFF786FE40F20D10084A2B46CF
:101410001268214600906320F1F794F9002003B090
:1014200030BD00BF4C070020F0BB0100D0BB010065
:101430005007002040F257132DE9F041174A184D8C
:10144000184C82B012682146009363202B46F1F7B6
:1014500079F9F0F705FD8046F0F754FD0746F0F7FF
:10146000EFFD0646F2F7B0FD4046F2F7FFFC3846C6
:10147000F2F7FCFC3046F2F7F9FCF0F76DFDF0F7FF
:1014800009FE4FF4B670084A2B46126821460090B8
:101490006320F1F757F902B0BDE8F0814C07002056
:1014A000F8BC0100BCBC010050070020CF222DE990
:1014B000F04FD44BADF66C0D00921A68D249D34B65
:1014C0006320F1F73FF9F0F7CBFCD0F80940F0F7D3
:1014D00019FDD0F809300425079308F0C7FCF0F790
:1014E000AFFDD0F8098008F0D5FC4FF470720021F0
:1014F0003AA808F002FD402200211AA808F0FDFCDD
:101500001E2200210AA808F0F8FC4FF47072002196
:101510000DF5956008F0F1FC402200212AA808F0A2
:10152000ECFC1E2212A8002108F0E7FCE268DDF8BE
:101530001CA00992043A08920DF6A60919AF0DF104
:10154000E606F2F7A9FEF2F7F9FEDDF820C00DF28B
:10155000E6446046A4F1400131F8022F50F8043F00
:10156000A14213440B80F7D140344C450CF1800C60
:10157000EFD1D8F810000DF14601043831F8022FF0
:1015800050F8043FB94213440B80F7D1DAF8103019
:101590000DF1A602A3F1040C32F8020F5CF8043F2F
:1015A000B24203441380F7D1013DCAD10DF2A640E7
:1015B0000DF6660600F1400530F9023F002BB8BF7A
:1015C00003339B10A8420380F6D1B042F2D10DF153
:1015D000460636F9023F002BB8BF03339B108E42FC
:1015E0003380F6D10DF1A60535F9023F002BB8BFC7
:1015F00003339B1095422B80F6D1F8F781FC0B2822
:10160000824F40F0F880F2F747FEF2F797FE4FF472
:1016100091723B4600927E4900226020F1F792F8D9
:101620002AAB0DF59562DDF820A00DF2E649A3EB9B
:10163000020B5046A646A9F140020BEB090132F914
:10164000023F50F8044F31F902CF1B1B9C45B8BF35
:101650000B809145F3D109F14009F14574460AF137
:10166000800AE6D1D8F810000DF146020DF12601EE
:10167000043832F9023F50F8044F31F902CF1B1BF6
:101680009C45B8BF0B80B242F3D1079B0DF1A60277
:1016900018690DF16601043832F9023F50F8044F21
:1016A00031F902CF1B1B9C45B8BF0B80AA42F3D176
:1016B0004FF0000A4FF0040B40F23713554A0593E0
:1016C0000392CDF800B0099B20220F2172200497CD
:1016D000CDE901AA4FF001097446F0F7EBFF4FF492
:1016E0009C714D4AD8F810307220CDF800B0CDE989
:1016F0000471039249460F22CDF808A0CDF804905A
:10170000F0F7D8FF40F23910079B444A1B6949465D
:10171000CDF800B00590039272202022CDE9019A05
:101720000497F0F7C7FF4FF0020B40F23B123C4B1F
:10173000CDE90472039320220DF595630F216220F9
:10174000CDE9019ACDF800B0F0F7B4FF4FF49E72E6
:10175000344B4946059203930F2212AB6220CDE928
:10176000019ACDF800B00497F0F7A4FF40F23D12C3
:101770002D4B49460592039320222AAB6220CDE9E6
:10178000019ACDF800B00497F0F794FF40F23F12B1
:10179000264BCDE90472039320223AAB0F21692036
:1017A000CDE9019ACDF800B0F0F784FF4FF4A072B4
:1017B0001F4B4946059203930F220AAB6920CDE9DE
:1017C000019ACDF800B00497F0F774FF40F241128F
:1017D000184B4946CDE90472039320221AAB6920C5
:1017E000CDE9019ACDF800B0F0F764FFF8F788FB77
:1017F0000B283FF408AF40F24F120F4B00921A68CB
:101800001CE000BF4C070020E4BC0100F8BC010054
:1018100084B401000CBD010020BD010034BD0100F5
:1018200048BD010058BD010060BD010068BD010058
:1018300078BD010084BD0100500700200449054B1C
:101840006320F0F77FFF00200DF66C0DBDE8F08FF0
:10185000E4BC0100F8BC0100A6222DE9F041554B83
:1018600082B000921A685449544B6320F0F76AFF23
:10187000FDF7D8FB0446F0F7F3FA0746F0F742FB12
:101880000546F0F7DDFB064608F0ECFAC5F80D005A
:1018900008F0FCFAC6F80D002046F0F737FB2046AA
:1018A000F0F7D2FB21463046F2F708FBF2F730FBA7
:1018B00021462846F2F702FBF2F72AFB214638467A
:1018C000F2F7FCFAF2F724FBF0F7CAFA0446F0F755
:1018D00019FB0646F0F7B4FB054608F0C7FA08F016
:1018E000D9FAFDF79FFB074600212078F2F76CFC40
:1018F00021463846F1F7C0FFD4F80130DB7A1BB13E
:1019000020782F49F2F760FCF2F7C6FCF2F716FDDB
:1019100000213078F2F758FCFDF784FB294A314664
:10192000F3F760FB30782849F2F74EFC0021287865
:10193000F2F74AFCFDF776FB224A2946F3F798FEB8
:1019400022492878F2F740FCF0F78AFA0446F0F7CB
:10195000D9FA0746F0F774FB054608F057FA8046B7
:1019600008F084FA064608F095FAD4F80D30046AB7
:101970001868D8F82020C1880830366AFEF7FEFDC6
:10198000D7F80D00324601890A30FEF7F7FDD5F889
:101990000D00224601890A30FEF7F0FDC9220C4BEA
:1019A00000921A680449054B6320F0F7CBFE02B0A1
:1019B000BDE8F0814C070020D0BC0100F8BC01005C
:1019C00081360000994200000D5200005558000079
:1019D000500700202DE9F04784B0F8F791FA35223E
:1019E000254B26490092054600226420F0F7AAFE06
:1019F000FDF7EEFD224A234B10701C68FDF7E8FD51
:101A0000214EA070DFF88CA00024DFF86C90DFF886
:101A100088801E4FFEB1102C1DD833689847AC4209
:101A200001D0F8F763FA0125CDB94FF0CD32394630
:101A30001748FBF707FDF8F763FA8442F4D0B36860
:101A400003909847FAF782F90398254604465AF816
:101A50002460002EDFD1F8F753FA0446F7E74B2253
:101A60004B460092414600226020F0F76BFE7368FF
:101A700098470546D9E700BFF0BD0100F8BD010059
:101A800084070020340A002040070020AC440020D6
:101A9000AC340020ACBD010084B4010084B02DE959
:101AA000F0438FB0BDF8A2C2B29DDFF8D0E005FBD5
:101AB0000CF58EFB0564EF17B5F5C84FC7EB64173F
:101AC0004FF00006B4BFB8464FF0FF08B39C054680
:101AD00004FB0CF00DF15C0CB0F5C84FCDE90866C5
:101AE000CDE90A668DF82080CDE90C668CE80E0001
:101AF0003DDA8EFB003EC417C4EB6E14E4B201263F
:101B00004FF000087022DFF878901A4B05923146AA
:101B10003246CDE90339CDE9018808AB009664204F
:101B20008DF82A40F0F7C6FD04244FF0750C1248DA
:101B30000EAB43F81C7D3246314600940390CDF83D
:101B40001090CDE90168CDF814C0642008ACF0F71E
:101B5000B1FD0FCC2860696003CC28612846AA60DB
:101B6000EB6069610FB0BDE8F04304B07047FF243B
:101B7000C5E700BF90BD010070C501001F85EB5196
:101B8000F0BD0100472370B50E4A0F4D0F4C82B0D7
:101B900012682146009363202B46F0F7D3FDF0F73F
:101BA0005FF90646F2F710FA3046F2F75FF94F2078
:101BB000074A2B461268214600906320F0F7C2FDC9
:101BC00002B070BD4C0700203CBE010020BE0100E9
:101BD00050070020382370B50F4A104D104C82B0CA
:101BE00012682146009363202B46F0F7ABFDFDF70A
:101BF00019FA0646F0F734F901463046F0F7E4FEEC
:101C00003F20084A2B461268214600906320F0F7D7
